:10000000802C0020194D0000BDA60000ED4C000022
:10001000ED4C0000ED4C0000ED4C00000000000035
:10002000000000000000000000000000094A00007D
:10003000ED4C000000000000B1490000ED4C000054
:10004000BD4A0000BD4A0000BD4A0000BD4A000094
:10005000BD4A0000BD4A0000BD4A0000BD4A000084
:10006000BD4A0000BD4A0000BD4A0000BD4A000074
:10007000BD4A0000BD4A0000BD4A0000BD4A000064
:10008000BD4A0000BD4A0000BD4A0000BD4A000054
:10009000BD4A0000BD4A0000BD4A0000BD4A000044
:1000A000BD4A0000BD4A0000BD4A0000BD4A000034
:1000B000BD4A0000BD4A0000BD4A0000BD4A000024
:1000C000BD4A0000BD4A0000BD4A0000BD4A000014
:1000D000BD4A0000BD4A0000BD4A0000BD4A000004
:1000E000BD4A0000BD4A0000BD4A0000BD4A0000F4
:1000F000BD4A0000BD4A0000BD4A0000BD4A0000E4
:1001000053B94AB9002908BF00281CBF4FF0FF317E
:100110004FF0FF3000F00CB8ADF1080C6DE904CEE3
:1001200000F008F8DDF804E0DDE9022304B07047D0
:10013000704700BF2DE9F04786468C460846089E6A
:10014000154674461946002B40F0C2808542B2FA2B
:1001500082F245D94AB1C2F1200300FA02FC2EFA1C
:1001600003F3954043EA0C0C94404FEA154EA8B2B5
:10017000BCFBFEF8230C0EFB18CC08FB00F943EA8D
:100180000C43994528D9EB1808F1FF3704D299455B
:1001900002D9A8F102072B44A3EB0903A4B2B3FBD5
:1001A000FEFC0EFB1C330CFB00F044EA0344A042AF
:1001B00014D92C190CF1FF3304D2A04202D9ACF1AE
:1001C00002032C44241A43EA07401EB1D440002302
:1001D00034607360BDE8F0874746DDE76346F1E7CA
:1001E00092BB431B01214FEA154EAFB2B3FBFEFC9D
:1001F000200C0EFB1C330CFB07F840EA0343984528
:1002000062D9EB180CF1FF3004D2984502D9ACF159
:1002100002002B44A3EB0803A4B2B3FBFEFC0EFBCD
:100220001C330CFB07F744EA0344A7424ED92C19B0
:100230000CF1FF3304D2A74202D9ACF102032C44E3
:10024000E41B43EA0040C0E7C2F1200320FA03F1B7
:10025000954090402EFA03F303434FEA154EAFB298
:10026000B1FBFEFC0EFB1C10190C0CFB07F841EA5D
:100270000041884504FA02F422D969180CF1FF30D4
:1002800004D2884502D9ACF102002944A1EB08014F
:100290009BB2B1FBFEFC0EFB1C110CFB07F743EA03
:1002A00001439F420ED9EB180CF1FF3104D29F425B
:1002B00002D9ACF102012B44DB1B41EA004192E779
:1002C0006046E3E76146F7E76046A3E76346B7E7C2
:1002D000834206D916B9002108467BE7C6E900E04B
:1002E000F9E7B3FA83F78FB9834201D3724508D88F
:1002F000BEEB020460EB030301209C461EB9002103
:1003000068E73846FAE7C6E9004CF8E7C7F1200C81
:10031000BB4022FA0CF41C432EFA0CF120FA0CF329
:10032000B84001434FEA14490EFA07F5B3FBF9F858
:100330001FFA84FE09FB18300B0C08FB0EFA43EA87
:1003400000439A4502FA07F240D9E31808F1FF305A
:1003500004D29A4502D9A8F102002344A3EB0A0370
:1003600089B2B3FBF9F809FB183308FB0EFE41EA2A
:1003700003418E452CD9611808F1FF3304D28E4514
:1003800002D9A8F10203214443EA0040A0FB0298ED
:10039000A1EB0E014145CE46434602D306D14D4561
:1003A00004D2B9EB020E68EB04030138002EA6D08C
:1003B000B5EB0E0261EB030101FA0CFC22FA07F324
:1003C0004CEA0303F940C6E9003198E74046C5E727
:1003D0004346D9E7014B1B681B681847700800208B
:1003E000014B1B685B68184770080020014B1B68B5
:1003F0009B68184770080020014B1B68DB68184792
:1004000070080020014B1B681B691847700800200A
:10041000014B1B685B69184770080020014B1B6883
:100420009B69184770080020014B1B68DB6918475F
:1004300070080020014B1B681B6A184770080020D9
:1004400018B1034B1860002070476FF0150070471B
:1004500070080020F0B5354F0028A7F108040646C3
:100460000CBF27460426A4F11C05002A38D095F8B5
:100470004D4038797F798000974214BF603030302A
:10048000C0B200F18040012700F5C04007FA04FC2B
:100490004FEAC40E002A3CD02C6D0022C4F8402143
:1004A000D4F84021C4F84035D4F8002242F48072D8
:1004B0003A43C4F800220EF1804202F5F83204F506
:1004C000A073C2F81035C2F81405194806F180432C
:1004D000C0F804C539B903F5805327601F60F0BD2B
:1004E00095F84E40C5E795F84C50EA0002F180427D
:1004F00002F5F83203F58053C2F81015C2F814451E
:1005000005F5117207FA05F540F82230C0F80455D8
:10051000E5E70EF1804303F5F833C3F81015C3F88F
:100520001405034BC3F804C5D9E700BF240000201D
:1005300000F0014038B5144BBFF35B8F15460C46F5
:10054000022253E8001F012904D143E8002CBCF12A
:10055000000FF6D1BFF35B8F13D10C4B18600C4B1F
:1005600001461C6001222B460020FFF773FF0CB9E7
:10057000002038BD00222B4621461046FFF76AFFB7
:10058000F6E76FF00F00F4E7740800207C08002005
:100590007808002008B5074B0246D3F8500600F053
:1005A00001001AB108F031FD0B3808BD08F011FD4B
:1005B000FAE700BF00100040F8B5174BBFF35B8FA0
:1005C000164607460D46022253E8001F012903D1B3
:1005D00043E800200028F7D1BFF35B8F18D10F4804
:1005E000012108F017FD044680B90D4B1F600D4B2B
:1005F00001221D60394633461046FFF72BFF2DB10F
:100600003346224629460120FFF724FF2046F8BD45
:100610006FF00F04FAE700BF7408002010000020FC
:100620007C08002078080020064BBFF35B8F014652
:1006300053E8000F43E80012002AF9D1BFF35B8FA3
:10064000704700BF7408002010B5144BBFF35B8FD8
:10065000022253E8001F002903D143E800200028AC
:10066000F7D1BFF35B8F15D10D48012108F0D2FC03
:10067000044640B901460B4808F0CCFC044610B9CA
:1006800012200BF0EBFAB4FA84F04009FFF7CCFF2C
:10069000204610BD6FF00F04FAE700BF7408002079
:1006A0003C0000201000002010B50F4BBFF35B8F03
:1006B000022253E8001F012903D143E8002000284B
:1006C000F7D1BFF35B8F0BD10848002108F0A2FCE3
:1006D0000446003818BF0120FFF7A6FF204610BDD2
:1006E0006FF00F04FAE700BF740800203C00002000
:1006F000F0B5214BBFF35B8F87B00546022753E867
:10070000002F012A03D143E800710029F7D1BFF37C
:100710005B8F2DD11F2D28D8184E0021304608F0B0
:1007200079FC0446D8B9C0238DF8043001ABCDE97B
:100730000237012102ABBD4030468DF805500493CD
:10074000059108F067FC044648B956F8100C836818
:1007500004AA1D68A6F10C012346A84704460120FF
:10076000FFF762FF204607B0F0BD6FF01504F6E713
:100770006FF00F04F6E700BF74080020100000209F
:1007800010B42448244C90F84D30012101FA03F2B2
:10079000DB0003F1804303F5F833C4F80825002299
:1007A000C3F81025C3F81425C3F814251B4B1B6888
:1007B000B3B190F84C309940C4F80815D9009B00AB
:1007C00001F1804103F1804301F5F83103F5F8337D
:1007D000C1F81025C1F81425C3F81029C3F8102951
:1007E0000F4B1B6893B190F84E300B4901229A4091
:1007F000DB0003F1804303F5F833C1F8082500223C
:10080000C3F81025C3F81425C3F8142510BC012023
:10081000FFF70ABF0000002000F001407C08002024
:100820007808002038B504460220FFF7FDFE0228B4
:1008300005460FD044B1012C06D06FF015042846B0
:10084000FFF7F2FE204638BD2146044808F0E2FBDF
:100850000446F4E76FF00F04F4E700BF4400002003
:10086000154890F8283090F829109B0003F1804338
:1008700003F5C04381F00101D3F8102522F4801262
:1008800042EA0152C3F8102590F8203090F8211068
:100890009B0003F1804303F5C04381F00101D3F8CD
:1008A000102522F4801242EA0152C3F810250021DB
:1008B000103008F0AFBB00BF0000002070B5674DDE
:1008C0002B6DE86BD3F8042522F00302C3F804254E
:1008D000D3F8082522F00302C3F80825D3F8102521
:1008E00022F00F0242F00402C3F810250AF0D8FFEC
:1008F00018B96FF01204204670BD05F13C0008F0F5
:100900009DFB04460028F6D1686C0AF0C9FF002858
:10091000EFD005F1440008F091FB04460028EAD12D
:1009200005F1200006F032F94D4B984202D06FF0ED
:100930000504E0E7EB6A4B4EB34203D04A4C191B67
:100940004C424C4195F83030484803F01F0343EACD
:100950004413EB61012385F8213006F017F9404B71
:100960009842E4D16B6BB34276D03F4A9A1A534215
:10097000534195F8381095F821403D48EA6901F057
:100980001F0141EA4311012385F829305C4095F8A5
:10099000203069629B0003F1804303F5C0431202DB
:1009A000D3F810650640C3F81065D3F8106502F45B
:1009B0007C52324342EA0452C3F81025D3F8102582
:1009C00042F00302C3F8102595F828309B0003F18C
:1009D000804303F5C043D3F810250240C3F8102527
:1009E000D3F81025234842EA0122C3F81025D3F892
:1009F000102542F00302C3F8102506F03FFA184B09
:100A00009842064693D11C4806F038FAB042044694
:100A10008DD11A4806F032FAA04288D128690AF02E
:100A20003FFF00283FF465AF154808F007FB044678
:100A300000287FF460AF134806F08CFE2860002881
:100A40003FF475AF0AF02CFF00283FF452AFBDE829
:100A500070400D48FFF7F4BC00238AE70000002037
:100A60000000AD0B40C0000028C00000280000209E
:100A7000FFC0ECFF4D0000204E0000204C00002085
:100A8000100000208CCD000038C200001FB51448B3
:100A900008F026FB002004F07DFC28B9114805B0C1
:100AA0005DF804EB08F01CBB002301930393694637
:100AB0000123029308F084FB011E05DA0A4808F0BE
:100AC0000FFB05B05DF804FB029B9B07FCD103996B
:100AD00009B10648F3E7064808F002FBF1E700BF5A
:100AE00092CD0000AFCD0000D0CD0000EACD0000D7
:100AF0000ACE0000012910B50C4603D108F0BFFF53
:100B0000204610BD022907D91368064A012108F0C2
:100B100091FF6FF01500F4E702D15368024AF5E740
:100B20000020EEE71DCE000037CE000008B5054BD3
:100B30000F225A700821044B044A08F07BFF002062
:100B400008BD00BF580000204CCE00006ECE000053
:100B500008B5054B06225A700821044B044A08F0D8
:100B600069FF002008BD00BF580000207DCE0000B6
:100B70006ECE000008B5054B05225A700821044BC3
:100B8000044A08F057FF002008BD00BF58000020AD
:100B90009ACE00006ECE000008B5054B04225A70B4
:100BA0000821044B044A08F045FF002008BD00BF9F
:100BB00058000020B7CE00006ECE000008B5054BEF
:100BC00003225A700821044B044A08F033FF002026
:100BD00008BD00BF58000020D0CE00006ECE00003F
:100BE00008B5054B01225A700821044B044A08F04D
:100BF00021FF002008BD00BF58000020E9CE000002
:100C00006ECE000010B5054B054A00245C7008212B
:100C1000044B08F00FFF204610BD00BF5800002015
:100C20006ECE000002CF0000012910B50C4603D1A2
:100C300008F025FF204610BD022907D91368064A8F
:100C4000012108F0F7FE6FF01500F4E702D15368B8
:100C5000024AF5E70020EEE71BCF000037CE000088
:100C6000034BD8229A700821024B034A08F0E2BED7
:100C70005800002036CF000055CF0000034BE22281
:100C80009A700821024B034A08F0D4BE5800002095
:100C900063CF000055CF0000034BEC229A7008216F
:100CA000024B034A08F0C6BE5800002082CF000065
:100CB00055CF0000034BF0229A700821024B034AE3
:100CC00008F0B8BE58000020A1CF000055CF0000AA
:100CD000034BF4229A700821024B034A08F0AABE83
:100CE00058000020C0CF000055CF0000034BF82271
:100CF0009A700821024B034A08F09CBE580000205D
:100D0000DFCF000055CF0000034BFC229A70082172
:100D1000024B034A08F08EBE58000020FDCF0000B1
:100D200055CF0000034B00229A700821024B034A62
:100D300008F080BE580000201BD0000055CF0000F6
:100D4000034B02229A700821024B034A08F072BE3C
:100D50005800002036D0000055CF0000034B03227E
:100D60009A700821024B034A08F064BE5800002024
:100D700054D0000055CF0000034B04229A70082184
:100D8000024B034A08F056BE5800002072D0000003
:100D900055CF0000034B05229A700821024B034AED
:100DA00008F048BE5800002090D0000055CF000049
:100DB000034B06229A700821024B034A08F03ABE00
:100DC00058000020AED0000055CF0000034B072292
:100DD0009A700821024B034A08F02CBE58000020EC
:100DE000CCD0000055CF0000034B044A0821997075
:100DF000034B08F01FBE00BF5800002055CF000075
:100E0000EAD00000012910B50C4603D108F037FEE6
:100E1000204610BD022907D91368064A012108F0AF
:100E200009FE6FF01500F4E702D15368024AF5E7B6
:100E30000020EEE71BCF000008D1000008B5054BED
:100E400002221A700821044B044A08F0F3FD002026
:100E500008BD00BF580000201ED1000038D100009E
:100E600008B5054B01221A700821044B044A08F00A
:100E7000E1FD002008BD00BF5800002052D1000055
:100E800038D1000010B5054B054A00241C7008211C
:100E9000044B08F0CFFD204610BD00BF58000020D5
:100EA00038D100006CD1000030B5424D424A85B0C7
:100EB0000821044608F0BEFD6B780F2B27D8DFE829
:100EC00003F0081A261C1E20222626262626262661
:100ED00026243A4B3A4A0821204608F0ABFDAB786D
:100EE000082B16D8082B1DD8DFE803F0521C504EF3
:100EF0004C4A48462400334BECE7334BEAE7334B8C
:100F0000E8E7334BE6E7334BE4E7334BE2E7334ABA
:100F1000E1E7F42B40D007D8EC2B41D0F02B3DD0AB
:100F2000D82B3FD02E4A07E0F82B33D0FC2BF9D139
:100F30002C4B00E02C4B2D4A0821204608F07AFD6E
:100F40002B78012B30D0022B30D0002B30D1284B06
:100F5000284A2046082108F06DFDEB680293AB6833
:100F600001932B7900932046EB78234A082108F05F
:100F700061FD002005B030BD204BDCE7204BDAE7F7
:100F8000204BD8E7204BD6E7204BD4E7204BD2E7C5
:100F9000204BD0E7204BCEE7204BCCE7204BCAE7D5
:100FA000204BC8E7204BC6E7204BD1E7204BCFE7CB
:100FB000204ACEE75800002084D1000002CF000074
:100FC0006ECE0000E9CE0000D0CE0000B7CE00000B
:100FD0009ACE00007DCE00004CCE000091D10000E2
:100FE000B8D10000FDCF0000EAD0000055CF0000CE
:100FF0006CD1000038D10000F0D10000CCD000004E
:10100000AED0000090D0000072D0000054D000009C
:1010100036D000001BD00000DFCF0000C0CF0000A2
:10102000A1CF000082CF000036CF000052D10000D7
:101030001ED10000CED10000012938B505460C466E
:1010400003D108F01CFD204638BD022907D91368DA
:101050000D4A012108F0EEFC6FF01500F4E750682E
:1010600009F033FB5028034605D9084A01212846D8
:1010700008F0E0FCF0E7064A0821D0702846054A4F
:1010800008F0D8FC0020DFE71DCE00004BD20000A6
:10109000580000206DD20000012938B505460C46E5
:1010A00003D108F0ECFC204638BD022907D91368AB
:1010B0000D4A012108F0BEFC6FF01500F4E75068FE
:1010C00009F003FB5028034605D9084A01212846A8
:1010D00008F0B0FCF0E7064A082110712846054ADE
:1010E00008F0A8FC0020DFE71DCE00004BD2000076
:1010F0005800002087D20000012938B505460C466B
:1011000003D108F0BCFC204638BD022907D913687A
:101110000D4A012108F08EFC6FF01500F4E75068CD
:1011200009F0D3FA6328034605D9084A0121284665
:1011300008F080FCF0E7064A082190602846054A3E
:1011400008F078FC0020DFE71DCE00009FD20000F1
:1011500058000020C7D2000038B5114C05460021C8
:101160001822204609F06EFC042323700D4B5A7898
:101170006270DA7822711A7962719A68A2602046E8
:101180001A691B7D2261237500F08CFC064B01223D
:101190001A702846054A082108F04CFC002038BD8A
:1011A00080080020580000205E140020DED20000DD
:1011B00038B5114C054618220021204609F042FCA2
:1011C000032323700D4B5A7899686270A1601A79D5
:1011D0005988A180A27120461A691B7D226123755E
:1011E00000F060FC064B01221A702846054A0821CF
:1011F00008F020FC002038BD8008002058000020A6
:101200005E140020E8D20000014807F069BF00BF6B
:10121000F2D200001FB504460C22002101A809F0FB
:1012200011FC01A800F01CFD2046094A082108F025
:1012300001FCDDE90112204608F009FC2046039B71
:10124000044A082108F0F6FB002004B010BD00BFDE
:1012500011D3000024D30000012938B505460C46FF
:1012600003D108F00CFC204638BD022907D91368C9
:10127000154A012108F0DEFB6FF01500F4E7506815
:1012800009F023FA012805D9104A0121284608F05F
:10129000D1FBF1E74FF08044C0B200F0F9FCD4F884
:1012A00080350B4A03F001030821284608F0C2FBF1
:1012B000D4F87835074A284603F00103082108F0DE
:1012C000B9FB0020D0E700BF1DCE00003BD30000DB
:1012D00058D30000BAD3000008B5044A082108F02A
:1012E000A9FBBDE808400120FFF7A4B8E4D3000043
:1012F00008B5044A082108F09DFBBDE8084000201D
:10130000FFF798B801D40000014800F0EDBC00BF21
:101310008008002037B50E4B5B780F2B044614D1A4
:101320000B390F2911D90B251A23CDE90053094A8E
:10133000094B082108F07EFB084A2B46082120466D
:1013400003B0BDE8304008F075BB03B030BD00BF4E
:10135000580000201ED400004CCE000054D40000E1
:10136000F8B5134C237806461BB100F06FFC002340
:101370002370104D104CE9783046FFF7CBFF182250
:101380000021204609F05EFB6B7863706B88A380B8
:101390002B69236100272B7D23752046277000F0E1
:1013A00081FB3046054A082108F044FB3846F8BD69
:1013B0005E140020580000208008002067D4000040
:1013C0002DE9F041214C23780646884617461BB18B
:1013D00000F03CFC002323701D4D3046E978FFF7F8
:1013E00099FFB8F1020F09D930463B68194A01212B
:1013F00008F020FB6FF01500BDE8F081164C1822B4
:101400000021204609F01EFB012323706B786370D6
:10141000AB782371EB78A3712B7863712B6923610F
:10142000B8F1020F2B7D237505D1786809F04DF9CD
:101430000A4BA060E360084800F034FB3046084ADD
:10144000082108F0F7FA0020D6E700BF5E1400205C
:10145000580000201BCF0000800800200912000067
:101460007DD40000012970B506460C4603D108F072
:1014700006FB204670BD022907D913681A4A0121CC
:1014800008F0D8FA6FF01500F4E7506809F01DF97C
:101490005A2805D9154A0121304608F0CBFAF1E760
:1014A000134D144CE978E8603046FFF733FF1822FB
:1014B0000021204609F0C6FA052323706B7863707B
:1014C000AB7823712B786371EB78A371EB68A36021
:1014D0002B69236120462B7D237500F0E3FA064B30
:1014E00001221A700020C5E71BCF00009DD4000028
:1014F00058000020800800205E14002038B5124DEE
:101500002B7804461BB100F0A1FB00232B700F4D7C
:1015100020460F4CE978FFF7FDFE182200212046F7
:1015200009F090FA022323706B786370EB78637193
:101530002B7823712B69236120462B7D237500F0C6
:10154000B1FA002038BD00BF5E1400205800002012
:1015500080080020012938B505460C4603D108F063
:101560008EFA204638BD022907D91368094A01219D
:1015700008F060FA6FF01500F4E7506809F0A5F87C
:10158000054A0346107508212846044A08F052FA15
:101590000020E7E71DCE000058000020C3D4000063
:1015A000012938B505460C4603D108F068FA2046F3
:1015B00038BD022907D91368094A012108F03AFA0F
:1015C0006FF01500F4E7506809F07FF8054A03460C
:1015D000106108212846044A08F02CFA0020E7E7A9
:1015E0001DCE000058000020EDD4000008B5114BBE
:1015F00000224FF0FF31C3F80022C3F80813C3F8EC
:101600001021D3F8102101221A61D3F81021002AE9
:10161000FBD00022C3F81021D3F81031FEF7F2FE00
:10162000FEF7F6FE044B1B781BB9BDE80840FEF739
:10163000D7BE08BD001000405F140020124BD3F845
:10164000302110B5044642B110490022C3F83021C0
:10165000D3F830210A6801320A60D3F80C218AB12C
:101660000022C3F80C210A4AD3F80C311368013365
:101670001360A268934205D1FFF7B8FFE368BDE8A5
:101680001040184710BD00BF00100040A008002007
:10169000A40800201C4B73B518700C46FEF79AFE88
:1016A0001A4B1879FF2801D0FEF7B8FE184805F04C
:1016B000DFFF184B0021D3F80022C3F800124FF0CF
:1016C000FF32C3F80823D3F810054FF47A53C0B2A1
:1016D000A4FB0343C0F1200624FA00F203FA06F645
:1016E000A0F1200523FA05F53243012300932A4394
:1016F00007480AF0BFF806480AF0A2F8044802B00A
:10170000BDE8704005F0A6BF6014002098080020D6
:1017100094C60000008000401FB54C4B40F20122EF
:10172000C3F850260022C3F83425C3F83825C3F87F
:101730002C25012291420446C3F8302526D00229E7
:101740001ED0002967D1AB22C3F824254FF0AB325D
:10175000C3F81C2500210D22684609F073F93C4BA3
:101760000293062C4FF001038DF80C3013D8042C93
:1017700053D866D000238DF805304FF4837318E0FA
:10178000CC22C3F824254FF0CC32E1E76A22C3F81B
:101790002425304ADCE70F2CECD102238DF80530EC
:1017A0007F238DF808300023ADF80A308DF80C3017
:1017B0008523294A9DF80B1013809DF807309DF86A
:1017C00001205B0743EA02239DF8022043EA02431B
:1017D0009DF8032043EA02539DF8042043EA825314
:1017E0009DF8052043EA02639DF8062043EA8263E0
:1017F000164A43F00803C2F814359DF80A301B045A
:1018000043EA01639DF808100B439DF80C1043EA6E
:101810004163C2F8183504B010BD40F20233ADF890
:10182000043003238DF80730ADF80A30074B40F23F
:101830000312C3F834250022C3F838254FF48B7304
:10184000B7E78DF8053040F20713B2E7001000400B
:10185000FF0004011B81FE585C14002038B50546CA
:101860000C46FFF759FF0F2D194A14BFFF237E23A3
:101870001370012344B1CC21022C17D1FF2BD1547A
:1018800010D00133DBB2F9E71249C1F80041D1F8B9
:101890000001D1F800010028FBD0D1F80805D05490
:1018A000FF2B0CD10C4BC3F8042538BD012C09D1FA
:1018B000F021FF2BD154F5D00133DBB2F9E701332E
:1018C000DBB2E2E7FF2BEDD00133DBB2D4E700BFA0
:1018D0006115002000D0004000100040F8B5174FFF
:1018E0003B7805460E4673B1154C206818B9314651
:1018F000FEF79AFD20605DB122681249BDE8F8400C
:101900000020FEF779BDFEF765FD0028ECD0F8BD9C
:101910002079FF280AD03B7843B9FEF77FFD28B134
:1019200021790948BDE8F84007F0DABB226805498B
:10193000BDE8F8400020FEF759BD00BF5F1400204D
:101940009808002010110040ACDD00000F28084B63
:1019500006D1A1F10B020F2A05D801EB8101323922
:10196000C3F8081570470522C3F80825704700BF63
:101970000010004070B504460E461546FFF736FECF
:101980000A4BC3F81045D3F8002242F00102294661
:101990002046C3F80022C3F80C65FFF7D7FF2146A5
:1019A0000020BDE87040FFF799BF00BF0010004065
:1019B000F8B5134C054617460E46FFF717FEC4F858
:1019C0001055D4F8003243F02103C4F800320D4B17
:1019D000C4F8043539462846FFF79EFE31462846AE
:1019E000FFF7B4FF084B00221A604FF48053C4F88D
:1019F000043329460120BDE8F840FFF76FBF00BF60
:101A00000010004061140020A0080020B0F5A07F65
:101A100010B50C462CD10978032916D11C4B6078DF
:101A2000217901221A701B4B1A78FFF7A3FF627904
:101A3000A079174B0021197016490B780133DBB2DE
:101A4000834298BF1A460A7010BD04290BD1104B6F
:101A5000607801221A700F4B22791978FFF7A8FFDE
:101A600022796079E5E7BDE810400B4807F038BB04
:101A7000B0F5A27FE8D1FEF7C5FCFEF7C9FC074B25
:101A800007491A68BDE810400020FEF7AFBC00BF50
:101A90005F14002060140020EEDD00009808002094
:101AA000101100402DE9F743614D02692A60027D63
:101AB0002A710278052A3ED8DFE802F0030B474F6F
:101AC000565942790179407803B0BDE8F043FFF7F9
:101AD00051BF4479457807798679FFF787FD21461C
:101AE0002846FFF7BBFE062D524C27D8042D27D9D8
:101AF000D4F8003243F4001343F00103C4F8003279
:101B00003146C4F810552846C4F80C75FFF71EFF7F
:101B1000494A00231360C4F80C31D4F80C21082280
:101B2000C4F8042329461846FFF7D8FE414AD2F8E4
:101B30000C31002BFBD003B0BDE8F0830F2DD7D0C4
:101B4000D4F8003243F02103D8E702794179407894
:101B500003B0BDE8F043FFF72BBF8168407903B0C5
:101B6000BDE8F043FFF796BD81680079F7E7447858
:101B700090F8059090F8048087798668FFF736FD25
:101B800049462046FFF76AFE2A4BC3F81045D3F8B2
:101B9000002242F00302C3F800223946C3F80C8544
:101BA0002046FFF7D3FEFEF715FC2879FF2801D069
:101BB000FEF734FC286818B92146FEF735FC28608A
:101BC0001E4B1F4A1B5D12881E485343C6F1640416
:101BD0005C43B4FBF6F41C4405F04AFD1A4BD3F801
:101BE00000220022C3F800224FF0FF32C3F808237E
:101BF000D3F81035DBB2250FC3F12001240124FAFC
:101C000003F205FA01F1A3F1200025FA00F00A43DE
:101C100001210243009102230A4809F02BFE0948E2
:101C200009F00EFE074803B0BDE8F04305F012BD11
:101C30009808002000100040A40800202FDE0000BB
:101C40005C14002094C600000080004008B50348E2
:101C500005F00EFDBDE80840FFF7C8BC94C60000C3
:101C6000084B094AD3F8103503F00F030F2B14BFAC
:101C70004FF480737F23C0E90023044B1B6883600B
:101C8000704700BF0010004061140020A008002031
:101C9000D8B94FF08043D3F88025D20710D44FF045
:101CA0008052D2F83011082909D1D2F83421052AFE
:101CB00005D80C498A5C12B10122C3F838260120EC
:101CC0004FF08043C3F880057047012809D14FF0D9
:101CD0008042D2F8783503F0010383F00103C2F8A3
:101CE0007835704729DE000030B5134B01221A60A9
:101CF000124B134A85B0CDE9023002A904461148BF
:101D000005F05AFC104B9842014602D00F4807F0EC
:101D1000E7F9002500220621082008F0BAFC0C4A49
:101D2000009523460621012008F0BBFC012002F0AB
:101D3000D3FD284605B030BD00D0004004000200AD
:101D40000D1A000094C600000000AD0B08DE000074
:101D50003D1600000B6801330B60014B1B681847F0
:101D60007000002007B50B46002102460191034890
:101D700001A900F013F903B05DF804FB551D000044
:101D80002DE9F047058B04462807904611D4022917
:101D900005F0070540F0CD80204607F0AEF978B198
:101DA0000138218B042811D8DFE800F0C3106D85BD
:101DB000950001290CBF45F0100545F0200525834D
:101DC00088F31188BFF36F8FBDE8F08701F0070A31
:101DD000AA4500F0A6800027B9463E46A368002B1E
:101DE00000F0BD8041F00801218388F31188BFF322
:101DF0006F8FA168002900F0BB800D68002900F0FA
:101E0000B780D1F80480334652462046C047002DA3
:101E100076D02B6829461D46F0E701F007035A1FCC
:101E2000012A1BD8002221F00701062B276889B25E
:101E3000C4E9002209D13B4603E0628B1B680132F2
:101E40006283002BF9D141F002012183204607F083
:101E500054F900287BD041F0200177E0042B0AD10F
:101E600021F0070189B22183204607F046F910B11D
:101E700041F020012183218B01F0070AAA4550D0AF
:101E80000027B946AAE7236921F0070141F00601BE
:101E9000062DD3F8009021832DD1B9F1000F40D049
:101EA00041F00801218388F31188BFF36F8F3A490D
:101EB0002046C84729E021F00701236941F00401C9
:101EC00089B2042DD3F804902183E6D000273E4642
:101ED0004FF0040A82E721F00701236941F0050170
:101EE00089B2052DD3F808902183D6D000273E462D
:101EF0004FF0050A72E700273E464FF0060A6DE7ED
:101F00002B4687E7B9F1000FD1D14FF02003EFF353
:101F1000118883F31288BFF36F8F238B23F008039C
:101F20002383258BEA062ED525F01003238305F0A5
:101F300007056669218B002EBFF66FAF0023276867
:101F4000C4E9003321F0070141F001012183218B15
:101F500001F0070AAA454FF000097FF43FAF002FB8
:101F60009BD041F00801218388F31188BFF36F8F64
:101F7000002FC7D03D68394633465246204607F009
:101F8000E8F82F46F4E7AB067FF51AAF25F02003FB
:101F9000238305F00705FFE67F9100002DE9F04F50
:101FA000814695B08B4617461C460025387808B9FF
:101FB000284658E37B1C2528039306D05946C8477A
:101FC0000028C0F25083013504E2182200210EA837
:101FD00008F038FD7B78252B7DD00023781C9846AF
:101FE0009E469C461E46014610F8012B2B2A00F007
:101FF000A18000F29880202A00F09F80232A00F020
:102000009F802BB19DF8403043F040038DF8403065
:10201000B8F1000F05D09DF8403043F020038DF853
:102020004030BEF1000F05D09DF8403043F0100362
:102030008DF84030BCF1000F05D09DF8403043F0E2
:1020400008038DF840302EB19DF8403043F0040372
:102050008DF840309DF8403003F04400442803D10F
:102060006FF386138DF840309DF840302A2A43F0F4
:1020700080038DF840307FD19DF8412042F001026D
:102080004B1C8DF841201A782E2A9DF841200CBF58
:102090000121002161F341028DF8412078D15A7865
:1020A0002A2A6ED0013300224FF00A0C194611F88B
:1020B000010BA0F13006092E40F295809DF84010EA
:1020C0001292C1F3400040EAD2700A4660F3410226
:1020D0008DF840205CE0BA1C03928DF843309DF8E7
:1020E0004130DA0740F12E8154F8048BB8F1000F2B
:1020F00007DA9DF8402042F004028DF84020C8F134
:1021000000085E0740F1278154F804ABBAF1000FD4
:1021100080F226819DF841306FF341038DF8413004
:102120004FF0FF3A1CE12D2A0DD0302A7FF469AF21
:10213000012358E74FF0010C55E74FF0010E52E72D
:102140004FF001084FE701264DE70EFB0262303ADF
:102150000346184610F8016BA6F1300CBCF1090FCC
:10216000F3D999428FD09DF840101192D20F62F3AB
:1021700041018DF8401086E70B4600224FF00A0E11
:10218000E7E79DF8412042F004028DF84120023338
:102190001A786C2A47D02BD8682A31D06A2A4BD0BB
:1021A0004C2A51D01A4612F8013B0392782B9DF825
:1021B00041208DF8433000F2BE806D2B51D8692B41
:1021C00000F2B980572B67D8412B03D0453B022B37
:1021D00000F2B1809DF84230042262F302038DF8D0
:1021E0004230012373E00CFB0202303A0B465DE7FC
:1021F000742A25D07A2AD5D19DF8412006210CE0F9
:102200005A78682A9DF8412006D1012161F3C6025F
:102210008DF841200233C5E7022161F3C6028DF833
:1022200041200133BEE75A786C2A9DF8412001D144
:102230000421EBE70321F0E79DF841200521ECE7BD
:102240009DF841200721E8E7BDF8402022F4F04244
:1022500022F0020242F4804242F00202ADF8402035
:10226000DFE76E3BD9B201238B4040F282410B4243
:1022700037D113F0240F51D1D8075CD59DF84230E7
:10228000032161F302038DF8423002F07803A3F1D9
:1022900040014B424B411AE0A3F15801C9B2012061
:1022A00000FA01F111F4624F94D140F60106314277
:1022B0001DD111F4043F3ED09DF8423060F302037B
:1022C00002F07802402A8DF8423034D000239DF885
:1022D0004020C2F340010B4363F341028DF84020DC
:1022E000FDE69DF84230022161F30203E8E79DF824
:1022F0004210022002F0780260F30201402A8DF8B9
:10230000421002BF9DF8401041F001018DF84010CD
:10231000632BDBD1131E18BF0123D8E79DF8423091
:10232000032161F3020312F0780F8DF8423014BFDD
:1023300001230023CBE79DF8403043F001038DF8E3
:102340004030C3E79DF94020002AB4BFDDF8448047
:102350004FF0FF38D5E698077FF5E2AEDDF848A0EC
:102360009DF841100023CDE911339DF8423003F070
:102370000703012BC1F3C30133D1CB1E042B04D8B7
:10238000DFE803F0104646101000236801294FEAE9
:10239000E372CDE90E320BD103F0FF030E9300235D
:1023A0000F9307E054F8043BDA17CDE90E3202E050
:1023B000022911D004349DF8403013F0030647D0B1
:1023C000039B3A465946484606F0A2FF0028C0F251
:1023D0004A810544039FE9E51AB20E9243F3C033E4
:1023E000DEE7022B24D1CB1E042B04D8DFE803F058
:1023F000181010181800012954F8043B4FF000027F
:1024000014D00229CDE90E32D5D19BB20E93D2E77A
:10241000073424F00704F4E80223CDE90E23CAE7C9
:1024200054F8043B0E9300230F93C4E7DBB2BCE7E0
:10243000042B08D1073424F00704D4E9002308341E
:10244000CDE90E23B7E7032BB5D154F8043BDDE704
:102450009DF843007828BDD862281CD825283FF471
:10246000ADAD5828B6D10DF136030093DDE90E016C
:1024700008AB10AA06F006FFBAF1000F074680F27B
:102480009A80002FA6D00DF13603D81B002E00F045
:10249000C1800130BEE0633815289BD801A252F8F4
:1024A00020F000BF792500008B250000D523000017
:1024B000D5230000D5230000D52300008B25000084
:1024C000D5230000D5230000D5230000D52300002C
:1024D00019260000B1250000D7250000D5230000F3
:1024E000D5230000FD240000D5230000B125000005
:1024F000D5230000D5230000B1250000BAF1000F5C
:102500000E9F35DB5146384608F041FA07EB000ACA
:10251000002F3FF45FAF00269DF8423013F0100209
:10252000059200F0938002305B06119A48BF129B1F
:102530000492104448BFC018B8F1000F40F3A080C7
:102540009DF84020A8EB0008C2F3800350070693D3
:1025500000F19680510640F189803EB159463046DF
:10256000C84700287FDB069B01351E4630227EE0EF
:10257000384608F005FAC9E70E9B8DF82030002692
:1025800008AF0DF1210A0120C6E719075CBFC3F3AC
:1025900000135E01DDE90E2348BF2B26002BBFF69A
:1025A00062AF524263EB4303CDE90E232D265AE777
:1025B000002658E700269DF840200DF13603DB1B6E
:1025C0006FF386129A458DF840207FF65AAFAAEB3A
:1025D0000303119355E70E9890B30DF13603009362
:1025E00010AA08AB002106F04DFEBDF8423003F002
:1025F000EF0343F4F04343F01003BAF1000F074632
:10260000ADF84230D6DA00283FF4E4AE0DF13603DF
:10261000181A00269A467FE70E9B07293FF6DAAE86
:10262000DFE801F00C04060C08080C0C1D70D1E664
:102630001D80CFE6EA17C3E90052CBE61D60C9E66C
:102640002E4F064607F1050A052065E71A0748BF21
:10265000013069E70793104606925946C84700289B
:10266000DDE9062304DA15B0BDE8F08F20224346E9
:102670001946002903F1FF33ECDC45446D1A9846F6
:102680002EB159463046C8470028ECDB01359DF88D
:102690004230DA0601D41B0705D559463020C84719
:1026A0000028E0DB0135059B33B19DF84300594616
:1026B000C8470028D7DB0135049E2E4405E0594663
:1026C0003020C8470028CEDB0135731B002BF6DC19
:1026D00053463A465946484606F01AFE0028C2DBE1
:1026E0000544A844A8EB0503002B7FF773AE5946B9
:1026F0002020C8470028B6DB0135F3E73FDE0000A5
:1027000008B54FF02002EFF3118382F31288BFF374
:102710006F8F02F083FC034806F0E2FC02F0B0F891
:10272000FCE700BF45DE000013B5044605F0D0FA13
:10273000C0F307230193C0F307430093044A030E39
:102740000821204607F076F9002002B010BD00BF36
:102750006EDE000038B5044609F07EFA4FF47A7553
:10276000A0FB052305FB0133D20B42EA434320467D
:10277000024A082107F05EF9002038BD87DE00001C
:1027800010B5044603F01CFE084A03460821204603
:1027900007F050F9064A2046082107F04BF9054892
:1027A000214605F023F9002010BD00BF96DE000091
:1027B000B5DE0000B9270000F0B587B0D0F8A070F2
:1027C00004460D4609F0F8F8064605F091FE234B45
:1027D000234A002E08BF1E46224BCDE90046844204
:1027E00018BF1346082128461F4A07F023F9D4E9E9
:1027F0000A23CDE9022394F90E300093237B1B4A70
:102800000821284607F016F9204605F037F9626ED0
:1028100000920346164A0821284607F00BF905A93D
:10282000204609F0D9F8034630B1124A082128465B
:1028300007F000F907B0F0BD059A6423B91ACDE995
:1028400000214B430C4AB3FBF7F30821CDE9027397
:1028500028463B4607F0EEF8ECE700BFC1DE00007B
:102860000EE60000BFDE0000C4DE0000D0DE000087
:10287000FCDE000013DF000040DF000070B5134EE7
:1028800088B004460146124805F0B0F807AA4FF494
:102890000061304609F094F807996422C1F50060A0
:1028A00042434FF400630025D20ACDE90303CDE98A
:1028B000013105922046074A0095A6F12003082120
:1028C00007F0B8F8284608B070BD00BF201F0020F0
:1028D000F528000077DF000010B5044608F0A4FDDD
:1028E000034A03460821204607F0A4F8002010BD43
:1028F000BDDF0000F0B5D0F8A06089B004460D46F9
:1029000007A909F069F8034630B1104A08212846A2
:1029100007F090F809B0F0BD204609F04DF80C4FD3
:10292000079A002818BF0746B11A6423CDE902218F
:102930004B43CDE90076B3FBF6F3064ACDE90463D9
:1029400008212346284607F075F8E3E713DF000067
:10295000C1DE0000D3DF00000346006810B50C465E
:10296000114608B1027822B9024A204602F02AFB39
:10297000204610BDDDE0000010B50C68D1E9011261
:10298000FFF7EAFF034A03460821204607F052F802
:10299000002010BDE2E000002DE9F0478AB00546B6
:1029A00001A804F0C9FE019E1B4ADFF87080DFF821
:1029B0007090DFF870A0182303FB006608212846FA
:1029C00007F038F8019CB44203D300200AB0BDE8F8
:1029D000F08705AF394614222046FFF7BDFF424677
:1029E00003460821284607F025F8204608F058FF3E
:1029F0000D4A00280CBF4B4653460821284607F0D5
:102A000019F8142320460949049302AACDE9025774
:102A1000183408F04FFFD6E701E100000BE1000099
:102A2000F8E00000F2E0000010E100007929000069
:102A30002DE9F043114BDFF8489053F82140013164
:102A400087B053F8218006460027A04503D83846B2
:102A500007B0BDE8F083204608F022FF054658B1D4
:102A6000142201A92046FFF777FF4A4603460821B2
:102A7000304606F0DFFF2F461834E6E7E0C70000D7
:102A800017E1000010B5082104461E4A06F0D2FFE7
:102A900000212046FFF7CCFF20B91B4A0821204621
:102AA00006F0C8FF08212046184A06F0C3FF01219E
:102AB0002046FFF7BDFF20B9134A0821204606F043
:102AC000B9FF08212046124A06F0B4FF0221204631
:102AD000FFF7AEFF20B90C4A0821204606F0AAFFF6
:102AE000082120460B4A06F0A5FF03212046FFF7E8
:102AF0009FFF20B9044A0821204606F09BFF0020D2
:102B000010BD00BF1DE100002CE1000034E1000019
:102B100043E1000051E100008B1E022B2DE9F04142
:102B200007468846144637D860681022002107F00F
:102B300064FEB8F1020F064607D1264A2023082179
:102B4000384606F077FF336816E00A220021A068B5
:102B500007F053FEC5B21F4A2B460821384606F03F
:102B600069FFB8F1040F1AD0102D0DD0202DEAD036
:102B7000082D0CD13378DBB2174A0821384606F00D
:102B800059FF0020BDE8F08133889BB2F4E7134A77
:102B90000821384606F04EFF6FF01500F2E7E068B6
:102BA0001022002107F029FE0D4A034604460821A1
:102BB000384606F03FFF102D06D0202D07D0082DF7
:102BC000E5D1E4B23470DCE7A4B23480D9E73460F4
:102BD000D7E700BFB5E10000E0E10000CAE1000076
:102BE000F1E1000070B5104E044633780D4681B116
:102BF0002BB1BDE870400D4A012106F01BBF012337
:102C000033700B4A0821204606F014FF012333706D
:102C100004E083F001033370002BF2D129462046F3
:102C2000BDE8704006F040BF6116002005E20000DC
:102C300040E2000070B504463C480378182B02D1EE
:102C40000B78112B31D0013A0B468D18AB4225D1B0
:102C50008B5C0A780370A2F13003092B344C04D941
:102C600022F02003413B052B04D823683149CA5484
:102C7000013323602368022B34D110222D48002118
:102C800007F0BBFD2C4A136803F8010B13602B4AB5
:102C90001368013313600023236023E013F8016BF2
:102CA000182ED3D11E78112ED0D1244D244A2B6852
:102CB0000821204606F0BEFE20460021FFF792FFC5
:102CC000204B187870B9204A2B681168042B0ADC55
:102CD00008B111602B6013F003010BD11268136867
:102CE0001BBA136070BD086800BA41F8040B043BBE
:102CF0000120EBE75B4203F0030358BF594202296E
:102D000004D1126813885BBA9BB2EAE70329E9D1C0
:102D1000106802681104C2F3074301F47F010B43FA
:102D200002F47F4213430360DCE700BF6216002019
:102D3000A808002064160020B4080020AC08002079
:102D40006AE2000063160020B00800202DE9F84F69
:102D50000D462B49DFF8AC80DFF8AC90DFF8ACB063
:102D600000230B602A4988F8003006460B601446A1
:102D7000012D274654F804AF1ED902224946504679
:102D800007F01AFE80B922689278003A18BF012233
:102D9000924420490222504607F00EFE30B901232A
:102DA00088F80030013DE3E70022F1E7494650464C
:102DB00007F0F6FDA8B9043700221146786807F03D
:102DC000A7FC154B002211461860786807F0A0FC9C
:102DD000124B134918603046FFF704FF0020BDE88E
:102DE000F88F9AF800202D2AE6D19AF80120002ABF
:102DF000E2D053465A460821304606F01BFED1E782
:102E0000A80800206316002084E200008AE2000087
:102E1000AC08002087E20000B4080020B0080020C1
:102E2000352C000013B5094808F03AFD58B1084A9E
:102E300006491268074800240094012300F062FD4F
:102E4000204602B010BD6FF01200FAE770C000001B
:102E500038C80000B8C0000010B50C4611464268E2
:102E60001068C0E90041916883600023C1E9023322
:102E7000C1E905334B600B61D168C1E90233C1E997
:102E800005334B600B61C360A36823B19B6C13B126
:102E9000044920469847A3689B6A0BB1204698478F
:102EA000002010BDB797000010B5816804460831B6
:102EB00001F0B8F8A168034A20460831BDE8104087
:102EC00001F050B83BE30000014906F01DBD00BF12
:102ED00075DF00008368022210B51A719A6B0446F0
:102EE000BAB983F84220DA63D3F86432DB040BD535
:102EF0000321084B084A07F065F9A0686FF4805178
:102F000000F5197006F0D5FC2046BDE8104001F030
:102F10000BB810BD49E300000DE1000037B50446D1
:102F20008068D0F864325A070D4605D5002106F0B6
:102F300029FDE06807F0B8FAE368DB686BB9002D9B
:102F400037D0A068423006F0D9FCA36898B303F1EB
:102F5000420103F5A17007F0E7FCA268E0680DF1FB
:102F600006034232294607F0A2FA58B9A06800F5D4
:102F7000A171423007F0D8FCA068423006F0BEFCD8
:102F8000ADF80600204607F06CF8A368D3F860326D
:102F90009B0603D50949606906F0B6FC204600F09F
:102FA000B1FEA368BDF80620DA879A87204606F0AE
:102FB000C3FF03B030BD83F84201CEE7F0C100008B
:102FC0002DE9F04F00239FB0CDE905338368044617
:102FD0004233029307F04BF8204606F099FF10B9F0
:102FE0006069FFF771FFA06814220021083007F024
:102FF00029FD204606F037FFA168E0688A8F42313C
:10300000002607F08BFA204607F009FB4FF0FF3847
:10301000B146039611AFB2463546B346DDE90532F7
:10302000012A61D00B2B62D8B8F1000F20D1BAF180
:10303000000F09D0204607F013FBA2680C23423290
:1030400011A905A806F09BFD059DA0681EAB03EB2A
:103050008503002243F8342C4369002B40F0B980EB
:10306000C6B1C368B3422BD00D9600F1080522E02B
:10307000029A0223394606A806F081FD06997A686D
:103080000292034631B101290AD148B1714A204662
:1030900007F098F86FF0070528461FB0BDE8F08FDD
:1030A000059B002B32D0386800F0E0FF98B166B184
:1030B000A5680D9608350CAE0FCE0FC533682B6092
:1030C0002046FFF7F1FE0125E6E7634A012120468D
:1030D00007F078F8DEE7059BC3B13A682946204639
:1030E00001F02CF9022809D1059B0B2B9FD9069BD7
:1030F000022B9CD1594B5A4A0121C8E7032805D01D
:10310000059B013305934FF0010A87E7039B2BB919
:10311000396807AA584606F027FE0546043708F125
:10312000FF38002D37D0EB68BAF1000F08D013B389
:10313000204606F09CFF204606F0FEFE494AC5E701
:10314000CBB1A368DDF81490AE4603F1080CBEE8DD
:103150000F00ACE80F00DEF80030CCF80030AB68B0
:103160004BB96B7CFE2B01BF95F8108009F1010370
:1031700008F1FF380593D5F804C0BCF1000F08D062
:10318000AE46BEE80F000CAE0FC6DEF8003033606E
:103190006646AB4603E0059B63B101230393069BA0
:1031A000B8F1000F02D1022B7FF438AF059B013339
:1031B000059333E7A368DB6913B1DB68002BECD11F
:1031C000294B0093294A119B0121204606F0FAFF62
:1031D000E3E7037EA5EB0905B3B1417E4FF6FF722D
:1031E000FF2918BF0A469D4202D313449D420BD9C2
:1031F00083681F4A0121204606F0E4FF2046FFF7BE
:1032000053FE6FF0150547E74FF4006100F51970A4
:1032100006F040FBA06800F53E7006F0CCFBA3680A
:1032200011AA294602EB89025B69204698470546A8
:10323000A0684FF0FF324FF0FF3300F53E7006F00C
:1032400070FBA0686FF4006100F5197006F031FBA7
:1032500022E700BF8DE30000A1E3000002E40000CC
:1032600019E10000BFE30000EEE3000084E6000087
:1032700026E400002DE9F04F04468068A9B0012142
:1032800000F5197006F006FBA3681B79022B17D115
:1032900000230993A36860689E6B03681D6909ABEE
:1032A000C6B110221BA9A847099A4AB11BA92046FA
:1032B000B047A3689B6B002BECD12046FFF70AFEBA
:1032C000A0686FF0010100F5197029B0BDE8F04F5A
:1032D00006F0EFBA01220DF12301A847099B002B4C
:1032E000EED09DF923209DF82330A068002AD1DB81
:1032F0004279032A00F2F782DFE812F004007B0231
:103300009202F5020D2B66D00A2B56D0B0F864223B
:10331000092B6FF3CA02A0F8642200F082803DD826
:10332000002BB7D0082B00F0F281D0F8602297076D
:10333000B0D5013B162BADD801A252F823F000BF47
:10334000BD38000049370000513700004137000008
:10335000B13800006F370000953200009532000050
:103360009532000095320000773700007F3700006B
:1033700095320000A937000095320000B3370000F5
:103380009532000095320000953200009532000021
:10339000B737000095320000E33700001B2B3DD00B
:1033A0007F2B00F0C081A3F120025E2ABDD801214D
:1033B00006F0E8FA9DF82310E4E0D0F86422C2F3A6
:1033C000C7029AB1D0F86422C2F3C7020A2A0DD00C
:1033D000D0F860325EE7D0F86422C2F3C7022AB1A7
:1033E000D0F86422C2F3C7020D2AF0E7B0F86422D5
:1033F000818F63F3CA02A0F8642259B906F0C2FAB9
:10340000E06807F051F86069FFF75EFD2046FFF7BE
:1034100061FD3FE72046FFF7D3FDF7E70123437146
:1034200038E7D0F860329E077FF534AF012106F00F
:10343000A9FAA068838FFF2B3FF42CAFC28F00F155
:10344000420100F5A17007F0F2FAA268D38F13448D
:10345000002583F842511BA90C2302F5A1720BA889
:1034600006F08DFB0B990C293FF614AF28AB03EB4C
:10347000810343F8345CA368DA8F134493F8413036
:10348000202B02D0093B042B46D8002947D1002528
:103490000A950A9B28AA02EB8303002653F834AC52
:1034A000504606F02BFAB3460290B046374616AAAD
:1034B0003946284600F0C0FB814600283BD1012E4A
:1034C00064D10A9B28AA02EB830353F8340C06F05C
:1034D00015FAA268064608324146284600F0ACFBC1
:1034E0000546006806F00AFA864206D02968821B63
:1034F00092B23144204606F0A3FEA068C38F034475
:1035000093F84230202B02D0093B042B29D801210B
:10351000204606F044FDBDE60129B8D90139002056
:103520000CAB009301900AAB1BAA06F03DFC0546CC
:103530000028AED1AEE6029AD9F80000514607F055
:103540003BFA60B9D9F8000007F01AFA584538BFBD
:1035500058461FFA80FB002E08BFB84601360137D7
:10356000A5E7D0F86032DD070BD5002106F014FA8C
:103570002021204600F0A4FCA068012106F00CFAEE
:1035800088E62021204600F09BFC83E67FF682AE91
:103590000A9A28AB03EB8202C24652F8343C0293EB
:1035A000184606F0ABF9A2680490A2F83090039692
:1035B000A26851460832284600F03EFB029B0746AF
:1035C0000AF1010A002B51D13B68002B58D1A268A7
:1035D0001386039B013B0393EAD16069FFF774FCF8
:1035E000204600F0A1FC0A9B28AA02EB830308F105
:1035F000010A53F8340C06F081F9414611AA8146BC
:10360000284600F019FB0746A0683968FF2200F53C
:10361000A17007F093F93B6802934FF6FF77B84625
:1036200016AA514628460AF1010B00F005FB0028B6
:1036300061D0A168036801F24111002211F801EF85
:10364000985C704503D110B101324245F6D1B9F111
:10365000000F01D04A4507DBBA4206F1FF36A8BF8A
:103660003A46012E97B246D0DA46D9E700680028DC
:10367000AAD0049A029907F09FF90028A4D097E7EE
:103680009A48069306F03AF9A16800EB0B0292B251
:1036900096484F8D079206F031F9069B0590184623
:1036A00006F02CF9079AA168059BA2EB0009088E89
:1036B000FF1A97FBF2F7BFB200F1010EB0FBF7F271
:1036C00007FB120080B2069BA1F830E01FFA89F9CF
:1036D00058B90093864A854B0621204606F072FDB4
:1036E0004946204600F0F8FA73E7824A0621204650
:1036F00006F068FDF4E7002F3FF4CCAD0299A7EB8C
:10370000090292B24944204606F09AFDC2E5D0F87B
:10371000603299077FF5BEAD012106F033F92046EE
:1037200006F0ABFDB6E5D0F860329A077FF5B2AD92
:10373000012106F027F9A368D3F860321B07EED405
:10374000204606F07FFDA5E5204606F097FCA1E5A2
:10375000204606F08CFC204606F0DAFB10B96069C2
:10376000FFF7B2FBA068012106F00CF94EE62046F7
:1037700006F08CFC8EE5204606F091FC8AE5D0F838
:1037800060329E0603D55C49606906F0BDF8A36807
:10379000D3F860329D0603D55849606906F0B4F845
:1037A000204600F0C1FB75E500212046FFF7B6FB7F
:1037B00070E50121F9E7204606F053FCA0680023DC
:1037C00080F84230C363012106F0DCF8A368D3F827
:1037D000603298067FF55EAD4949606906F094F85D
:1037E00058E5204600F0D4FAA068012106F0CAF896
:1037F00050E55B2B01D1022311E6D0F8602291073E
:1038000006D5622B08D14FF0FF31204606F0EBFBC6
:10381000A36800225A713DE5662BF9D10121F4E736
:1038200000224271D0F8602292077FF533AD313B20
:103830001B2B3FF62FAD01A252F823F0B938000040
:10384000C5380000D7380000AD38000095320000C0
:10385000953200009532000095320000953200004C
:10386000953200009532000095320000953200003C
:10387000953200009532000095320000B337000009
:10388000A93700006F37000049370000953200006B
:10389000B138000095320000BD38000095320000BC
:1038A0009532000095320000C938000003234371AF
:1038B000204606F0DCFBEDE403234371204606F0CE
:1038C000D0FBE7E403234371D0F8601201F001015B
:1038D00081F0010152E603234371D0F860329B0767
:1038E0007FF5D8AC2CE7002399E500BF0DE600007A
:1038F00041E400000DE10000F5C10000FAC1000044
:10390000F0C100002DE9F043044680688846D0F8F5
:103910000C1389B015461F46002961D14FF444723B
:1039200007F090F8A3682268E0681A6006F05DFE70
:10393000A06800F53E7008F063F84FF42A794FF460
:103940001A76A068304408F0DBFAA06800228319D8
:1039500001214844103608F0B6FAB6F52A7F09F17D
:103960001409EED1A369A068002602211E6000F5AB
:10397000197005F08FFFA3681B4A9A62186805F05A
:10398000BDFFA368194A83F82C00606866F38205BE
:10399000C3F86052036841461D682346A8470546A0
:1039A000D0B9A36801221A71D4E9090100220023C9
:1039B000CDE906230E230393109B0495CDE90173F3
:1039C00000940B4B4FF4006204F0FAF8A368216AEC
:1039D000C3F80C0304F042F8284609B0BDE8F083B0
:1039E0006FF07705F8E700BF180050002799000036
:1039F000413A000010B5044680680379012B19D1C3
:103A00004FF0FF324FF0FF3300F53E7005F089FFB5
:103A10000821204600F07EF90849606905F074FF2E
:103A20002046FFF757FAA06800F53E7005F0C3FF87
:103A3000002010BD6FF08500FBE700BF74DF0000C1
:103A4000F8B504464068036800219B689847002841
:103A50003FD12046FFF7CEFF00283AD11D4F1E4E22
:103A6000A06800F52A704FF0FF324FF0FF330321BA
:103A700004F004FF0546A0684FF0FF324FF0FF331B
:103A800000F53E7075B105F04CFF20462B46134AF9
:103A9000012106F097FBA068BDE8F84000F53E70F4
:103AA00005F089BF05F03DFF606803685B6903B1FD
:103AB00098473A462046022105F00AFF2046324642
:103AC000002105F005FFA06800F53E7005F073FFCA
:103AD000C6E7F8BD3B9900007532000047E40000DE
:103AE00010B50D4A0446082105F0A4FF20460B4AF4
:103AF000082105F09FFF2046094A082105F09AFF9A
:103B00002046084A082105F095FF2046064A002174
:103B100000F028FA002010BD5EE400009CE40000E4
:103B2000FBE400004FE50000E9E50000F8B51E46A3
:103B300017460B462F4A0821044605F07BFF6EB35B
:103B40003B782D4A0821204605F074FF01256A07BD
:103B500004D12A4A0821204605F06CFFAE4223D941
:103B60007B5D254A0821204605F064FF0135102DB4
:103B7000EDD1234A0821204605F05CFFD6B91F4A43
:103B80000821204605F056FF0125AE422B4613D8EA
:103B90001A4A0821204605F04DFF18E0194A08216D
:103BA000204605F047FF0125164A0821204605F06A
:103BB00041FFDBE700252B46FB5CA3F120025F2AD7
:103BC00028BF2E23104A0821204605F033FF013577
:103BD000102D07D06B07D8D1084A0821204605F0E0
:103BE00029FFD2E72046094ABDE8F840082105F040
:103BF00021BF00BFFFE5000006E600000EE6000062
:103C000010E600000CE6000032E6000012E60000BC
:103C100010B5044613460A4601460648FEF7BEF9AB
:103C200023691B7923B12046BDE8104005F03FBF52
:103C300010BD00BFC79A000010B50B46144660B90E
:103C40000F4A1049891AB3EBD10F02D30024204642
:103C500010BD02EBC3025468F9E781680029F5D072
:103C60004A68097831B11846214690472368002BED
:103C7000EDD1EBE714214B43D418D358F7E700BF3D
:103C8000E4C00000B4C100008368D3F860329B0632
:103C900003D50249406906F01AB9704700C2000016
:103CA000014906F014B900BF75DF00000A1E0DDCE3
:103CB0000ED042238168D1F86012890608D5002A07
:103CC00004494069B8BF524206F001B94123F1E707
:103CD000704700BF2EE600000A1E0DDC0ED0442304
:103CE0008168D1F86012890608D5002A0449406924
:103CF000B8BF524206F0EBB84323F1E7704700BF6C
:103D00002EE60000826802494069423206F0DFB8C0
:103D10000DE1000008290A4616D8836893F82E1092
:103D2000914211D0082A83F82E20D3F8603205D0B2
:103D3000990609D50549406906F0C9B89B0603D51F
:103D40000349406906F0C3B8704700BF35E600007C
:103D500005C2000038B50D4609780446FFF7DAFFC2
:103D60006A78072A10D8A36893F82F1091420BD0D5
:103D700083F82F20D3F860329B0605D5606903498C
:103D8000BDE8384006F0A3B838BD00BF3EE60000ED
:103D9000F8B583689A8FD98F0446002A4FD000293E
:103DA0004DD0413103F142050B441846A84206D3D9
:103DB000014611F80169202E38D0A84238D286B2C7
:103DC0009DB2AB1B9BB2591C471CD21A014438460A
:103DD00006F016FEA268938F711B13FA81F39BB253
:103DE00093871A44002382F8423009B2204606F035
:103DF000D6F8A368D3F860329A0603D510496069F3
:103E000006F065F83B460F4A0821204606F0DAF92D
:103E10002046FFF739FFA368D3F860329B060ED522
:103E200060690949BDE8F84006F051B80846BDE7A9
:103E3000014611F80169202EC1D00846BDE7F8BD42
:103E40000AC200000DE100000EC200002DE9F041A1
:103E500004460D4617460AB1FFF716FFA368DA8F2E
:103E6000D3F86012423213444A071FD5184606F0B1
:103E700087FDDFF84480064696B9A3689A8FDA87F3
:103E8000204606F031F820B107B115B16069FFF79F
:103E900007FF6942204609B2BDE8F04106F07FB84D
:103EA0006069414606F013F8013EE5E7034A082140
:103EB000204606F087F9E0E7BFDE00000DE10000D4
:103EC00013B583688DF80710D3F860220446D00735
:103ED00021D5D98F9A8F8A421DD0481C19449DF84C
:103EE0000720D88781F84220D3F86012890710D5BF
:103EF000D3F8603260690B4913F0040F18BF2A220F
:103F000005F0E5FF204606F003F810B16069FFF701
:103F1000C7FE02B010BD01220DF10701204606F0D8
:103F20005EF9F6E732E6000083680A4A1B6810B5BE
:103F30000446022106F046F9A368D3F860329B07D5
:103F400007D52046FFF7DEFE2046BDE8104006F00C
:103F500003B810BD0DE10000014906F09FB900BF94
:103F600075DF00002DE9F04F0E4600218BB00446AE
:103F700017460D4605AA304601F10108FFF75CFE21
:103F8000A0B985B127B13A460821204606F01AF9B2
:103F9000214FDFF888B0002105AA304601F1010A5F
:103FA000FFF74AFE60B90BB0BDE8F08F006810B1B2
:103FB00006F0E6FC80B2854238BF05464146D9E7A7
:103FC0000368D0F804900393384606F0D9FC039BAD
:103FD00080467BB11A786AB1CDE90053104A3B465E
:103FE0000821204606F0EEF8B9F1000F04D160690F
:103FF000FFF7B2FF5146CFE75A4620463B4608211D
:1040000006F0E0F86A1C02EB480292B249462046EC
:1040100006F051F9EEE700BF60E600004EE6000052
:1040200047E60000F7B5064608680D46B8B106F049
:10403000A7FC84B20B4F384606F0A2FC00972B6811
:10404000094A04440821304606F0BCF8A4B2696865
:104050002246304603B0BDE8F04006F02CB90446D5
:10406000E8E700BF5CE6000042E4000010B5074945
:10407000044606F095FC38B10549204606F090FC50
:10408000B0FA80F0400910BD0120FCE752E60000C4
:1040900055E6000010B58368D3F860329B060446ED
:1040A00003D50449406906F07AF9A368024A9A6286
:1040B000002010BD12C200001800500008B583692E
:1040C000034A1B68082105F0B5FC002008BD00BFAD
:1040D00063E600007FB50F4E04460025A268E06845
:1040E0000DF10E0302F5A172012106F0E0F9BDF811
:1040F0000E00A36850B103F5A173009332462B461E
:104100000821204605F096FC0135E7E783F84201D7
:1041100004B070BD73E60000022907B50DD15368E5
:1041200001930E4B009313680D4A012105F082FCA8
:104130006FF0150003B05DF804FB8368094AD3F8FB
:10414000603213F0020F4FF00801074B08BF13460F
:10415000064A05F06FFC0020ECE700BF8AE600008D
:1041600081E600007DE6000078D600009FE60000B2
:1041700010B58368D3F860329A06044603D5074920
:10418000406906F00CF9A368D3F860329B0603D5AA
:104190000349606906F003F9002010BD19C2000050
:1041A0001EC20000F0B5012985B004460CD053684A
:1041B00001935B4B009313685A4A012105F03AFCC6
:1041C0006FF0150005B0F0BD8368D3F86032990632
:1041D00003D55549406906F0E2F86FF0F901204631
:1041E000FFF764FDFA212046FFF776FDA068002561
:1041F0004FF48072294600F5A1708DF80B5006F03F
:1042000021FC4A49606906F0CAF8606905F04FFC74
:104210004FF47A766068036801221F690DF10B0183
:1042200003ABB847039BDBB9013E4FF47A70B6B2DB
:1042300007F014FD002EEDD1A368D3F860329B0681
:1042400003D53B49606906F0AAF8A368394A9A6227
:104250002046394A032105F0EDFB6FF00700B1E776
:104260009DF80B20A3681B2A4ED093F842111B29FE
:10427000D0D1522A48D11D44002285F8422193F81A
:1042800043115B2949D103F243101646022510F869
:10429000011F2A463B2905F10105ADB21ED1FF2AB7
:1042A000CAD002F5A17213FA82F1002211F8010FAF
:1042B000F0B9FA2A28BFFA22FA2E5A85324628BFC8
:1042C000FA221A8583F84201D3F860329A0603D5A0
:1042D0001749606906F063F8002073E706EB860271
:1042E000303901EB4201B5F5807F8EB2CFD1A3E723
:1042F000013502EB8202ADB2303800EB4200B5F579
:10430000807F82B2D2D197E759190135ADB2092D1C
:1043100081F842217FF67EAF002283F842218BE7AD
:104320008AE6000081E6000024C20000EAE6000000
:1043300028C2000018005000B0E600002DE9F04F40
:10434000074689B01546894621B90324204609B09D
:10435000BDE8F08F104606F04EF90028F5D04FF07A
:1043600000084146022424E05C463CE029460AF568
:10437000A17006F0B9FA064600284CD006F000FB02
:1043800082B2601C01323146304406F039FB2246CD
:104390005946304606F04BFB4FF020033355BAF830
:1043A000403001331C44AAF8404008F101080024C1
:1043B00001994B1C03AA48460193FFF73DFC0646B2
:1043C000E8B131680022284605F08DF90028EFD1C8
:1043D000D6F800B0D7F808A0BBF1000FC4D05846FB
:1043E00006F0CEFA84B2BAF840302344FF2BBDDD8C
:1043F0000A4A2B460321384605F0E4FE0124B8F1B1
:10440000000FA3D0B8682A4600F1400100F5A17062
:1044100005F083FC9AE70224F1E700BFB3EA00004D
:104420002DE9F84305464FF02003EFF3118683F39F
:104430001288BFF36F8F0E4B0E4F1C68DFF8388069
:104440004FF00C092CB986F31188BFF36F8FBDE8CC
:10445000F883D4E90123002D18BF13462BB198F837
:10446000142009FB02F2B85C98472468EAE700BF11
:10447000F00B0020E40B0020401200200A4ABFF39A
:104480005B8F430902EB830200F01F00012383408E
:10449000DB4352E8000F184042E800010029F8D140
:1044A000BFF35B8F704700BFE00B002070B5194B66
:1044B0001C7DBFF35B8F04F01F0301229A40164B53
:1044C000610903EB8103D04353E8001F01EA0005B3
:1044D00043E80056002EF7D1BFF35B8F0A4213D09A
:1044E0000E4B0F4D8BB10C236343EA18E85C5178F7
:1044F00006F0CAFA0020FFF793FF0C235C432A1949
:1045000000232B51C2E9013370BD83F31188BFF33F
:104510006F8FEFE740120020F80B002089AA0000FF
:10452000E40B00202DE9F843324B334A1C7DBFF3E6
:104530005B8F63094FEA830852F823302F4EBFF395
:104540005B8F04F01F0943FA09F313F0010F0746CC
:104550000AD10146204600F069F828B107C80C23AB
:1045600003FB046383E807000C236343F218F55C44
:104570002DB92046FFF782FF2846BDE8F8837B1C53
:1045800010D0D2F808C01E4D1E4A4FF40040002142
:10459000ECFB005100232846FBF7B2FD0121381A3D
:1045A00007F03AFB03F0CCFE0120FFF739FFBFF321
:1045B0005B8F154B9844012303FA09F358E8002F49
:1045C0001A4348E800210029F8D1BFF35B8F0F4B55
:1045D00033B10C236343F218F05C517806F048FACB
:1045E000FFF764FF2046FFF749FF03F0BDFE0120FF
:1045F000C3E700BF40120020E00B0020E40B0020C6
:104600003F420F0040420F00F80B002071AA00004B
:10461000054BBFF35B8F53F82000BFF35B8F00386F
:1046200018BF0120704700BFFC0B00202DE9F74F99
:10463000884601A900F042F8441E24B204EB440469
:10464000DFF86C900546A40025B92F46384603B024
:10465000BDE8F08F019B185D1F19FFF7D9FF0646D3
:1046600010BB7868134A4FF4004ACC463146E0FB51
:104670000AC100236046FBF743FD8346B8680D4A34
:10468000CC463146E0FB0AC100236046FBF738FD0B
:10469000094B1B685A1C01D0834205D9B8F1FF3F72
:1046A000D4D058444045D1D9013DADB20C3CCBE704
:1046B0003F420F0040420F00F400002008B9024BB7
:1046C0000B600020704700BF88CA0000014804F05A
:1046D000F1BA00BF88CA000010B5044618B90D4BE6
:1046E0000D485B689847616831F004030CD00829D5
:1046F0000AD011F0020108D00848214607F02CF931
:10470000002323600023636010BD2068142206F09C
:1047100099F9F7E7EC02002005EB000018110020E2
:1047200008B508B34368042B10D101220368BFF316
:104730005B8F53E8001F002903D143E800200028C5
:10474000F7D1BFF35B8F0BD1002008BD53B10068D8
:104750004FF0FF324FF0FF3303F0DAFA0028F3D0C6
:104760000348F2E70348F0E76FF4E040EDE700BFED
:10477000E98FFFFFEA8FFFFF08B5C0B14368042B44
:1047800010D100220368BFF35B8F53E8001F01299B
:1047900003D143E800200028F7D1BFF35B8F09D194
:1047A000002008BD43B1006803F02AFBF8E76FF46E
:1047B000E040F6E70148F4E70148F2E7E98FFFFF40
:1047C000EA8FFFFF10B5044618B9164B16485B6810
:1047D00098476368042B23D0082B21D0CBB92368DA
:1047E000BBB912484FF0FF324FF0FF33214603F0C0
:1047F000CFF808B923681BB90A4B0D485B68984786
:1048000020681422002106F01DF9636843F00203BA
:104810006360206807F0F4F8636843F001036360A5
:1048200010BD00BFEC02002005EB000018110020B5
:104830002BEB000008B5064906484023142207F078
:1048400070F8BDE808400449044804F093BA00BF7A
:10485000180C00201811002090CA0000A4CA000003
:10486000034B43F8302003EBC0035960704700BF8F
:104870004C030020014910220A60704710ED00E04F
:1048800072B6404080F31188BFF36F8FBFF34F8F34
:1048900030BF62B6BFF36F8F704700BF72B649403A
:1048A00081F3118820BF80F3118862B6704700BF82
:1048B0000028ACBF00F16040064B4FEA4111ACBF8D
:1048C00000F5614000F00F00C9B2B4BF195480F880
:1048D0000013704714ED00E040B2002807DB044AE3
:1048E0004109012300F01F00834042F82130704746
:1048F00000E100E040B200280CDB4309064900F06B
:104900001F0020330122824041F82320BFF34F8F44
:10491000BFF36F8F704700BF00E100E0054B420915
:1049200000F01F0053F82220012303FA00F010408A
:10493000704700BF00E100E030BFFFF7FDBF00BFE0
:104940000B4A08B50B4B22F07F029A60BFF34F8FE2
:10495000BFF36F8FD3F8882022F47002C3F8882049
:1049600002F042FF03F032FE00F0CAF902F084FFC9
:104970000000000000ED00E00A4A0B499368096856
:10498000C3F8B0100949C3F8AC004B6843F080533A
:104990004B60002383F31188BFF36F8F9368D3F8C4
:1049A000B00070474012002000CD000000ED00E094
:1049B00013498A684FF030001044EFF3098C80E807
:1049C000F01F202080F31288BFF36F8F0D4F4FF040
:1049D0000066CA698A603E60D2F8AC000023C2F863
:1049E000AC3080F3118804B5104600F02DFABDE814
:1049F000044002F1300090E8F01F8CF30988704702
:104A00004012002004ED00E01EF0040F0CBFEFF395
:104A10000880EFF30980816911F8021C0229FFD098
:104A200001B505F032FE01BD42F8203C009B42F882
:104A30001C3C0A49019B42F8183C029B42F8143C7A
:104A400021F001014FF0807342F8043C42F8081C49
:104A50000023203A0265C0F8AC3070477192000024
:104A60000A4A0346906878B113F1160FD0F89C00FB
:104A700005D0A0F120029A4205D8834203D2814298
:104A800028BF002070470020704700BF4012002060
:104A900008B5094B98600D46144600F0D5F920463C
:104AA00085F30988002163B681F31188BFF36F8F06
:104AB0000022002304F0DCFB4012002001B572B696
:104AC0000B4A906900281EBF0021916106F089FF02
:104AD00062B6EFF30580A0F110004FEAC00005496F
:104AE000014409C99847BDE801400349084700004F
:104AF000401200204C030020FD4A0000044B99683E
:104B0000D869884203D003494FF080520A60704749
:104B10004012002004ED00E00D4B9A6A9A6A9A6AEE
:104B2000920508D59A6B9A6A120404D518B19A6A4C
:104B300022F400429A629A6A9A6AD205044A58BFDD
:104B40009B6A936A002043F47F4393620870704726
:104B500000ED00E01D4B70B515469A6A9A6A9A6A94
:104B60009207064622D5586B9A6A14061ED519B1CB
:104B70009A6A22F080029A629A6A9A6A9A6A134C36
:104B800012F0100F15D19B6A990712D40020A36A66
:104B90000E4A9B0642BF636A23F400536362936A22
:104BA00043F0FF03936200232B7070BD6FF015007C
:104BB000E2E763681A05E9D53146FFF751FF00289F
:104BC000E4D080F309880220E1E700BF00ED00E0B7
:104BD00070B5414B5B688AB00546C3F308030026F5
:104BE00086F31188BFF36F8F02F07F40B0F17F4FE3
:104BF00011D102F00C0008280DD010074CBF0D4653
:104C000001260022033B8DF80720032B3BD8DFE869
:104C100003F00453575B3546F3E72F4BDA6A9107ED
:104C200031D4DA6A002A2EDBDA6A52002BD5AA695F
:104C300032F8021C4DF6027291420AD093F82820F5
:104C40004AB10DF1070201212846FFF783FF044610
:104C50001AE02C6818E093F829202AB10DF1070119
:104C60000120FFF759FFF2E75A8D92B25AB19A6AC2
:104C70009A6A9A6A9A6A9A6A9A6A9A6A6FEA02427F
:104C80006FEA12429A6200249DF8073093B92022FD
:104C9000294602A805F0CBFE099BBEB1C3F308026A
:104CA00022B96FEA53236FEA4323099302A92046EE
:104CB00005F0E9FC0AB070BD0DF107020021C3E761
:104CC0000DF107010020CCE7034BD0E723F4FF737D
:104CD00023F00103E9E700BF00ED00E0024A536959
:104CE00043F010035361704700ED00E0EFF30880DC
:104CF000EFF3098101B57246FFF76AFF01BD00BFFE
:104D0000044800232021C2180133302B82F80013FD
:104D1000F9D1704700E100E0002080F31488BFF370
:104D20006F8F07F02FF9002011490860BFF34F8FF4
:104D3000104880F3088800F033F8202080F31188B1
:104D40000D484FF0AA014FF4026205F07BFE0A48BD
:104D50004FF40261401880F30988EFF314800221B8
:104D6000084380F31488BFF36F8FFFF7E9FD00005D
:104D700094ED00E0802C0020001F00200749D1F8AE
:104D800090200023C2F307221846934200DB7047AD
:104D9000C1F89830C1F8A0000133F6E700ED00E05B
:104DA00008B572B6002383F31388FFF7E7FF144BAF
:104DB0004FF0FF32C3F88020C3F88420C3F8882066
:104DC000C3F88C20C3F89020C3F89420C3F898202F
:104DD000C3F89C20C3F88021C3F88421C3F888213C
:104DE000C3F88C21C3F89021C3F89421C3F898210B
:104DF000C3F89C2162B6BFF34F8FBFF36F8F08BD1E
:104E000000E100E0084B9B6883420BD1EFF3058380
:104E100043B1064B5A6842F080525A605A6A22F4F3
:104E200000425A6203F06ABB4012002000ED00E02D
:104E3000024B034A0348012100F072B8000004202D
:104E400000000020B4CA0000D0F89C20054B203A96
:104E50001A60054A2021C3E901121846012100F019
:104E600069B800BF3411002000000B15F0B5204ECA
:104E700000258D4201DB1046F0BD446874B353B188
:104E800004F1FF3C14EA0C0F2FD11F2C2DD9076819
:104E90001CEA070F29D1202C0768D0F808C05FFA58
:104EA00082FE1ED9B4F1004F1DD8013CB4FA84F43F
:104EB000C4F11F046400BEF1070F4CEA040C14D8BF
:104EC00027F01F04144344F01004C6F89820C6F8D5
:104ED0009C404CF00104C6F8A040013201350C3072
:104EE000C7E70824E7E73E24E5E76FF01502C2E7CD
:104EF00000ED00E0044B0522C3F89420BFF34F8F70
:104F0000BFF36F8F704700BF00ED00E0BFF35F8F0E
:104F1000024B0022C3F89420704700BF00ED00E070
:104F200010B5034C01232278FFF7A0FF207010BDBD
:104F30008416002008B5094A00231278FFF796FF6F
:104F400010F1160F02D0064A072800DD08BDC2F88E
:104F50009800C2F8A0300130F6E700BF84160020A8
:104F600000ED00E014490868082810B521D8FFF7C3
:104F7000CDFF124C49680022904201F10C0105D18D
:104F80000F4B1870FFF7B6FF002010BDC4F8982033
:104F900051F80C3C23F01F03134343F01003C4F8F3
:104FA0009C3051F8043C43F00103C4F8A0300132B6
:104FB000E2E74FF0FF30E8E7C0CA000000ED00E094
:104FC000841600200CB41FB509B90DF10300CDE91A
:104FD000020107AB069A0648019302A9FCF7DEFF1F
:104FE000029B00221A7005B05DF804EB02B0704716
:104FF00057AA00004FF02002EFF3118382F31288CA
:10500000BFF36F8F044A0121C2F8401583F3118862
:10501000BFF36F8F0020704700E001404FF08043E6
:10502000C0B2C3F81C05BFF34F8F0549054BCA68D2
:1050300002F4E0621343CB60BFF34F8F00BFFDE784
:1050400000ED00E00400FA0520B1034B800143F0BD
:1050500001031847704700BF30C20000084B70B50D
:10506000C31A0D4607499B1004465943064840227F
:1050700005F02CFD2B4601462046BDE87040184740
:1050800054110020B76DDBB610C0000073B50C4C96
:105090000C4A4023041B00930D460B460A49A410FA
:1050A00061430646094805F03EFD011E05DA30461B
:1050B0002B4602B0BDE87040184702B070BD00BF7B
:1050C0005411002093AB0000B76DDBB610C0000098
:1050D00010B506F0C1FD4FF47A72A0FB0203074C35
:1050E00002FB0131C00B40EA4140C90BC4E9000199
:1050F000BDE81040012006F054BA00BFF8050020BA
:10510000002270B501210446104605F0C2FA0F488E
:1051100001F00AFB0E4B984215D106F035FA2669CC
:105120000C49304604F039F800280BDB24690949A2
:105130000125356404F11C0004F02FF8002801DB80
:10514000E564002070BD6FF00400FBE78D510000A6
:105150000000AD0BE0CA000001460C2309484B4398
:1051600070B5C418D4E90E5600224033A263184427
:1051700005F099FC2DB132462B460348BDE870403E
:10518000184770BD5411002010C0000010B1012854
:1051900004D07047034B1B6C5B0701D1FFF7DCBFEA
:1051A000704700BF5411002008B54FF02003EFF303
:1051B000118183F31288BFF36F8F114A136843F094
:1051C00002001060DA0707D481F31188BFF36F8FF4
:1051D000BDE80840FFF77CBF4FF08043D3F80C24B4
:1051E000D3F80C34D307EFD5064805F05CFC81F307
:1051F0001188BFF36F8F0020BDE80840FFF7ACBFF8
:10520000A4110020941100207FB500220123CDE9D4
:10521000022304ABCDE90433094ACDF800D06B4634
:10522000CDF804D005F0AEFC002805DB4FF4804239
:105230000023684602F04EFE07B05DF804FB00BF95
:10524000B1AB00002DE9F74F4FF080480546D8F884
:10525000186406F480364FF02003EFF3118783F3D0
:105260001288BFF36F8F06F0F7FC4FF47A72A0FB41
:10527000024302FB0133E40BD8F80C9444EA4344A4
:10528000D8F80C34234BD3F800B0234BD3F800A04C
:1052900087F31188BFF36F8F204ADFF88480214F96
:1052A0002846082104F0C6FB19F0010FDFF87890BA
:1052B0001E4AB9F81A30009328460CBF43463B46B5
:1052C000082104F0B7FBA4EB0B03009328465B46D0
:1052D000174A0821A4EB0A0404F0ACFB5346284605
:1052E000144A0094082104F0A5FB2846124A08211C
:1052F00004F0A0FBB9F83630009328460B4A002E84
:105300000CBF43463B46082104F094FB002003B049
:10531000BDE8F08FF8050020F00500206CEB0000E0
:1053200067EB000076DF00005411002077EB0000EF
:1053300091EB0000B3EB0000D4EB000010B506F0D9
:105340008BFC4FF47A72A0FB0203074C02FB013185
:10535000C00B40EA4140C90BC4E90001BDE8104060
:10536000012006F05AB900BFF0050020084BBFF33A
:105370005B8F53E8002F22F0020143E80010002861
:10538000F7D1BFF35B8FD30701D4FFF7D7BF7047C7
:10539000A4110020024AC3B21C2003FB0020704766
:1053A000541100202DE9F0413849BFF35B8F0746C7
:1053B000012251E8003F41E800200028F9D1BFF365
:1053C0005B8F33B9324933484B60CB608A6003F05E
:1053D000F7FE7B1E012B2BD8012F07D14FF0804306
:1053E000D3F81C3403F00303012B21D006F0DEFABE
:1053F0000546F8B9284B1B78E3B14FF080430222F1
:10540000C3F808230646DFF894804FF08044D4F8B0
:105410001834D4F81824D20316D503F00303012B53
:1054200001D0012F10D15DB386F31188BFF36F8FC8
:10543000BDE8F0814FF02003EFF3118683F312886B
:10544000BFF36F8F0125DEE7ADB13046FFF726FAD7
:10545000D4F81835002BDAD1D4F80421002AD6D09C
:10546000C4F80431D4F804310123C4F81835C8F85D
:105470008031A360CBE70021212003F01FF8E7E78C
:105480004FF080430222C3F80423D1E750110020DB
:105490004011002070110020C516002000E100E03E
:1054A00030B54068057B01F01F04B2F5001F85B0E0
:1054B00044EA451404D1204601F0B6FB00204AE03E
:1054C0000025B2F5800FCDE9025514D1B3F1007F6C
:1054D0000CBF042305238DF808300023194602AAC7
:1054E000204601F0E1F9204B98423AD101212046B3
:1054F00001F052FBE2E7B3F1C06F2ED0B3F1007FB1
:1055000014BF012302238DF808308368CB40D907EC
:10551000E3D4B2F1A07FE0D16209012A04F01F03B5
:10552000124A03F5E07318BF4FF0A04252F823303F
:10553000DB07D2D40DF107052946204601F0D8FA41
:105540000B4B98420BD1284601F020FB064B9842AA
:1055500005D06FF00B0005B030BD0323D3E70395F2
:10556000BBE76FF00400F6E70000AD0B000300504E
:105570000400AD0B10B501F0F9FA044668B901F06A
:10558000CDFA084B98420AD10748214601F0AAFA01
:1055900022460521062005F07CF8002010BD6FF0A2
:1055A0000400FBE70000AD0BAD550000420970B5EB
:1055B000034602D0012A17D070BD0D4E32695168E2
:1055C0000029F9D003F01F0301250C689D40002934
:1055D000F2D08A682A4002D04B68304698472CB1F6
:1055E000236821461C46F2E7024EE7E72346F8E728
:1055F00040C0000028C000002DE9F04347683B7B15
:1056000001F01F0585B00E4645EA43151446D2B990
:1056100002A9284601F06CFA0446284601F02CFB4A
:10562000464B984204D06FF0040005B0BDE8F0830B
:10563000844201D00020F8E79DF8080001F0A0FAAC
:10564000A042F7D0EFE74FF000090DF1030130461B
:10565000CDE9029901F04CFA4B46804602AA494630
:10566000284601F021F9354B984202D06FF0150021
:10567000DBE7804503D19DF8030001F081FAA30325
:105680004CD540F20663234040F20622934219D0E3
:105690000CD8062B17D004D8ABB1022BE6D10423CB
:1056A00011E0B3F5007FE1D101230CE040F20242AA
:1056B000934227D0B3F5C06F26D0B3F5806FD5D114
:1056C000022300E007238DF8043084F48033C3F311
:1056D0000043E0068DF8053054BFC4F340130323A4
:1056E00021038DF8063011D57A680123B340C2F842
:1056F0000835002201A9284601F084F90F4B984291
:1057000098D0B3E70523DEE70323DCE7620341BF5C
:1057100001237A68B340C2F80C35EAE7E3064FF09C
:10572000000354BFC4F3401403241A4601A92846B9
:105730008DF8044001F0B8F8E0E700BF0000AD0BC1
:10574000034630B51D694068AA6D2B6E85B02ABB33
:105750008BB3696DAB6614461A46CDE90014E96D4A
:10576000029131B3002B18BF134600226946039300
:1057700001F07EFC114B98420ED06FF00404002221
:105780001146284605F08DFA2C6405F1280002F038
:105790007BFB002385F86C3005B030BD696D13B11B
:1057A0009A4228BF1A460029AA6614BF144600244C
:1057B000D3E70B46D9E71C46E1E700BF0000AD0B7D
:1057C0002DE9F04F99468B8804698046980489B08A
:1057D0000E46924600F1C7804FF0FF324FF0FF3384
:1057E00004F1100002F076FB6660D8F810B0D8F82B
:1057F000043000939BF86D3001931BB1DBF800304F
:105800009E425FD0B788390500F1DC8017F0090FA0
:1058100040F0D580C7F34513082B40F0D0803568A1
:10582000744B9D4240F2CB80009B03F1080EBEE812
:105830000F000DF10C0CACE80F00DEF80030CCF8D6
:1058400000306D4B9D4240F297806C4B9D4240F280
:1058500096806B4B9D4240F295806A4B9D4240F290
:105860009480694B9D4240F29380684B9D422CBFCF
:105870004FF000454FF08045BA07059507F0040347
:1058800040F18980002B14BF032302238DF81830C8
:10589000019BC7F300178DF819702BB1009801F028
:1058A000AFFB00238BF86D305B46594A009803A983
:1058B00001F0F8FA574B984271D101238BF86D3003
:1058C000CBF80060012384F86C30BAF1000F7CD172
:1058D000C4F844A00023A36404F1580204F1480171
:1058E00004F1440005F0B8F96065B9F1000F75D115
:1058F000C4F84C900023236504F1600204F15001C8
:1059000004F14C0005F0A8F900263246E0650121BB
:105910002046266405F0C5F94046FFF711FF256EC5
:10592000A36D27469D4238BF1D464FF4FA535D4391
:1059300057F8283B4FF4004C1B68B5FBF3F5314694
:10594000C83540F2E7304FF47A720023E5FB0C01D2
:10595000FAF7D6FB02460B46384602F0BBFA00289F
:1059600044D1256C1DE0A369002B7FF435AF63683B
:1059700099427FF431AF38E74FF000757CE74FF084
:10598000806579E74FF0006576E74FF0805573E763
:105990004FF0005570E7003B18BF012376E76FF02A
:1059A000040523689B8813F4005304D1636004F159
:1059B000100002F069FA284609B0BDE8F08F6FF0D8
:1059C0001505EEE76FF08505EBE7DAF80030636464
:1059D000002B3FF47FAFDAF804307CE7D9F80030D1
:1059E000E364002B86D0D9F8043084E76FF07305A8
:1059F000D7E700BF47E801008FD003001FA10700D1
:105A00003F420F007F841E00FF083D0000127A0015
:105A1000DFAD00000000AD0BF0B504694668A56D70
:105A2000236E85B08DB9002B36D11D46002211465C
:105A3000204605F03CFA256404F1280002F024FA1F
:105A4000002384F86C3005B0F0BD616D03BB31BB41
:105A5000B36800919D4228BF1D46636DA5661BB1CA
:105A6000A36D002B18BF2B460193E36D02931BB16E
:105A7000236E002B18BF2B46002269463046039345
:105A800001F0FCFC0E4B9842DDD06FF00405CDE731
:105A90009D4228BF1D46DAE7616D1D46D8E701F03B
:105AA0006043B3F1005FD3D0082D28BF082504F16F
:105AB0006E072A46384604F0BAFF3946C8E700BFE9
:105AC0000000AD0B2DE9F04F98468B88046907461E
:105AD00098048BB00D46914600F1D8804FF0FF320C
:105AE0004FF0FF3304F1100002F0F4F96560D7F8CD
:105AF00004B0D7F810A0DBF80C3003939AF86D309F
:105B000001931BB1DAF800309D426DD0AE883105AB
:105B100000F1F18016F0090F40F0EA80C6F345135A
:105B2000082B40F0E5802B680293029A7D4B9A4245
:105B300040F2DE800BF1100EBEE80F000DF1100CEC
:105B4000ACE80F00DDE90223934228BF13469EE82C
:105B50000300754A93428CE8030040F2A080734A28
:105B6000934240F29F80724A934240F29E80714A73
:105B7000934240F29D80704A934240F29C806F4A6B
:105B80009342C0F09B806E4A9342C0F09A806D4A67
:105B900093422CBF4FF0A0534FF02063B2070693FF
:105BA00006F0040340F19080002B14BF032302236E
:105BB0008DF81C30019BC6F300168DF81D602BB1CB
:105BC000584601F0FDFB00238AF86D3053465E4ACB
:105BD00004A9584601F0FAFA5C4B984278D10123A7
:105BE0008AF86D30CAF80050012384F86C30B9F19E
:105BF000000F40F08380C4F844900023A36404F1B4
:105C0000580204F1480104F1440005F02BF96065E5
:105C1000B8F1000F7BD1C4F84C800023236504F158
:105C2000600204F1500104F14C0005F01BF900265C
:105C30003246E06501212046266405F038F93846F1
:105C4000FFF7EAFE256EA36D27469D4238BF1D462D
:105C50004FF4FA535D4357F8283B4FF4004C1B6850
:105C6000B5FBF3F53146C83540F2E7304FF47A72B0
:105C70000023E5FB0C01FAF743FA02460B463846CF
:105C800002F028F900284AD1256C23E0A369002BF3
:105C90007FF424AF636899427FF420AF27E74FF089
:105CA00000737BE74FF0806378E74FF0006375E7A0
:105CB0004FF0805372E74FF000536FE74FF080438F
:105CC0006CE74FF0004369E7003B18BF01236FE723
:105CD0006FF0040523689B8813F4005304D16360BC
:105CE00004F1100002F0D0F828460BB0BDE8F08FA8
:105CF0006FF01505EEE76FF08505EBE7D9F800309A
:105D00006364002B3FF479AFD9F8043076E7D8F814
:105D10000030E364002B80D0D8F804307EE76FF0C9
:105D20007305D7E747E801008FD003001FA10700E4
:105D30003F420F007F841E00FF083D0000127A00E2
:105D40000024F4000048E801EBAF00000000AD0BB8
:105D5000F0B54B79012B26D0032B21D110268B795E
:105D6000032B1DD1CC790CB1012C19D10A7912B1B8
:105D7000022A15D10E220B684568B3F5164F2D681F
:105D800065D02DD8B3F5165F64D016D8B3F5966FED
:105D900062D00AD8B3F5967F61D0B3F5167F61D093
:105DA0006FF0850052E00026D9E7B3F5166F5CD09E
:105DB000B3F5965FF4D1374B3CE0B3F5E14F57D0E4
:105DC00007D8B3F5615F55D0B3F5964FE8D1324BA4
:105DD00030E047F61227BB42E2D14FF4000329E03E
:105DE000B3F5613F48D013D8B3F5963F47D009D8F3
:105DF0004DF6C027BB4244D0B3F5614FD0D14FF42C
:105E00006B0317E0B3F5E13FCAD14FF0EB7311E03C
:105E1000B3F5612F38D008D8204FBB4237D0B3F547
:105E2000E12FBDD14FF0E86304E01D4FBB42B7D175
:105E30004FF080530069C5F82435031D03C934436E
:105E40002243C5F86C2583E803000020F0BD4FF421
:105E50001D03EFE7134BEDE74FF49E23EAE74FF402
:105E6000A033E7E74FF41C33E4E74FF41D23E1E7E9
:105E70000D4BDFE70D4BDDE74FF06C73DAE70C4BB2
:105E8000D8E74FF46503D5E74FF07063D2E74FF0E2
:105E90008063CFE700B0130000A04E0090D0030055
:105EA00040420F000050270000C0750000F03A008B
:105EB00000903A01F8B5066905460F4605F076FDF3
:105EC000B0B9204B1B789BB16424686805F098F941
:105ED000F8B9012005F056FB013CF6D10021212044
:105EE00002F0ECFAF0E784F31188BFF36F8FF5E767
:105EF0004FF02003EFF3118483F31288BFF36F8F09
:105F0000686805F07DF988B984F31188BFF36F8F55
:105F1000EEE74FF02003EFF3118483F31288BFF311
:105F20006F8F686805F06CF90028DCD031460122DB
:105F300001F8147F686805F048F984F31188BFF30D
:105F40006F8FF8BDC516002070B5012383400E4A3F
:105F5000BFF35B8FDC4352E8001F01EA040542E80F
:105F60000056002EF7D1BFF35B8F4FF48032824092
:105F70000648C0F80823BFF35F8FBFF36F8F0B4253
:105F800014BF0120002070BDC4110020001001408A
:105F90001B49F8B5044622F07F450868C1E9002393
:105FA000A5F50013101AB3F5400F0FD302F0F2FB62
:105FB000A30003F1804303F58833D3F840259542CD
:105FC0001DD14FF40002C3F8402512E00D4B1B68B1
:105FD0001A0A1B065E190C4B42F10007C3E9006761
:105FE00002F0D8FB094A04F5A87352F823309D4209
:105FF00005D1064A4FF48033A340C2F84433F8BDBC
:1060000010060020C81100201806002000100140D2
:1060100011B3BFF35B8F0123104A834052E800CFD6
:106020004CEA030C42E800C10029F7D1BFF35B8FB3
:106030000B4A4FF480338340C2F80433094BBFF35B
:106040005B8F1B68BFF35B8FC340DB0742BF064B10
:106050004FF40032C3F80021704700BFC411002084
:1060600000100140C011002000E100E00D4B186855
:10607000010A0006BFF35F8F0B4BD3F804351818E5
:1060800041F10001B3F5801F0AD2084BD3E9002388
:10609000904271EB030303D210F1807041F10001D3
:1060A000704700BFC81100200010014018060020F2
:1060B0002DE9F74F14461D460746FFF745FF0090B0
:1060C000FFF7D4FFA04271EB05037AD2464B201AAA
:1060D00065EB0101984271F1000180F08180434B32
:1060E00003EB0713D3E902239D4208BF944253D028
:1060F0004FEA870A0AF1804A07F150090AF5883AFF
:106100004FEA89091FFA89F924F07F4809F180498B
:106110004FF48033DAF84005354A09F58839BB4039
:106120004646D2F804B5A0EB0B0020F07F402BF0E0
:106130007F410128CAF8401505D10193132005F0CD
:106140008DFD2B4A019B0BF1020CA6EB0C0020F0FD
:106150007F40B0F5000F88BF66460020C9F80000F8
:10616000D9F80000C2F8443326F07F40CAF8400551
:10617000D2F80405834506D0301A023820F07F405B
:10618000B0F5000F1BD8A6EB080626F07F4636199F
:1061900045F1000334461D4614490C983B0101EBC0
:1061A0000712C8500D9B5360C2E9024500243846CF
:1061B0000099FFF72DFF204603B0BDE8F08F304671
:1061C000AFE701230B4ABFF35B8FBB4052E8000FE0
:1061D000184342E800010029F8D1BFF35B8FDBE7E9
:1061E0006FF01504E3E700BF010000010006002086
:1061F00000100140C011002073B5194B194D002447
:106200004FF0FF304FF0FF31C5F80845C3E90201F8
:106210004FF48033C5F80433134B02264FF4003299
:106220000121C5F804631120C3F88021224604F03F
:1062300030FA1120FEF750FB0C4A0123AB602B60B3
:1062400013600B4B0B4A0093019400232046FFF789
:106250002FFF3046FFF7A6F8204602B070BD00BF02
:10626000000600200010014000E100E0C411002001
:10627000915F0000FFFF7F002DE9F743334CD4F816
:1062800004339A070BD5D4F8043143B1304A0023C4
:10629000C4F80431D4F804311368013313604FF0AB
:1062A0002003EFF3118283F31288BFF36F8FD4F8CA
:1062B0000433DB0329D5BFF35B8F264B53E8001F64
:1062C00021F0010043E80005002DF7D1BFF35B8FFB
:1062D00011B9D4F84031C3B10025C4F84051D4F805
:1062E000403182F31188BFF36F8FFFF7BFFE4FF08D
:1062F0002003EFF3118283F31288BFF36F8F164BE5
:10630000D3E90267B042B94106D282F31188BFF3E4
:106310006F8F03B0BDE8F0834FF0FF384FF0FF39C7
:10632000D3E90010C3E902891D604FF48033C4F83B
:10633000483382F31188BFF36F8F0029E9D00090B2
:1063400032463B4628468847E3E700BF001001403D
:10635000C8110020C011002000060020431C13B506
:1063600021D0012821DDB0F5000F20DA441EFFF70F
:106370007DFE104BD3E90013421AB2F5000F0E4810
:1063800028BF002401322244824228BF024652180C
:106390004FF0000009490190009143F10003FFF71D
:1063A00087FE02B010BD0448E0E70024DFE7024C9E
:1063B000DDE700BF10060020FFFF7F00915F0000B7
:1063C00008B5FFF753FE024B1B68C01A08BD00BF9B
:1063D00010060020036803F01F025B09012B026016
:1063E000024818BF4FF0A040704700BF00030050A4
:1063F0004FF08053D3F83021082A06D1D3F8343136
:10640000052B02D8024AD05C70470020704700BFBD
:1064100044EC0000024AD2F80034002BFBD0704755
:1064200000E0014008B54FF08053D3F83021082A2E
:106430004ED14FF080420021C2F80C11C2F8101169
:10644000C2F8381502F54042D3F80414C2F82015FA
:10645000D3F80814C2F82415D3F80C14C2F8281580
:10646000D3F81014C2F82C15D3F81414C2F8301550
:10647000D3F81814C2F83415D3F81C14C2F8401518
:10648000D3F82014C2F84415D3F82414C2F84815E0
:10649000D3F82814C2F84C15D3F82C14C2F85015B0
:1064A000D3F83014C2F85415D3F83414C2F8601578
:1064B000D3F83814C2F86415D3F83C14C2F8681540
:1064C000D3F84014C2F86C15D3F84434C2F87035D0
:1064D000FFF78EFF18B1384B384AC3F88C26FFF708
:1064E00087FF18B1364BFB22C3F81825FFF780FF52
:1064F00070B14FF080414FF08053D1F8E42ED3F8C3
:10650000583222F00F0203F00F031343C1F8E43EA8
:10651000FFF76EFF20B12B4B4FF40072C3F84026FB
:106520004FF08053D3F83031082B1AD14FF080430D
:10653000D3F80024D20744BF6FF00102C3F800244F
:106540004FF08053D3F83431052B02D81E4AD35C68
:106550003BB14FF01023D3F808224FF08043C3F82B
:1065600058254FF01021D1F80C32DB071FD5174802
:106570000123C0F80435FFF74DFFD1F80C3223F0AA
:106580000103C1F80C32FFF745FF0023C0F80435C2
:10659000FFF740FFBFF34F8F0D490E4BCA6802F45F
:1065A000E0621343CB60BFF34F8F00BFFDE70A4BA0
:1065B0000A4A1A6008BD00BF00500040488103002D
:1065C00000F00040009002403EEC000000E001407E
:1065D00000ED00E00400FA05580200200090D0030E
:1065E00070B501250268BFF35B8FB2FA82F3C3F185
:1065F0001F03DBB205FA03F422EA040450E8006F3B
:10660000964204D140E8004CBCF1000FF6D1BFF334
:106610005B8FE7D101480B7070BD00BF0000AD0B70
:106620000368CB40DB0710B514D401238B4002680C
:10663000BFF35B8F43EA020150E8004F944204D15C
:1066400040E8001CBCF1000FF6D1BFF35B8FEED128
:10665000014810BD0148FCE70000AD0B0400AD0B84
:10666000F7B5044618B1012822D003B0F0BD4FF0B1
:1066700080430222C3F80823C3F80401D3F804219D
:106680000122DA60074601238DF8073042F21075C7
:106690004FF08046CCB1012CE7D1C7B3D6F80C340B
:1066A00003F001033B70D6F80C34DA0321D516E071
:1066B0004FF080430022C3F80803C3F80021D3F849
:1066C000002158600DF10707DDE7B7B1D6F818349F
:1066D00003F003033B60D6F81834D803C5D59DF802
:1066E0000700012803D104F04DFF013DD2D1012C58
:1066F000BBD10C4B00225A71B7E7D6F81834D90336
:10670000B3D5012004F03EFF013DF6D1ADE7D6F848
:106710000C34DB03EDD5012004F034FF013DF6D14C
:10672000E7E700BFCC110020044B1A7922B90122FF
:1067300018609A800248704702487047CC110020C8
:106740000000AD0B0C00AD0B4FF0804310B5D3F83B
:1067500000216AB10022C3F80021D3F800210122F0
:10676000C3F80823114B587910B95A711B68984720
:106770004FF08043D3F8042172B10022C3F8042102
:10678000D3F80421D3F81824D3F81814920704D1AD
:106790000122C3F818259A6010BD0222C3F808230D
:1067A000024BBDE810401B6801201847CC110020A7
:1067B000036803F01F025B09012B0260024818BF47
:1067C0004FF0A040704700BF00030050034B08305B
:1067D00033F81000C0F34010704700BF5C02002087
:1067E00070B500F108030C4C34F81330DA05054697
:1067F0000E4607D5C3F3432304EBC30254F83330EA
:1068000052689847A3682BB1E26831462846BDE834
:106810007040184770BD00BF5C020020124A08306B
:1068200010B432F81030D9051BD5C3F3432123F43B
:10683000F85322F8103002F10E04002034F8023F21
:1068400013F4807F03D0C3F34323994209D001306E
:106850003028F3D1002342F83130044810BCFFF750
:10686000DFBE10BC704700BF5C020020D0020020D9
:1068700038B50246FFF7AAFF094C02F1080540B1FE
:1068800034F8153007495B0B03F5A273002041F87B
:1068900023001046FFF7C2FF002324F8153038BD4F
:1068A0005C020020006000402DE9F043044685B002
:1068B00090461D46F1B14E4F00F1080937F81960B6
:1068C000B30702D5FFF782FF18BB002326F00206AC
:1068D000CDE900338DF80E308DF80F300DF10F0239
:1068E0000B4620460DF10E0146F0010604F097FE1E
:1068F00027F81960B8F1000F26D03D4B98F80070CA
:10690000D8F8042004F1080633F81610880702D5D9
:1069100092B138481AE021F02001C904C90C23F8CB
:1069200016104AB1032FF4D892F800C08FB9324A3A
:106930000CF5A27C42F82C7033F8162022F01C02D1
:1069400042EA870223F816204DBB2C4805B0BDE86B
:10695000F0834FEA8C0202F1804202F5C04241EA24
:106960004C31D2F8100520F00300C2F81005D2F81F
:10697000100520F44F3020F44070C2F810052002BA
:10698000D2F810E500F47C5040EA074040EA0E00DF
:1069900041F0200123F81610C2F81005CCE7D5E924
:1069A00000672046FFF73AFF002ECED0104DD5E904
:1069B0000023964201D19F4218D011480DF10F01DA
:1069C000FFF70EFE0D4B9842C0D19DF80F2045F801
:1069D000326005EBC20308345F6035F8143043EAD7
:1069E000422343F4807325F81430AEE70022EEE72B
:1069F0005C0200200400AD0B006000400000AD0B05
:106A0000D00200202DE9FF410446154609B3324F5C
:106A100000F1080837F81860B20703D4FFF7D6FE74
:106A2000002857D116F01C0F02D04B78012B51D003
:106A300001238DF80F300023CDE900134A1C8B1C75
:106A400020460DF10F0146F0030604F0E8FD27F89B
:106A500018601DB9214804B0BDE8F0811E4E04F154
:106A6000080736F81700830734D595F800C061464B
:106A7000890020F0200001F18041C00401F5C041EF
:106A8000C00C26F817000023C1F810356A78002AD8
:106A9000E0D0D1F81035AD7823F4991323F4F853EE
:106AA000C1F81035D1F810E5230203F47C53120429
:106AB00002F4403243EA0E0313432A0502F4801223
:106AC00040EA4C30134340F0200026F81700C1F88C
:106AD0001035BFE70248BEE75C0200200000AD0BA6
:106AE0000400AD0B014BC3E9020170475C020020BA
:106AF00008B50246FFF76AFE38B1054B0548083273
:106B000033F812305B0B0B7008BD0348FCE700BF85
:106B10005C0200200000AD0B0400AD0B38B50F4C3B
:106B200094F87850BDB96022294604F1100003F0B2
:106B300089FF0620FDF7D0FE094B0A48C3F87C51B7
:106B4000D3F87C214FF00042C3F80423012384F8DA
:106B50007830636738BD0448FCE700BF5C02002062
:106B6000006000400000AD0B0500AD0B034B93F837
:106B70007800003818BF0120704700BF5C02002079
:106B800001460148FFF74CBDCC02002001460148F8
:106B9000FFF726BDCC02002037B50446FFF716FEEE
:106BA00004F108021E4B33F81230E8B113F002056D
:106BB0001AD15B0B9A0002F1804000F5C24002F14D
:106BC000804202F5C04205600068D2F8100540F02E
:106BD0000100C2F8100529B1012202FA03F3114A9B
:106BE000C2F8043303B030BDC3F38203042B12D0C8
:106BF000052B12D001A80194FFF7DAFD019BD0F814
:106C00001015D94001F001010231204603B0BDE862
:106C1000304004F04DBD0321F7E70221F5E700BF46
:106C20005C0200200060004008B50246FFF7CEFD80
:106C3000C0B102F108010E4B33F81130990711D49D
:106C40005B0B01229A409B000A4903F1804303F544
:106C5000C043C1F80823D3F8102522F00302C3F87B
:106C6000102508BDBDE808400021104604F020BDF5
:106C70005C020020006000400E4B00F1080213B5DA
:106C800033F81230DB07044611D5FFF7CDFF20465D
:106C9000FFF7EEFD01A80194FFF78AFD019B03F5C4
:106CA000E073022240F82320034802B010BD0348DD
:106CB000FBE700BF5C0200200000AD0B0400AD0B41
:106CC0002DE9F04F684B69486949002687B00122D9
:106CD00034461D6835B1D0F8045315421EBF1C6000
:106CE0001D68164304338B424FEA4202F1D1DFF8AC
:106CF0007C91D9F87C31002B00F099804FF0A043B3
:106D0000D3F820250492C3F82025D3F82028059233
:106D1000C3F820284FF000080DF1100A4FEA48137D
:106D200000934FF0010B49E0009B524A94FAA4F4FF
:106D3000B4FA84F41C44E00804F10803039432F824
:106D400013701AF8003004F007020BFA02F223EA7B
:106D500002030AF8003003A8FFF72AFD039B03F59E
:106D6000E073B90850F82330C7F382054A072F466D
:106D7000C3F301432CD520463946DDB2FFF730FD81
:106D800003A80394FFF714FD039B03F5E07350F889
:106D90002330C3F301439D4207D10021204604F074
:106DA00087FC2946204604F083FC03A80394FFF7E0
:106DB000FFFC039B0BFA03F3C0F820355AF8284078
:106DC000002CB1D1B8F1000F1DD14FF00108A5E79B
:106DD000022B0CD10321204604F06AFC05F00503C8
:106DE000012BE2D139462046FFF7FAFCDDE702210C
:106DF0002046019304F05CFC032DF3D0019B032B90
:106E0000D3D1022DEDE74FF0A042C9F87C41D9F86B
:106E10007C311949D2F820350493C2F82035D1F8D5
:106E2000202505921343C1F820257FF473AF012478
:106E300016B907B0BDE8F08F96FAA6F3B3FA83F35C
:106E400004FA03F29B0003F1804303F5C04326EAF2
:106E50000206D3F81005D3F81015C0F30520C1F3CE
:106E60000141FFF7BDFCE3E7006100400060004026
:106E7000206100405C0200200003005001460148F0
:106E8000FFF7AEBBD8020020036803F01F025B09C6
:106E9000012B0260024818BF4FF0A040704700BFAE
:106EA000000300502DE9F34790F80480514D174638
:106EB000282202FB08F2AE18347F002C40F09780A5
:106EC00004687360AF50CB7B86F8253091F803904F
:106ED00086F81E904A79F2770E7B002B45D191F807
:106EE00000A0012E504679D804F00CFC01A8CDF882
:106EF00004A0FFF7C9FF019B03F5E073012240F8EE
:106F0000232091F801A0BAF1FF0F0DD0504604F0F4
:106F1000F9FB01A8CDF804A0FFF7B6FF019B03F52C
:106F2000E073032240F823208B78FF2B0CD001A8BC
:106F300091F80EA00193FFF7A7FF019B03F5E07303
:106F40004FEA8A0240F82320B9F1FF0F0DD04846DE
:106F500004F0CBFB01A8CDF80490FFF795FF019B4F
:106F600003F5E073032240F823200B7C93B94B78A0
:106F70000878FF2B18BF1A468B78C4F8080508BF9D
:106F80004FF0FF32FF2B08BF4FF0FF33C4F80C2542
:106F9000C4F810358B68C4F824354B7B003B18BF10
:106FA0000123022E1DD0032E1ED0012E01D143F04D
:106FB0000203C4F854350123C4F800351FB144F36B
:106FC0000730FDF789FC282303FB085500236B7766
:106FD000094801232B7702B0BDE8F08704F085FB58
:106FE00084E743F00403E4E743F00603E1E70348E2
:106FF000F1E700BFD41100200000AD0B0500AD0B80
:1070000070B50679194C056828237343E35833B1EA
:1070100045F30730FDF76EFC0423C5F80833002361
:10702000C5F80035282303FB064393F82530BBB988
:10703000D5F8080504F04BFBD5F81005421C01D02B
:1070400004F045FBD5F80C05431C01D004F03FFBD0
:10705000282303FB0643987FFF2801D004F037FB69
:10706000282303FB06440023237770BDD41100209E
:107070002DE9F04707793A4D28237B439046EA18DB
:107080000E46517F8246002968D155F80390B9F128
:10709000000F01D00123537796E80F00282404FB4A
:1070A000075404F10C0C8CE80F00A07F0023FF288C
:1070B00084F8243001D004F025FB2823B8F1000F18
:1070C00006D003FB0753002226485A77BDE8F08715
:1070D000DAF8004003FB07530422C4F80823C3F87E
:1070E0002080C4F80881D4F8082172686AB1336836
:1070F000012A1978C4F81C150BD1F368012B0BD9A0
:10710000282303FB0753DB7F04E0DB7FC4F81C3537
:10711000F3E75B78C4F81C35B9F1000F04D0042301
:10712000C4F804331048D1E707EB870105EBC10130
:10713000D4F80831002BFBD0C4F808912046D4F8CD
:10714000083104F0ECFA0028F2D1282303FB07559C
:10715000A87FFF28E6D004F0C8FAE3E70348B5E7C4
:10716000D41100200300AD0B0000AD0B0B00AD0BE4
:107170000C480D49002310B5C0F80831D0F808318B
:1071800004F0CDFA68B9887FFF2801D004F0ADFA89
:1071900000230B724B77BDE81040D1E90031034862
:1071A000184710BD00300040D4110020DC11002031
:1071B000036803F01F025B09012B0260024818BF3D
:1071C0004FF0A040704700BF000300502DE9F04F82
:1071D000774E057985B0009206EB4512127F002AA2
:1071E00040F0E280002D40F0E180009A046891F8C0
:1071F00011B0D1F808A0C6E90023CA7CB37F62F3BE
:107200000003B37791F80490DBB269F341036BF3A9
:107210008203B377CF78F777002A61D10B7B91F89F
:107220000080BAF1A05F08BF0325012B404600F2A1
:10723000A78004F0B4FA03A8CDF80C80FFF7B8FFDC
:10724000039B2D0203F5E07345F0010240F8232073
:107250004878FF280ED0019004F0A1FA019803901D
:1072600003A8FFF7A5FF039B03F5E07345F00302B6
:1072700040F823208A78FF2A0DD08B7B019303A846
:107280000392FFF795FF039A019B02F5E07245EA2E
:10729000830340F82230FF2F10D03846B9F1000F99
:1072A00071D004F07CFA03A80397FFF781FF039BDA
:1072B00003F5E07345F0030240F82320C87BFF2864
:1072C0000ED0019004F05EFA0198039003A8FFF736
:1072D0006FFF039B03F5E07345F0030540F823506F
:1072E0000B7D2BBB4B780878FF2B18BF1A468B7889
:1072F000C4F8080508BF4FF0FF32FF2B08BF4FF05E
:10730000FF33FF2FC4F80C25C4F810353ED0BBF175
:10731000000F3BD08B7CC4F81475C4F86895C4F892
:107320006435CB7BFF2B08BF4FF0FF33C4F86C35BF
:107330000B7CC4F86035C4F824A54B7B0A7B003B6A
:1073400018BF0123022A29D0032A2AD0012A01D1F9
:1073500043F00203C4F854358B79C4F8C0350723D1
:10736000C4F80035009B1BB144F30730FDF7B4FAB5
:10737000002373770F480123337705B0BDE8F08F02
:1073800004F000FA57E704F0FDF98CE74FF0FF3303
:10739000C4F814350023C4F86835C0E743F004038B
:1073A000D8E743F00603D5E70348E6E70348E4E7F8
:1073B000FC1100200000AD0B0500AD0B0300AD0B70
:1073C0002DE9F34103792A4D04685E0105EB43186A
:1073D000AB590746CBB144F30730FDF78BFA254B89
:1073E000C4F8083398F81D307BB1012363614FF076
:1073F0006408D4F804312BB9012004F0C3F8B8F1C3
:107400000108F6D1AB1900225A770023C4F80035E1
:10741000AB199B7FDB071FD4D4F8080504F0CCF927
:10742000D4F8100504F0C8F9D4F80C0504F0C4F938
:107430003B791BB9D4F86C0504F0BEF9AB19DB7FBE
:10744000FF2B09D001A80193FFF7B2FE019B03F5C2
:10745000E073022240F82320074B9C4208BF01231F
:10746000354408BF636000232B7702B0BDE8F0818C
:10747000FC1100205201080000F002402DE9F04705
:107480003A4F037907EB4318154698F81D208246BA
:107490000C465E01002A66D157F80690B9F1000F3C
:1074A00005D015F0140F04BF012288F81D2094E8C0
:1074B0000F0007EB060C0CF10C0C8CE80F000121FF
:1074C000404604F089F92168DAF8003021B101F072
:1074D0006042B2F1005F06D1A26852B102F0604092
:1074E000B0F1005F05D03E44002321487377BDE82A
:1074F000F0876068C3F84415C3F84805E168C3F82D
:1075000034250022C3F83815C3F81821D3F8182100
:1075100015F0010218BF0122C3F8502515F0020230
:1075200018BF0122C3F840252A0708D5B9F1000F7A
:107530000ED10021404604F04FF90E48D7E7012252
:107540001A61BA5922B9D3F81821002AFBD0F0E702
:1075500015F0040F4FF0400202D0C3F80823ECE707
:10756000C3F80423E9E70448C1E700BFFC11002089
:107570000A00AD0B0000AD0B0B00AD0B0C4BD3F8AC
:10758000182170B592B10B4C0025C3F8185129464B
:107590002046D3F8183104F01FF92572D4E90031E0
:1075A000657704F10800BDE87040184770BD00BF62
:1075B00000F00240FC110020F8B50779224E0C467D
:1075C0000C21794305467018037A002B3AD172508A
:1075D00062684260697928689C46DAB2914229D88B
:1075E00040F30730FDF778F92B686278D3F804157B
:1075F000164821F0030102F003020A43C3F80425F0
:10760000D3F80815A27821F0030102F003020A431F
:10761000C3F80825D3F81015227821F00F0102F0E5
:107620000F020A43C3F810250C2303FB076601234E
:107630003372F8BD9A0002F5A072013340F802C01F
:107640008258CAE70248F4E71C1200200000AD0B84
:107650000500AD0B036801221A600279034B0C216F
:1076600001FB023302221A72704700BF1C12002075
:10767000036801221A610179024B0C2000FB0133DF
:107680001A7270471C12002002490348042204F0B9
:10769000B3B800BF1C120020008000402DE9F84F55
:1076A000DFF848B0124D9A46A5EB0B05114BED10D3
:1076B00080460F4691465D430026BE4202D13046C9
:1076C000BDE8F88F38F91640002C0DDDA5420BD32C
:1076D000013C24B204EB44040BEBC4005146C84700
:1076E0000028EDDB0136E8E70020F7E710C00000D6
:1076F000B8C00000ABAAAAAA0E4B70B553F8204040
:10770000013053F82060A64200D870BDD4E900359E
:107710002846984765B1EB6830B10028B8BF4042B1
:10772000FF28A8BFFF2018705A7842F001025A7053
:107730000834E8E7ECCC0000034A044B02609B1AD3
:107740000348DB105843704710C00000B8C0000069
:10775000ABAAAAAA70B5054610B90024204670BD90
:107760000378002BF9D00E4C0E4EB44208D10C4CCD
:10777000B442F2D0204604F093F850B91834F7E739
:10778000204604F08DF810B12368AB42E6D01834DF
:10779000EBE72168284603F003F90028EED1DDE786
:1077A00010C00000B8C00000014B986898307047C6
:1077B0004012002008B50A4B012202201A70FFF780
:1077C0009BFF04F0AAFB0320FFF796FF00F024FACA
:1077D000F9F75CF9034A137B23F00103137308BD27
:1077E000C5160020D806002008B50348034A00212A
:1077F000121A04F092F808BD38050020C8160020BF
:1078000070B5174E174D184986B0B82303FB0066B4
:10781000164B059301220F23CDE903320023CDE956
:107820000133182303FB005504464FF4B07000FBEE
:1078300004110F4B00954FF4A072304600F058F938
:10784000737B0C4AEE6023F0040373734FF40263FE
:1078500004FB033313442C756B6006B070BD00BF8E
:107860002006002040120020202700204AEC0000C3
:10787000D97C0000001F002080B52D4BB4B083F3ED
:1078800008882C4D2C4E6B692C4F43F40073002458
:107890006B61E02385F82230EC772C766C76AC7641
:1078A00085F820406B6A43F4E0236B6285F823403F
:1078B000FDF714FAFCF7DEFF4FF0FF33AB62EB622B
:1078C000FDF750FBFDF7B4FA40F20113ADF8243098
:1078D00006ABB360CDE92D44309403F0E0FF2046C1
:1078E000FFF70AFF0120164DFFF706FF00F058FDD5
:1078F000144BF5610593012313490094CDE903432B
:107900004FF480623B46CDE90144284600F0F0F890
:107910006A7B064622F0040228466A7304F0DCF80B
:107920002046FFF76DFF3A4631462846FDF7B0F88E
:107930002027002000ED00E040120020B577000075
:10794000D80600204FEC00008028002070B50E4BB8
:107950000E4CA34201D3002070BDD3E9030141EADC
:10796000000212F003020BD19D685A61AA4201D1B4
:107970001C33EEE75E690E60013259610144F5E7A0
:107980006FF01500E8E700BFE8040020E8040020DD
:1079900073B50C464FF02005EFF3118185F3128883
:1079A000BFF36F8F45695DB125602B6843618369C3
:1079B00001338361002081F31188BFF36F8F11E0E1
:1079C00052EA030603D125606FF00B00F3E7CDE91F
:1079D00000230246083000F0F7FB18B9024B9B6801
:1079E0005B69236002B070BD40120020F8B5054607
:1079F0000E464FF02003EFF3118783F31288BFF395
:107A00006F8F064B9C6A24B987F31188BFF36F8F81
:107A1000F8BD20463146A847646FF4E740120020C5
:107A20004FF02003EFF3118183F31288BFF36F8FC0
:107A3000094A936A834207D15B6F936281F311888D
:107A4000BFF36F8F70471346002BF7D05A6F8242F7
:107A5000F9D1426F5A67F1E74012002010B5044691
:107A600008B9054B9C681F2204F1780002F066FFFC
:107A7000002084F8970010BD40120020437B102B9B
:107A80000ED8102B1CD8DFE803F0091D131B151BA3
:107A90001B1B171B1B1B1B1B1B1B19000B487047B9
:107AA000202B11D00A4A0B48802B18BF1046704774
:107AB00009487047094870470948704709487047A6
:107AC00003487047084870470848704776DF000051
:107AD00054EC000085EC00005CEC000064EC00005D
:107AE0006DEC000072EC00008CEC00007CEC0000FF
:107AF0002DE9F04F85B0984600F15803C0E91633E0
:107B00000732129B037322F0070A0423002501F1B8
:107B1000200B43730AF12007119B85600446C0E9DE
:107B200006550E468373C5730F445246AA21584624
:107B3000DDF84C9002F086FF109BC4F8A450C4E915
:107B400027BA02930F9B01930E9B00933A4643463C
:107B500031462046FCF768FF0E9BA3660F9BE36649
:107B6000109B6565C4F8648023674FF02002EFF333
:107B7000118382F31288BFF36F8F104EB26A62676F
:107B8000B46283F31188BFF36F8FB9F1000F11D086
:107B90001F22494604F1780002F0D0FE84F8975085
:107BA000B3680BB1D3F8A830C4F8A830384605B094
:107BB000BDE8F08F84F87890F2E700BF4012002013
:107BC000F0B587B000250595109D04950F9D039590
:107BD0000E9D0295DDE912760D9D01950C9D009597
:107BE0000446FFF785FFB6F1FF3F08BFB7F1FF3F3F
:107BF00005D056EA070305D1204600F051FB204688
:107C000007B0F0BD03493A46334604F1180000F0CE
:107C100043FDF4E745BA00002DE9F043294C2A4D15
:107C200087B02646AE4204F130040FD300F088FB43
:107C3000244CDFF898904FF4004640F2E737AC420E
:107C400020D307B0BDE8F04300F08EBB54F8043CED
:107C5000059354F8103C049354F8143C039354F8DF
:107C6000183C029354F81C3C019354F8203C0093B8
:107C700054E90A2354E90C01FFF73AFF54F8303C69
:107C80005E65CEE7636A5A1C0DD023EAE3730021D8
:107C90003846C3FB060151EAC333D4F8008004D14F
:107CA000404600F0FDFA3034C9E74FF47A72002301
:107CB000F8F726FA02460B4608F11800494600F08C
:107CC000EBFCF0E7E8040020E804002045BA0000DF
:107CD000004870470063000308B50B4C0B4D4FF094
:107CE0002002EFF3118382F31288BFF36F8F03F04A
:107CF00083FF2B78A06113B9FCF7C2FDEFE7FCF717
:107D000011FC0028EBD1F7E740120020C516002037
:107D10002DE9F341044617461E464FF02003EFF3CA
:107D2000118883F31288BFF36F8FC368324A7BB127
:107D300080689168884219D057EA060318D188F301
:107D40001188BFF36F8F6FF00F0002B0BDE8F081B4
:107D5000916891F90E1021610133E3609368A3608B
:107D600088F31188BFF36F8F0020EEE72169F2E7F7
:107D700091F90E1090F90E309942A8BF19466FF094
:107D80007E029142B8BF11468B422EDD03F030FED9
:107D90000546CDE9007619482246414600F014FA1E
:107DA0000028E1D04FF02003EFF3118683F312880F
:107DB000BFF36F8F236821699C420AD04BB193F9BE
:107DC0000E309942A8BF19466FF07E039942B8BFA2
:107DD0001946A06803F00CFE48B945B986F311882E
:107DE000BFF36F8F6FF00A00AFE70025D1E70348BC
:107DF000314600F043FAF5E740120020C616002095
:107E000038B583680446002B33D01D4A92689342EC
:107E100032D1DA7B013ADA73C368012B05D9013B11
:107E2000C36000F0A1FA002038BD4FF02003EFF34B
:107E3000118583F31288BFF36F8F0169806803F0A7
:107E4000D7FD204603F058FEA06060B190F90E20E7
:107E500022610022C0F8B02003F03EFE0948294606
:107E600000F00CFADDE7E06085F31188BFF36F8F57
:107E7000D7E76FF01500D7E74FF0FF30D4E700BF2A
:107E800040120020C616002038B504464FF02003EB
:107E9000EFF3118583F31288BFF36F8F03F02CFE8D
:107EA00050B10022C0F8B02003F016FE2946084861
:107EB000BDE8384000F0E2B9D4E902329A4218BF76
:107EC0000133A360022104F1100004F00BF8EDE788
:107ED000C616002013B54FF02004EFF3118184F390
:107EE0001288BFF36F8F846844B1013C846081F3D2
:107EF0001188BFF36F8F002002B010BD52EA030457
:107F000006D181F31188BFF36F8F6FF00F00F3E795
:107F1000CDE900230246024800F056F9ECE700BF25
:107F2000C616002038B5074D2C6854B1FEF748FA44
:107F3000054B04441C6128680021BDE8384003F06B
:107F40006BBE38BD741200204012002038B50D4DB4
:107F50002B4653F8204F9C4200D004B9EC68AB6824
:107F600038B95A7BD20604D1A26912B9DA897F2ABC
:107F700005D89C4202D02046FFF7D4FF2346EB6190
:107F800038BD00BF4012002070B590F90D20437B32
:107F9000002A014604DA03F07F03437303F037FD40
:107FA0004B7B154A63F07F0310464B7350F8203F1C
:107FB000546A834208BF002323B9C1E90004216049
:107FC00051620CE091F90E5093F90E60B5420ED05B
:107FD000AE420CDD5868C1E900300160596090681C
:107FE000431A5842BDE870405841FFF7AFBF9C426A
:107FF000E3D01B68E0E700BF4012002070B490F9A6
:108000000D30427B002B29DBD30627D183692BBBA4
:10801000134962F07F0242730A4652F8204F94429D
:1080200018BF23464C6A23B9C0E900242060486287
:108030000CE090F90E5093F90E60B5420AD0AE42B2
:1080400008DD5A68C0E900321060586070BC00203A
:10805000FFF77CBFA342E7D01B68E4E770BC704722
:108060004012002008B590F90D20437B002A0146FC
:1080700004DA03F07F03437303F0C9FC044B9868F0
:10808000431A58425841BDE80840FFF75FBF00BFA0
:10809000401200202DE9F041064615461C464FF0DF
:1080A0002003EFF3118783F31288BFF36F8F03F080
:1080B000EBFC87F31188BFF36F8FB4F1FF3F08BF6C
:1080C000B5F1FF3F08D02A46234606F118000349C0
:1080D000BDE8F04100F0E0BABDE8F08145BA00002B
:1080E000F8B504460D464FF02003EFF3118783F3F4
:1080F0001288BFF36F8F00264FF4004C40F2E73038
:1081000031464FF47A720023E4FB0C01F7F7F8FFD5
:10811000B44202DD0228B8BF0220074A074B1060B4
:10812000074A98681E611560FFF7FCFE87F3118807
:10813000BFF36F8FF8BD00BF741200204012002003
:108140007012002038B54FF02003EFF3118583F350
:108150001288BFF36F8F174B174A9C6811688C42C7
:1081600007D12046FFF7DEFE85F31188BFF36F8F3E
:1081700038BD00211160114A1268C2B1E2897F2A1C
:1081800015D8627BD20612D10D4A94F90E101268EE
:1081900091420CDB0B4A944209D01A69824203DCFB
:1081A0002046FFF7F1FEDCE7121A1A61DCE7002235
:1081B000FBE700BF401200206C1200207412002068
:1081C000701200202006002010B5074B9868074B5E
:1081D0000C4618601146DDE90223FFF75BFF2046DD
:1081E000BDE81040FCF7C8BB401200206C12002014
:1081F000F8B504464FF02003EFF3118683F312889D
:10820000BFF36F8F437BDA0649B219D18569BDB9D7
:1082100003F07F03437303F0FAFB437B164A817339
:1082200063F07F034373134653F8200F984218BF3F
:108230000546506A5DB9C4E900300460546211E03B
:10824000A173002086F31188BFF36F8FF8BD95F9F5
:108250000E70B9420BD08F4209DD6B68C4E9005340
:108260001C606C600120FFF771FE0120EAE7A84264
:10827000E1D02D68DEE700BF4012002049B9EFF3DE
:10828000058030B9054BDA699B689A4201D0FCF74A
:1082900073BB81F31188BFF36F8F704740120020CA
:1082A00010B54FF02002EFF3118482F31288BFF370
:1082B0006F8F427B510704D484F31188BFF36F8F13
:1082C00010BD22F004024273FFF798FE21460248D7
:1082D000BDE81040FFF7D2BFC616002070B50446B7
:1082E000183003F073FC4FF02003EFF3118683F393
:1082F0001288BFF36F8F94F90D20637B002A05DA93
:1083000003F07F036373204603F081FB0B4D637B17
:10831000A86843F010036373031B58425841FFF7EA
:1083200015FE86F31188BFF36F8FAB68A34203D1AC
:10833000BDE8704003F01CBC70BD00BF40120020BF
:108340004FF02003EFF3118183F31288BFF36F8F97
:10835000044B9A68D37B013BD37381F31188BFF33D
:108360006F8F70474012002010B54FF02003EFF3DD
:10837000118483F31288BFF36F8F084B9A68D37B05
:108380000133D3730020FFF7E1FD84F31188BFF3BD
:108390006F8FBDE8104003F0EBBB00BF4012002020
:1083A000044B002103F12002C3E908220846FFF72D
:1083B00097BE00BF40120020F8B54FF02003EFF346
:1083C000118583F31288BFF36F8F19498868437B47
:1083D00003F07F03437303F01AFB437B0A4663F009
:1083E0007F03437352F8203F4C6A934208BF002337
:1083F00023B9C0E90024206048620CE090F90E60C7
:1084000093F90E70BE420ED0B7420CDD5A68C0E937
:108410000032106058600120FFF798FD2846BDE843
:10842000F840FCF7A9BAA342E3D01B68E0E700BF1D
:108430004012002050EA01032DE9F04105460E46A6
:1084400003D1FFF7B9FF00202CE0831C71F1FF334B
:108450002ADB03F0FDFB44194FF02003EFF31188F2
:1084600083F31288BFF36F8F114F124BB8681860F7
:10847000FFF7F8FDB86810492A463346183000F077
:108480000BF9BA68537B43F0100353734046FCF773
:1084900073FA03F0DDFB201A63EB0303012873F189
:1084A0000003D0DBBDE8F0816FF00104241AD3E7AC
:1084B000401200206C12002045BA0000B1F1FF3FCD
:1084C00008BFB0F1FF3F08B506D1084B9868FFF729
:1084D00005FF4FF0FF3008BDFFF7ACFF4FF47A7394
:1084E00080FB0303C00B40EA4340F4E74012002046
:1084F000014B9868704700BF401200202DE9F04101
:1085000004464FF02003EFF3118683F31288BFF384
:108510006F8F437B1A0705D586F31188BFF36F8FE2
:10852000BDE8F08123F0200242F00801D20923D1F6
:108530004173A36813B1204603F071FA04F11800E7
:1085400003F044FB04F158074FF00008A56DBD424D
:1085500000D0CDB90120FFF7F9FC2046FFF760FA03
:10856000104B9B68A342D7D1EFF30583002BD3D1E7
:108570003046FCF701FACFE703F05F0343F008034E
:10858000437303F044FAD4E7284603F048FA05F1B0
:10859000180003F01BFBC5F8B0802846FFF72EFD3E
:1085A000D4E700BF40120020D3B5DDE90667089C80
:1085B000CDE90067FFF708FE1CB1034B9B685B69C0
:1085C000236002B0D0BD00BF4012002008B50648AD
:1085D000064A0749121A03F0A2F9BDE80840054A05
:1085E0000549064803F09BB900000020380500202B
:1085F0009CEC0000000000009CEC0000000000204B
:10860000034B1B680BB9FDF7DBBE0020704700BFB2
:1086100078120020114B10B51C689C420AD1FFF75C
:10862000EFFF6FF000400E4B1B6913B19842A8BFDB
:10863000184610BDFFF7E4FF002CF2D0D4E9043255
:108640001B1A62EBE072B3F1004F72F10001E8DA3D
:10865000002AACBF18460020E5E700BFDC0200207E
:10866000401200200B4A03685268904230B509D08E
:1086700043B1D3E90421D0E90445121941EB0501C6
:10868000C3E90421426813605A600023C0E9003343
:1086900030BD00BFDC020020B3F1FF3F08BFB2F1E4
:1086A000FF3FF8B504461D46164661D081604FF085
:1086B0002003EFF3118783F31288BFF36F8F01322A
:1086C00075F1FF3324DA3049D1E900206FF001035E
:1086D0009B1A4FF0FF3262EB00009E1B60EB05001F
:1086E000012E70F1000301DA01260020C4E90460C4
:1086F000264ED6F800C07568B44508BF4FF0000C90
:10870000BCF1000F0DD1C4E900652C6074601CE061
:10871000FFF776FF013645F10005361845EBE070AE
:10872000E4E7DCE90420D4E90431934271EB000E64
:108730001FDAD21ADCF8043060EB0100CCE9042027
:10874000C4E900C31C60CCF804403368B3420BD0CA
:108750009C4209D1FFF75EFF18B10D4B1B698342A4
:1087600002D00021FDF7FAFD87F31188BFF36F8F68
:10877000F8BD9B1A61EB0001AC45C4E90431C2D0DD
:10878000DCF800C0BCE700BF90070020DC0200203E
:10879000401200202DE9F8430546FFF7D3FC4FF0C7
:1087A0002003EFF3118483F31288BFF36F8F244EFD
:1087B000DFF890803560244DD8F8000032684045DD
:1087C000D5E9001E4FEAE2770BD050B1D0E9043C66
:1087D0009A4277EB0C0916DA9B1A6CEB070CC0E98E
:1087E000043C51184EEB0707C5E90017002535601A
:1087F000FFF710FF2946FDF7B1FD84F31188BFF3A1
:108800006F8FBDE8F88359184EEBE377D31A3360C6
:1088100000220023C0E90423C5E90017FFF722FF67
:1088200084F31188BFF36F8F836898474FF020035C
:10883000EFF3118483F31288BFF36F8FBCE700BF9F
:1088400078120020DC0200209007002010B54FF0C5
:108850002003EFF3118483F31288BFF36F8FFDF7CA
:10886000AFFD054AD2E90031C01841F1000184F39F
:108870001188BFF36F8F10BD900700202DE9F347DB
:108880001D46294B9F68012387F8603087F86130C7
:1088900052EA050316460CBF0123002307F16002CC
:1088A000804603F010FA81464FF02003EFF3118A5F
:1088B00083F31288BFF36F8F97F8604064B9014665
:1088C0005246404603F0D0FA8AF31188BFF36F8F07
:1088D000204602B0BDE8F087002387F8603056EAF2
:1088E000050306D18AF31188BFF36F8F6FF00A0476
:1088F000EEE7CDE900650D4A0D485146FFF764FCEF
:1089000004464FF02003EFF3118583F31288BFF381
:108910006F8F2A464946404603F0A6FA85F3118830
:10892000BFF36F8FD4E700BF40120020E4020020A5
:10893000C616002038B503464FF02002EFF311852C
:1089400082F31288BFF36F8FC160012181600068DC
:10895000834206D185F31188BFF36F8F0024204630
:1089600038BDD0E9003213605A600023C0E90033FB
:1089700003F020FA294604460148FFF77FFCEEE7A2
:10898000C61600201FB5094B029302AB00240093CA
:10899000074908488DF80C404FF0FF334FF48062D0
:1089A00000F008F9204604B010BD00BF92EC0000B2
:1089B000A02C0020980700202DE9F04FDFF83C9113
:1089C00085B004464FF0FF364FF0FF374FF02003DD
:1089D000EFF3118883F31288BFF36F8FD4F8B85088
:1089E0008DB9022104F1D00003F098FA002843D198
:1089F0000023CDE90067029304F1C00241464048DC
:108A0000FFF7D2FDE2E7D4F8BC202B68C4F8B830F9
:108A1000954208BFC4F8BC30D4F8D03043F002030C
:108A2000C4F8D030EB6823F0040343F00103EB609B
:108A30006B6888F31188BFF36F8F284698474FF013
:108A40002003EFF3118B83F31288BFF36F8FEB6872
:108A5000990723F0010219D4EA60D4F8D03023F04A
:108A60000203C4F8D0308BF31188BFF36F8FDB059E
:108A7000ACD4FFF7A1FCA9E704F1C805002201214D
:108A8000284603F07FF80028F8D1B1E723F003036C
:108A9000EB60D9F80030002BDFD04FF00008D3F89E
:108AA00000A04146002BD8D05A689542184612D1F2
:108AB0001A68D9F80400B8F1000F15D18342C9F83B
:108AC000002001D1C9F80420184640F8081BFFF720
:108AD000DBF940460021BAF1000F0CD0DAF8002093
:108AE000534680469246DDE78342C8F8002008BF1F
:108AF000C9F80480E8E75246F2E700BF7C12002084
:108B0000C6160020F8B5C3680F4699070446C3F39C
:108B100040062BD45A0719D43A680AB982683A60D9
:108B2000DD0744BFA3683B603D684CBF02260126B9
:108B3000002D3AD01E4B9B68AB420AD0D5F8D030FE
:108B4000D807C3F3800214D46FF0120600233B60F1
:108B500025E002F02BFFD5F8D0300028F0D1D9075E
:108B6000C3F3C002F0D552B15B0708D46FF00F0613
:108B7000ECE7002AFAD1C3F3C003002BF6D100239F
:108B80002360D5F8BC3063B9C5E92E44284603F00C
:108B9000D0F9E36843F00403E3603B68A360304628
:108BA000F8BD1C60C5F8BC40F0E76FF01506CDE7D6
:108BB00040120020F0B589B004460020C4E92E0020
:108BC0000E9D04F1C000C4E9300004F1C800C4E9FE
:108BD00032001DB32879002840F2011008BF01209F
:108BE000C4F8D00000204FF0FF364FF0FF37CDE93A
:108BF0000330CDE90100CDE90667094B009420461A
:108C0000FEF7DEFF25B1296811B12046FEF726FFE9
:108C1000204609B0BDE8F04002F0D0BE0120DFE7F9
:108C2000B989000010B50A4C23681BB101232360E9
:108C3000002010BD00F0CEF80028F7D0013806283B
:108C400003D8044B53F8200010BD034810BD00BFEB
:108C50008412002004CD0000FE8FFFFFBFF34F8F72
:108C60000549064BCA6802F4E0621343CB60BFF3C8
:108C70004F8F00BFFDE700BF00ED00E00400FA05E4
:108C800010B4094B09490A4C4FF0FE32C3F80024D6
:108C90004968C3F80424C3F80824C3F80C2400234B
:108CA000C4F8003510BC084700B00250EC020020A8
:108CB00000A00250D0E90012014BC3E90012704736
:108CC000EC02002010B5044630B16368DB0602D523
:108CD00000232360636010BD024B03485B68984724
:108CE000F3E700BFEC02002020CD0000B0B14368E4
:108CF00093B1DB060ED5012350E8002F194640E85A
:108D0000001C9CF0000FF7D1012AF5D0BFF35F8F54
:108D10000020704703487047034870476FF4E040F5
:108D2000704700BFE98FFFFFEA8FFFFF68B143681C
:108D30003BB1DB0607D5BFF35F8F00230360184606
:108D4000704703487047034870476FF4E04070472E
:108D5000EA8FFFFFE98FFFFF10B5044620B1002224
:108D600011232260636010BD0148FFF789FFF6E719
:108D700048CD000070B5D0E90023134C134D63605B
:108D8000D0E90230C4E902302260114B0868186053
:108D90004868586088689860D1E90301D860196113
:108DA000D5F81831DB060DD50023C5E94533C5E9F3
:108DB0006E3305F58A709047236805F5DC70BDE8D1
:108DC0007040184770BD00BFFC0200209C120020BC
:108DD0000C03002038B500F02FF820B1032400F078
:108DE00063F8204638BD00F031F898B900F0ACF8CF
:108DF00098B90F4DD5F828391B0EF02B08D1D5F8AE
:108E0000242A0C4B9A420AD0072400F017F8E6E710
:108E10000624FAE70424204638BD0024F5E70120A3
:108E200000F092F804460028F7D1C5F80C0AD8E7FC
:108E300000B002500000E020002070470020704782
:108E4000014BC3F8040A704700B0025010B5114836
:108E500000F048F800B110BD0F4800F043F80028BA
:108E6000F9D10E4C204600F03DF80028F3D10C4B10
:108E70000C481C6000F036F801460028EBD100F0E9
:108E80002DF8044608B1204610BD00F03FF82046FA
:108E9000FAE700BF4403002038030020400300200D
:108EA000480300203C03002008B5084800F024F8DF
:108EB000074800F021F8074800F01EF8064800F0C7
:108EC0001BF8BDE8084000F00BB800BF44030020C9
:108ED00038030020400300203C030020002070479E
:108EE000704700BF08B5034B02681B6810689847BD
:108EF000002008BDFC02002008B5034B02685B6837
:108F000010689847002008BDFC02002070B5094C8D
:108F1000094D2069AB68984718B1084B08485B6851
:108F20009847084AEB68206900211160BDE870404D
:108F3000184700BF0C030020FC020020EC020020B8
:108F40006CCD00009812002070B51B4D1B4E0446DE
:108F5000B26828699047F8B95CB1194C2368B3B17D
:108F6000012B1BD0013B23602869F3689847002040
:108F700070BD134C216841B9124B0122C3F8002582
:108F8000114AD2F81039002BFBD101312160F3686E
:108F900028699847002070BD0C4870BD0A4AD2F875
:108FA0001039002BFBD1074A6FF07E40C2F8003524
:108FB000FFF746FF2368D5E70C030020FC020020E2
:108FC0009812002000A0025000B00250E98FFFFF6D
:108FD0007047062905D8042912D8032905D0042989
:108FE00008D0002808BF822007E000280CBF82209C
:108FF00029207047002808BF812018BF282070470B
:10900000002814BF2A2084207047002814BF28207D
:109010008220704703460A4600681979012303FA43
:1090200001F103691B68194218BF82F0010212B1F5
:109030008368DB68184783681B69FBE7F0B4034665
:1090400000681979DB88066987683468DA0754BFD5
:1090500043F4B01383F4D01301258D4023F4801220
:10906000DB074CBF2C43AC433B683460F0BC184773
:10907000F7F7C8BEF7F7C6BE08B5F8F7E7FD00205A
:1090800008BD034640B1426802F00302022A06D03E
:10909000032A04D0012A05D06FF0150070471A6822
:1090A000002AF9D0002098607047426802F003025D
:1090B000022A10B5034681604FF0000407D0032A4E
:1090C00002D05C60002001E018685C6010BD186888
:1090D0005C600028F6D0FFF72DFCF3E70020704716
:1090E0000FB407B504A951F8040B0191F8F73AFE43
:1090F00003B05DF804EB04B07047038B13F0070373
:1091000005D10368002B0CBF002003207047022B01
:1091100005D1408BB0FA80F0400980007047012BE8
:1091200005D10368002B0CBF0020052070470020EC
:10913000704710B50C4600B111B96FF0150010BDA5
:10914000081DFFF79EFF0028F9D1A368032BF6D96D
:10915000F3E72DE9F0410D4607461946281D9046D4
:109160001E46FFF7A2FF044638B133464246294661
:109170003846A446BDE8F0416047BDE8F08110B430
:109180004FF02004EFF3118284F31288BFF36F8F46
:10919000416110BC0121F8F7F3BD38B50C46054616
:1091A00058B151B10B6843B14B6833B11C22002157
:1091B00001F048FC2C61002038BD6FF01500FBE782
:1091C00070B505460E46FFF7B4FF041E15DB4FF0E1
:1091D0002003EFF3118283F31288BFF36F8F6B8B41
:1091E0002C8B4FF6FF718B4204F0070407D182F3FA
:1091F0001188BFF36F8F6FF00A04204670BD022CF8
:109200000CD101336B8382F31188BFF36F8F00237E
:10921000224631462846FFF79CFFEEE7062C14D87D
:10922000DFE804F004131313041A0400002333606E
:109230006B683BB9C5E90066ACB902212846F8F76E
:109240009FFDDAE71E606E60F6E782F31188BFF3D8
:109250006F8F6FF00404D0E782F31188BFF36F8F34
:109260006FF08504C9E782F31188BFF36F8FC4E7FD
:10927000044608B5084611461A46A047FFF738F9D4
:10928000FBF7C0FD2DE9F84F9A46D3786F2B804647
:109290000F461546A3F1410B29D024D8582B0CBFFB
:1092A00010260A26DDF8289032460023404639462B
:1092B000F6F726FF092AD4B21ED83034B045E4B2FE
:1092C00077F1000709F8014D01D3D14511D82B786A
:1092D0009B0605D5082E15D1AB7843F00803AB707B
:1092E0004846BDE8F88F03F0F703702BD7E7082650
:1092F000D8E780460F46D7E7BBF1190F94BF373444
:109300005734DBE7102EEBD1AB7843F01003E6E7E0
:109310002DE9F0410746884615461E461446B442DC
:1093200005D30EB1601B08E02378002BFAD014F8A7
:10933000010B4146B8470028F1DABDE8F081C36966
:10934000F0B54568C66804464069AF1B281ABB42A1
:109350009446A3EB00029CBFFF1AF6186245A3EBEC
:10936000070028BF624623689042A5EB060628BF87
:109370001046334405440B606560F0BDD0E901231D
:10938000D21A8A420CD31944C368C269C0E90111D8
:10939000C91A8A4201D9002070471344C360FAE712
:1093A0006FF0150070472DE9F34180460E461546D3
:1093B00000272A4601A94046FFF7C1FF314604466F
:1093C0000246019801F033FB2D1B2744264401D0AF
:1093D000002CEED139464046FFF7D0FF384602B0A8
:1093E000BDE8F081F0B5044605698669A368C069E7
:1093F000AF1BB8429446A3EB05029CBF36183F1A38
:109400006245A0EB070028BF624623689042A5EBA7
:10941000060628BF1046334405440B602561F0BDA5
:10942000D0E90423D21A8A420CD31944D0E9063277
:10943000C0E90411C91A8A4201D9002070471344B7
:109440008361FAE76FF0150070472DE9F34180461C
:109450000D4616460027324601A94046FFF7C2FFD7
:1094600004462DB102460199284601F0E0FA254450
:10947000361B274401D0002CEDD139464046FFF77A
:10948000CFFF384602B0BDE8F0810B0704D5A0F14C
:109490004103192B98BF203070472DE9F04F87B05A
:1094A000144601910393054618B9012007B0BDE8A1
:1094B000F08F019B002BF8D0039B002B00F00F8155
:1094C000019AA946214619F8010BFFF7DEFF034672
:1094D000C0B23F281678074625D013F0C00F0BD135
:1094E000C8B12A2836D021463046FFF7CEFF874242
:1094F00002F101021ED0D8E75B287DD05C28F2D1B2
:10950000E307F0D46878FFF7C0FF10F0FF0718BF3B
:1095100005F10209E7E7E70601D52F2EC6D0301E78
:1095200018BF0120C2E7002EBFD02F2E04D1A507FF
:10953000BBD401324D46C4E72E2EFAD16007F8D5D0
:10954000019B9A42B1D0A107F3D512F8013C2F2B11
:10955000EFD1AAE76878FFF798FFC1B22A2919D09E
:109560002E2E0AD1630708D5019B9A429DD0A707EA
:1095700003D512F8013C2F2B97D079B914F00200D3
:1095800094D0E60600F1AD802F21104601F0EAF9F3
:109590000038C5E719F8010F2146DCE72F2923D150
:1095A000A50721D5104601F0DDF902460028C1D1FA
:1095B0007BE73B46424659464846FFF76EFF012887
:1095C0007FF474AF2F2D03D1BAF1000F7FF46DAF8C
:1095D000B34621469BF80000FFF757FF10F0FF0548
:1095E00006F10106E5D160E7039B16465F1E24F0F5
:1095F000040804F0020AEBE7002E3FF456AF2F2ECA
:1096000002D1A0073FF551AF3046FFF73EFF6B7820
:10961000212B824601D05E2B23D1023501230293F8
:10962000012304EA03014FF0000B04912F46214669
:1096300017F8010B0593FFF728FF5FFA80F8B8F1E0
:109640005D0F059B10D10BBB029B5B453FF42DAF1B
:10965000791C03D15B2E7FF428AF4F460132B94607
:1096600068E74D460023DAE7B8F12F0FF2D0B8F1E2
:109670005C0F07D1049B4BB96878FFF706FFAF1C5E
:109680005FFA80F8B8F1000F3FF40FAF3B782D2B55
:109690001FD178782146FFF7F8FE10F0FF0018D0B0
:1096A0005D2816D05C2807F102050AD1E30708D42B
:1096B000B878FFF7EAFE10F0FF0007F103053FF46A
:1096C000F4AED04503DC5045A8BF4FF0010B00239A
:1096D000ACE73D46D04508BF4FF0010BF7E703204C
:1096E000E4E60846E2E64023FFF7D7BE704708B538
:1096F0000020F9F705F808B50120F9F701F88368AB
:109700001B6A03B11847704743681B6810B51C6893
:109710002046FFF7F4FFA368DB6A0BB120469847A9
:10972000002010BD08B543681B68197411B1186892
:10973000FFF7E5FF002008BD10B51C464368D86858
:10974000FFF783FE2060002010BD2DE9F041456841
:109750001E462B681B7C0C46174653B101EB0208D2
:1097600044452B6820D1D3E901213760012090477F
:1097700017E0A868FFF717FE2B6830600C33012153
:10978000BFF35B8F53E8002F43E800100028F9D1A6
:10979000BFF35B8F2AB92B6818688368DB6903B154
:1097A00098470020BDE8F081186814F8011B836811
:1097B0005B689847D4E72DE9F34104460D4683687A
:1097C0005B6C03B19847A3685B6B03BB4FF0000869
:1097D000E86801A9C269FFF7B2FDA368074600283F
:1097E00034D09B69019933B3024620469847064618
:1097F00020B3E8683146FFF7C1FDB7424FF00108DA
:10980000E6D02B680020D3E90121904703E02046F1
:1098100098470028DAD1A3685B6A03BBA86801A94E
:10982000C269FFF7DFFD064600BB2046FFF767FF72
:109830002B68DE6025E06FF05706DAE70146E8683E
:10984000FFF79CFDB8F1000FE5D0DAE79B69002B2C
:10985000F8D001220DF1030120469847F2E7204697
:1098600098470028DAD102B0BDE8F081A3680199D9
:109870005B6963B10246204698470146A868FFF736
:10988000CFFD2B680120D3E901219047EBE76FF072
:109890005701F3E710B50346BFF35B8F53E8000FA2
:1098A00040EA010243E80024002CF7D1BFF35B8FAC
:1098B00010BD10B50346BFF35B8F53E8000F00EAFD
:1098C000010243E80024002CF7D1BFF35B8F10BDE9
:1098D00073B58568090101F51A71044616460D44F1
:1098E00001AA6946284602F013FB009B23B12846D3
:1098F00002F00BFB2046B04702B070BD08B510B1B6
:1099000001F03EF880B208BD0EB403B503AA52F8C8
:10991000041B0192FAF77CF902B05DF804EB03B086
:109920007047FEF7F5B98B6820B903F51A7000216E
:10993000FFF700B803F52670F9E738B58368D3F868
:109940006432DB0704461AD4406803685B689847B2
:10995000054620B9E06800F0D5FDA3681D71A36835
:109960005B6B13B1294620469847A3680022C3F8D1
:109970000C23FEF7BDFDBDE83840FBF743BA6FF09E
:109980000F05ECE700F5197011B10421FFF782BF54
:109990006FF00401FFF78DBF08B500F5187029B10D
:1099A0000121FFF777FF00F0010008BD6FF0010112
:1099B000FFF77FFFF7E7FEF723BAF8B504468068A4
:1099C0001F460379022B0D46164607D0BDE8F84026
:1099D0004FF4805100F51970FFF75CBF4FF0FF3274
:1099E0004FF0FF3300F53E70FFF79BFFA368D3F8FD
:1099F0006422110504D49B6B13B9204600F058FB78
:109A00003B4632462946204600F0B2FBA368D3F815
:109A10006422120504D49B6B13B92046FAF784FA2A
:109A2000606900F044F8A068BDE8F84000F53E70B9
:109A3000FFF7C1BF0CB407B504AB53F8042B019377
:109A4000FFF7BBFF03B05DF804EB02B070472DE9F0
:109A5000F04107460E4614460D460CB9BDE8F081AC
:109A6000102CA04628BF4FF010082A46A91B4346D9
:109A70003846FAF75BF8A4EB08044544EDE710B567
:109A8000044680684FF0FF324FF0FF3300F53E7020
:109A9000FFF747FF2046F9F707FAA068BDE8104036
:109AA00000F53E70FFF787BF8368996370470269CE
:109AB00083681268016810B50446C0689847236936
:109AC00000221A6010BD38B5CB681B7C022B0546FE
:109AD0000C4604D10A2802D10D20FFF7F4FF2369B8
:109AE00022681B68D55422691368013313606268C9
:109AF000934202D12046FFF7DAFF002038BD20282C
:109B000005D0093804288CBF0020012070470120AF
:109B1000704708B510B100F033FF80B208BD10B532
:109B2000047B438922442144B2FBF3F003FB10225F
:109B3000B1FBF3F003FB1010101A10BD10B5047B3D
:109B4000438921441019B1FBF3F1B0FBF3F0401A43
:109B500010BD30B5057B43892944B1FBF3F403FB09
:109B6000141101312A4401340180B2FBF3F103FBEB
:109B70001122848001324C1CC480428030BD2DE90A
:109B8000F74F002607468846144699460660B246B7
:109B90002078002800F0BD80FFF7B1FF20B104F865
:109BA00001ABF5E70026F3E73A68531C4B453B60F1
:109BB00048F8224000F0AD8006462278002AE7D01F
:109BC000A6B9164623461C46272E04D05C2E20D06C
:109BD000222E40F091802046FFF79BFF611C024639
:109BE000204600F00DFF2278002AD1D0B242A346D1
:109BF00004F101041BD15846FFF78BFF21460246B2
:109C0000584600F0FDFE9BF800605C46002ED9D15E
:109C1000BEE72046FFF77DFF651C02462946204629
:109C200000F0EEFE66782C46002ECDD1B0E75C2A1F
:109C30009BF80120D8D1B242104608D15846FFF710
:109C400068FF21460246584600F0DAFEB5E7302AA2
:109C500025D1022300251BF80300A0F13001C9B271
:109C6000072919D8ED000133EDB2052B45EA0105AE
:109C7000F1D1591E5944584601930091FFF749FF0D
:109C8000019B0099023BC21A584600F0B9FE9BF8AE
:109C900001208BF80050A7E7DBB2022BE9D178282E
:109CA00025D1022100251BF80130A3F13000C0B2FC
:109CB000092808D82D01EDB20543022901D004235B
:109CC000D7E70321EFE7A3F16100052805D82D01AF
:109CD000EDB2573B1D43EDB2EFE7A3F1410005287C
:109CE00003D82D01EDB2373BF4E7022902D10BF185
:109CF000010479E70323BCE73046FFF700FF0028A3
:109D00007FF450AF6678631C002E7FF45CAF1C4676
:109D10003EE7304603B0BDE8F08FF8B50E46114679
:109D20001546074600F0E0FD04462846FFF7F1FE21
:109D30000546C4B1A74207D214F8013C202B02BF4C
:109D40000135ADB204F1FF342046FFF7E2FE33885F
:109D5000421C5B1B521B33806119204692B2BDE846
:109D6000F84000F04DBEF8BD2DE9F041884686B0C0
:109D70001746044628B10146142201A800F057FEF8
:109D800001AC002631463A462046F9F755FF013628
:109D9000054628B12968404600F002FE0028F1D1AE
:109DA000284606B0BDE8F0812DE9F0471C46DDF8F5
:109DB00020809DF8249000230F46164623602368D8
:109DC000BB4205461BD256F8230000F014FC236862
:109DD000824618B1013323602846F0E756F8231075
:109DE00042462846FFF7C0FF48B123685A1C22604C
:109DF000B9F1000FE3D08045E1D1236055462846F4
:109E0000BDE8F0872DE9F0410746FFF782FE0646E0
:109E100037BBBDE8F08154B18AB2B21A01330132C6
:109E20003944F81800F0ECFD341BA6B24446731E0A
:109E30009D42EEDA785DFFF762FE2B460135ADB24A
:109E40000028F4D029468AB29642F0D9785CFFF710
:109E500056FE80460028DED001340131A4B2F2E77C
:109E600000252C46E3E7F8B5846894F842300546AF
:109E700053B9AB689A8FDA87F8BD013A92B2A287DC
:109E800022B984F84220F4E704F14206A28FB31805
:109E900013F8010CFFF733FE03460028EDD1B05450
:109EA0009AB216FA83F1B05CFFF729FE1F46013320
:109EB0000028F5D1BFB2002FDBD0A38F01339A1A4F
:109EC000304600F09DFDA38FDB1BA387D1E70EB4C6
:109ED00003B503AA52F8041B0192F9F799FE02B0E8
:109EE0005DF804EB03B0704738B583680446186822
:109EF0009D8F10B100F044FD80B2A268528D4319CD
:109F0000B3FBF2F102FB1130B0FA80F0400938BD2A
:109F100038B5836804461868DD8F10B100F030FD55
:109F200080B2A268528D4319B3FBF2F102FB1130EB
:109F3000B0FA80F0400938BD10B50446FFF7E8FFDD
:109F400020B16069BDE81040F9F7AABE2046FFF7CE
:109F5000CBFF0028F5D110BDF8B584680546A28F67
:109F6000E18F04F12000FFF7F4FD2846A78CE68C72
:109F7000FFF7BAFF10B16869F9F792FEB74207D14F
:109F8000218C638C2846C91ABDE8F840F9F7A4BEB5
:109F9000E18CA38C2846C91AF9F788FEF0E7F8B5DA
:109FA000044680680D46C18F828F20300D44FFF734
:109FB000D0FDA068ADB2C18F2A462030FFF7BEFDAC
:109FC0000746A0682A46C18F2030FFF7A8FD7942D6
:109FD00006462046F9F76AFE31462046F9F77CFE30
:109FE000A368DD87F8BD2DE9F0410C1E064636DA80
:109FF000644224B24FF0FF35A4B2AFB216E0B368AA
:10A00000B3F83EC0B3F83C8003F1420E6146002233
:10A0100081B96B1C02D0B8F1000F0FD1A1EB0C017C
:10A0200009B23046FFF7BBFF013CA4B2002CE6D1D9
:10A03000BDE8F081884501D1012DEFD01EF8013037
:10A0400043F020006138192807D9303B092B04D987
:10A05000002AE3D1394489B2DAE70122FAE701257F
:10A06000CAE78368D98F494209B2FFF798BF83686E
:10A07000998FDB8FC91A09B2FFF791BF8368DB8F15
:10A080001BB14FF0FF31FFF78ABF70478368DA8F4B
:10A090009B8F9A4202D20121FFF781BF70478368EC
:10A0A000DA8F9A871344002283F84220F9F7ECBD37
:10A0B00010B504468068828FC18F2030FFF749FDBC
:10A0C000A368198C2046C1F10101F9F705FEA368C8
:10A0D000998C20460139F9F7E9FD2046BDE810408A
:10A0E000F9F7D2BD2DE9F041054686B00F4614467A
:10A0F0000026A4B906B0BDE8F081D3F86422920727
:10A10000FBD5BFF35B8F03F5197353E8001F21F0F4
:10A11000020143E80012002AF7D1BFF35B8F6868A1
:10A1200003682246D3F80C80B9196B46C047009AE1
:10A130001644A41A002ADCD1AB6819790329EED0A1
:10A140000229DAD803F52673012101A801F0BBFE2C
:10A150004FF0FF324FF0FF33012101A8FEF78EFBD5
:10A16000A86800F5267001F0D0FED8E7FFF7BABF67
:10A17000F7B50F4681681E46D1F86032DB0604460B
:10A18000154617D591F82E30BB4213D002222E313E
:10A1900001A800F04CFC39462046F9F7BBFD606988
:10A1A00032462946F9F734FD01A92046F9F7D2FDD8
:10A1B00003B0F0BD60693246294603B0BDE8F04007
:10A1C000F9F726BD0CB407B504AB53F8042B019383
:10A1D000FFF7CEFF03B05DF804EB02B070472DE946
:10A1E000F0418668B58FAB18FF2B074688461446AA
:10A1F0001EDCF38FED1A42331E44ADB22A463146BF
:10A20000301900F0FDFB22464146304600F00FFCBD
:10A21000B9688B8F23449BB28B870B44002283F851
:10A220004220D1F860329B0704D4CB8F1C44CC87EA
:10A23000BDE8F08129463846BDE8F041F9F706BE91
:10A24000FFF7CDBF38B505468068C28F848FA41A4A
:10A25000A4B28CB142321044411C224600F0D0FB23
:10A26000AA68938F611E013B938728460122BDE8AF
:10A27000384089B2F9F7EABD38BD83689A8F10B5C6
:10A28000044652B1DB8F43B14FF0FF31FFF787FE39
:10A290002046BDE81040FFF7D5BF10BD0EB403B592
:10A2A00003AA52F8041B0192F9F7B2FC02B05DF860
:10A2B00004EB03B070472DE9F843054690460E467F
:10A2C000002966D00024335D202B02D0093B042BEB
:10A2D0003ED80134F7E74B460027B84214D013F8B4
:10A2E000012B0A2A19D16869FFF7E1FB49463A4672
:10A2F0002846FFF7F7FE6869F9F72EFE013441465C
:10A3000028463C44F9F7E8FC68693119FFF7C6FFB5
:10A310006869BDE8F843F9F71FBE0137DDE71F465E
:10A320006869FFF7C4FB3A4649462846FFF7DAFE5C
:10A330003C44335D202B02D0093B042B01D801346F
:10A34000F7E76869F9F708FE41462846F9F7C4FCC3
:10A35000304600F015FBAB68598D80B2001BA1EBB5
:10A360000803984206EB0409B5D94846002710F8BF
:10A37000012B202A06D0A2F1090CBCF1040F02D84F
:10A380000A2ACDD03B4608EB07029142C7D90137D4
:10A39000EDE7BDE8F88383690020186070470EB4CC
:10A3A00003B503AA52F8041B0192F9F731FC02B07D
:10A3B0005DF804EB03B070478368BFF35B8F03F570
:10A3C000187353E8001F21F0080143E80012002A27
:10A3D000F7D1BFF35B8F002070478368BFF35B8FBB
:10A3E00003F5187353E8001F41F0080143E8001219
:10A3F000002AF7D1BFF35B8F002070478368BFF35B
:10A400005B8F03F5187353E8001F21F0020143E846
:10A410000012002AF7D1BFF35B8F002070478368DA
:10A42000BFF35B8F03F5187353E8001F21F0100191
:10A4300043E80012002AF7D1BFF35B8F002070477A
:10A440008368BFF35B8F03F5187353E8001F41F077
:10A45000100143E80012002AF7D1BFF35B8F002000
:10A4600070478368BFF35B8F03F5187353E8001FD1
:10A4700041F0020143E80012002AF7D1BFF35B8FDD
:10A480000020704708B583680068D3E900210A609E
:10A4900051600021C3E900111A895B891A440C320A
:10A4A000FEF7D3FF012008BD0023C3607047F8B555
:10A4B0001F460346164653F8044F9C4202D1002023
:10A4C0003880F8BDC568B1B9002DF8D0AC4202D1D2
:10A4D0000023C360F3E76C68C460002CEFD02289CE
:10A4E00004F10C01304600F0A2FA23893B800022DF
:10A4F000F2540120E5E7002DEED08368AB42E7D0AF
:10A500002C68E9E738B50446051D6368AB4204D002
:10A510002046FFF7B7FF0028F7D138BD2DE9F04FEF
:10A52000036802F10C05C5F10009DB6909F00309B4
:10A5300085B04D449D4204460191174610D8002332
:10A54000C3606AB1466800F1040AB2450BD05EB13F
:10A550003389934208D106F10C0000F041FA18B992
:10A5600005B0BDE8F08F1E464FF000082068026974
:10A5700083689A4201BFC0E90288C0E90588C0F833
:10A580000480C0F810802A4603A9FEF7D8FE854251
:10A5900083461ED920682A4603A9FEF7D0FE8542CD
:10A5A00018D172895A447281AB44039D01992F815D
:10A5B0003A46A5F80A9005F10C0000F038FA6268F6
:10A5C0002068C5E9002A594655606560FEF7D6FE49
:10A5D000C6E7EAD020680021FEF7D0FE63689A45FE
:10A5E000C4D02046FFF74EFFC0E7031DC0E901338A
:10A5F0000023C360704710B5044628B100F0C0F9CD
:10A60000002380B2984201D8002010BDE25C3F2AAE
:10A6100003D02A2A01D00133F4E70120F5E710B571
:10A62000044680684FF48072002100F5A17000F0AC
:10A6300009FAA068828F00F1420100F5A17000F0D4
:10A64000F6F9A06800F5A170FFF7DCFBA06800F543
:10A65000A17000F095F9A3680130A3F8400010BD87
:10A6600010B504468068B0F8402000F5A171423072
:10A6700000F0DDF9A368B3F840209A8710BD08B553
:10A680000020F8F73DF801F02DB90146006801F00F
:10A6900029B9013140B2FAF70BB900210120FFF7C7
:10A6A000F2BF38B504460D4611461A46FAF7D8F8F7
:10A6B00060B2691CFAF7FCF8204638BD08B5FAF715
:10A6C0003BF9BDE80840FAF719BA10B50278202A1C
:10A6D000034600F10100F9D0A2F109010429F5D9DE
:10A6E0002B2A08D02D2A0ABF034600210121013B55
:10A6F00000200A2404E003460021F8E76043801AA2
:10A7000013F8012F303A092AF8D901B9404210BD97
:10A710002DE9F843844688460446214614F8013B57
:10A72000202BFAD0A3F109000428F6D92D2B23D130
:10A730004B788C1C01212ABB302B30D00A2201F12E
:10A740000047013F0026B7FBF2FE304602FB1E79B0
:10A75000A3F13005092D29D82B469A4236DD751C08
:10A7600007D070452FD801D14B452CDC00FB0230BF
:10A77000012614F8013BEBE72B2B04BF4B788C1C14
:10A780000021D8E7102ADAD1302BD8D1207800F078
:10A79000DF005828D3D1637810220234CFE7227823
:10A7A00002F0DF02582AF6D00822C8E743F020055D
:10A7B000613D192D0AD8A3F141051A2D34BF372563
:10A7C00057255B1BC9E74FF0FF36D2E7731C09D151
:10A7D000FCF7EAFF222303603846B8F1000F07D1E7
:10A7E000BDE8F88301B14042B8F1000FF8D00EB1D6
:10A7F00004F1FF3CC8F800C0F2E72DE9F0418446BF
:10A800000F460446214614F8013B202BFAD0A3F151
:10A8100009000428F6D92D2B25D14B788C1C4FF03C
:10A82000010E3ABB302B32D00A224FF0FF31002507
:10A83000B1FBF2F102FB01F86FEA08082846A3F128
:10A840003006092E2AD833469A4237DD6E1C07D0CF
:10A85000884230D801D143452DDC00FB0230012570
:10A8600014F8013BEBE72B2B04BF4B788C1C4FF00B
:10A87000000ED6E7102AD8D1302BD6D1217801F09E
:10A88000DF015829D1D1637810220234CDE7227834
:10A8900002F0DF02582AF6D00822C6E743F020066D
:10A8A000613E192E0AD8A3F141061A2E34BF37266D
:10A8B00057269B1BC8E74FF0FF35D1E76B1C07D12C
:10A8C000FCF772FF22230360284647B9BDE8F081F8
:10A8D000BEF1000F00D04042002FF7D00DB104F1BF
:10A8E000FF3CC7F800C0F1E72DE9F04191F8008086
:10A8F0000546B8F1000F10D04C1C204600F040F87F
:10A9000007462E4616F8013B63B1984508D13A46F2
:10A910002146304600F050F810B92846BDE8F081D5
:10A920003546EEE71D46F8E70139034611F8012FD9
:10A930000AB91A70704703F8012BF7E710B501390F
:10A94000034622B91A440021934208D110BD11F8E0
:10A95000014F002CF6D003F8014B013AF1E703F860
:10A96000011BF1E7C9B203461A788A42184603F17F
:10A97000010304D0002AF7D1002918BF0020704736
:10A98000034600201A5C02B970470130FAE703461B
:10A9900000201A5C0AB1884200D170470130F8E704
:10A9A000431E013913F8012F11F8010F824201D122
:10A9B000002AF7D1101A704770B50B4605466AB1E8
:10A9C00010F8016B1C78B44201F1010100D11CB9EF
:10A9D0002A781B78D01A02E0013AEEE7104670BDE3
:10A9E00010B55AB10139841810F8012B11F8013F44
:10A9F000A04201D09A42F7D0D01A10BD1046FCE711
:10AA0000431A934210B500EB020308D30139024602
:10AA10009A420BD011F8014F02F8014BF8E70A44B3
:10AA200012F8014D03F8014D8A42F9D110BD10B55D
:10AA3000431E0A44914200D110BD11F8014B03F8A6
:10AA4000014FF7E7C9B202440346934200D1704771
:10AA500003F8011BF9E74B68012B07DD0B68187041
:10AA60000B6801330B604B68013B4B600020704763
:10AA7000062808D14FF080430122C3F80025BFF318
:10AA80004F8F20BFFDE77047002383F31188BFF38A
:10AA90006F8F70470369C9B20C2201FB0233186C37
:10AAA00000F0070070474FF02003EFF3118283F3AB
:10AAB0001288BFF36F8F036803F0C00343F00203F3
:10AAC000036082F31188BFF36F8F704770B503691D
:10AAD000C9B24FF02004EFF3118584F31288BFF35D
:10AAE0006F8F0C2606FB0134246C14F0C00408D0D0
:10AAF000A24206D085F31188BFF36F8F4FF0FF306D
:10AB000070BD06FB013301221A6485F31188BFF37F
:10AB10006F8F436803EBC1035B6898470020EFE742
:10AB20008022FFF7D3BFF8B5069F0469C9B24FF082
:10AB30002005EFF3118685F31288BFF36F8F0C2584
:10AB400005FB0144256C05F0070CBCF1010F0CD18D
:10AB5000276486F31188BFF36F8FC4E90E2343681F
:10AB600053F8313098470020F8BD05F0C005AF42DA
:10AB700086F31188BFF36F8F0CBF6FF077004FF033
:10AB8000FF30F1E713B580240094FFF7CCFF02B04B
:10AB900010BD006910B4CBB21C2403FB04000021DB
:10ABA00010BC1047002000F0FCBC002000F035BDB8
:10ABB0001046FDF769B943685B68D3F810350B6040
:10ABC0000020704743685B68D3F8040542400A40A0
:10ABD0004240C3F804250020704743685B680020AA
:10ABE000C3F80815704743685B680020C3F80C156C
:10ABF000704743685A68D2F804354B40C2F80435B0
:10AC0000002070470369586810B548B1884213D1D5
:10AC10009C6808685860A14200D1986000200860D4
:10AC20007AB9002010BD814206D10868206098687A
:10AC30008142F3D19C60F1E7044600680028F2D11C
:10AC40003AB15A680A609A685960002AE9D1996055
:10AC5000E7E76FF01500E5E730B50B6813B913604F
:10AC6000184604E00468656815B12068156030BDB9
:10AC70000834013B04600B60EFE703460A460068B6
:10AC80001979012303FA01F103691B68194218BFFE
:10AC900082F0010212B18368DB68184783681B6980
:10ACA000FBE738B503680446E3B19868D0B105689E
:10ACB000C5B149B10121FFF7E0FF23689B6898689F
:10ACC000BDE8384000F0CABF12B99B88DB0409D444
:10ACD000806800F0C3FF236800219868BDE8384011
:10ACE000FFF7CBBF38BD10B5012200210446FFF7A6
:10ACF000D8FFA36933B9636004F11000BDE81040C8
:10AD0000FDF7C2B810BD006903688B4210B506D1CB
:10AD100090F86C4034B9FFF7E6FF204610BD6FF0A5
:10AD20001500FBE76FF00F00F8E72DE9F34104464B
:10AD30000569002201210320FFF7ABFC6368DC6991
:10AD400001AA0021204600F073FB002841DB019B93
:10AD500022681979186800F0A2FB002839DBAC687A
:10AD600001260834D5E9023203EBC203A4F108023C
:10AD7000934204D82846FFF7B6FF002029E054F894
:10AD8000080C00F08DFD38B354F8080C14F8041CBE
:10AD900034F8023CD0F810C0D0F80880DCF800701D
:10ADA000DA0754BF43F4B01383F4D01323F48012B2
:10ADB00006FA01FEDB074CBF4EEA070727EA0E073B
:10ADC000D8F80030CCF800709847002804F1080447
:10ADD000C8DA02B0BDE8F0816FF01200F9E738B5CB
:10ADE00003780C46002B3CD18B6D8D6E93B19D4248
:10ADF00010D85B1B8B6543BB4B6C08334B648B6C6F
:10AE0000013B8B6401F1580204F144004831FFF723
:10AE100023FF6065236E9BB19D4211D85B1B2366A7
:10AE2000CBB9E36C0833E364236D013B236504F184
:10AE3000600204F1500104F14C00FFF70DFFE065E2
:10AE4000606EBDE83840FAF77BBC4B6D002BE1D05B
:10AE50002B444B65DEE7E36D002BF1D02B44E3651B
:10AE6000EEE738BD30B50B6813B91360184604E03F
:10AE70000468656815B12068156030BD0834013B71
:10AE800004600B60EFE703460A4600681979012366
:10AE900003FA01F103691B68194218BF82F001022D
:10AEA00012B18368DB68184783681B69FBE738B514
:10AEB00003680446E3B19868D0B10568C5B149B1EB
:10AEC0000121FFF7E0FF23689B689868BDE83840E0
:10AED00000F0C4BE12B99B88DB0409D4806800F07E
:10AEE000BDFE236800219868BDE83840FFF7CBBF5E
:10AEF00038BD10B5012200210446FFF7D8FFA36931
:10AF000033B9636004F11000BDE81040FCF7BCBF2A
:10AF100010BD006903688B4210B506D190F86C40F3
:10AF200034B9FFF7E6FF204610BD6FF01500FBE7D0
:10AF30006FF00F00F8E72DE9F341044605690022A0
:10AF400001212F20FFF7A5FB63689C6A01AA00215D
:10AF5000204600F06DFA002841DB019B2268197938
:10AF6000186800F09CFA002839DBAC680126083428
:10AF7000D5E9023203EBC203A4F10802934204D8DC
:10AF80002846FFF7B6FF002029E054F8080C00F02F
:10AF900087FC38B354F8080C14F8041C34F8023C4D
:10AFA000D0F810C0D0F80880DCF80070DA0754BF81
:10AFB00043F4B01383F4D01323F4801206FA01FE95
:10AFC000DB074CBF4EEA070727EA0E07D8F8003028
:10AFD000CCF800709847002804F10804C8DA02B0E1
:10AFE000BDE8F0816FF01200F9E738B503780C4640
:10AFF000002B3CD18B6D8D6E93B19D4210D85B1BA5
:10B000008B6543BB4B6C08334B648B6C013B8B648F
:10B0100001F1580204F144004831FFF723FF606555
:10B02000236E9BB19D4211D85B1B2366CBB9E36CA9
:10B030000833E364236D013B236504F1600204F1EE
:10B04000500104F14C00FFF70DFFE065606EBDE8B4
:10B050003840FAF7E1BC4B6D002BE1D02B444B6537
:10B06000DEE7E36D002BF1D02B44E365EEE738BD5E
:10B0700002690B46D2E9010183E803000020704712
:10B0800043681B68D3F88004C3F8800470474368A2
:10B0900002691B68D3F8100148B1527D0A70002084
:10B0A000C3F81001D3F8102101221A6070474FF045
:10B0B000FF307047002A10B504460FDD43681B6857
:10B0C000D3F8100148B122690020C3F81001D3F869
:10B0D0001001527D0A700120186010BD0020FCE7AD
:10B0E000436801691A684FF02000EFF3118380F381
:10B0F0001288BFF36F8FC968002088734FF48001F6
:10B10000C2F8041383F31188BFF36F8F704703698C
:10B11000DB6801229A7370470369DB689A7B02F04F
:10B12000FF0162B942681268D2F8580140B1D2F802
:10B13000040310F4800003D019610120704700203F
:10B14000704743681B68D3F81001003818BF01200E
:10B15000704743681B681022C3F804237047436894
:10B160001B681022C3F80823704743681B684FF41C
:10B170000072C3F80423704743681B684FF40072E1
:10B18000C3F80823704738B543681D68D5F8043301
:10B190005B02044605D4D5F8040310F0100006D174
:10B1A00038BDFFF7B9FF0028F5D00120F8E72046A9
:10B1B000FFF7C7FF003818BF0120F1E701207047F3
:10B1C0000369DB68C3E9001270470368C3F84415DC
:10B1D000C3F848250022C3F82021D3F82011C3F872
:10B1E0005821D3F858214268D20641BF0822C3F83B
:10B1F00000254FF48002C3F8042301229A607047AF
:10B2000002680346D2F8580140B95B689B0706D430
:10B21000D2F82001003818BF012070470120704784
:10B22000F8B50569EB689C89BFF35B8F9442A8BFB2
:10B2300014461033012253E8006F002E03D143E877
:10B240000027002FF7D1BFF35B8F0CBF13460023FD
:10B250001ED01C462046F8BDEA68CE5C9268D654E3
:10B260000133A342F8DB4FF02003EFF3118783F3A0
:10B270001288BFF36F8F46683046FFF7C1FFEB6857
:10B2800040B91861044687F31188BFF36F8FE1E777
:10B290000023E6E7996822463046FFF796FFF2E77B
:10B2A00042681368D3F80413C90510B418D5D3F84D
:10B2B0002011A9B14FF02004EFF3118184F312881B
:10B2C000BFF36F8FD3F8204134B10024C3F820417D
:10B2D000D3F820410124DC6081F31188BFF36F8F24
:10B2E0005268D2061AD54FF02002EFF3118182F393
:10B2F0001288BFF36F8FD3F8582112B10022C3F820
:10B3000000250269D2680AB112691AB94FF48002A5
:10B31000C3F8082381F31188BFF36F8F0269D268E5
:10B320005AB1D3F8581151B1947B0021116134B155
:10B330004FF48000C3F80803917310BC7047D3F832
:10B34000241121B10021C3F82411D3F8243113684A
:10B35000002BF2D0516810BC18472DE9F341466824
:10B3600005693468F7680021C4F800158046286034
:10B3700001AA384600F05CF8002833DB019B3A68EC
:10B380001979186800F08BF800282BDB291D40463E
:10B39000FAF7DEFC30BB0823C4F80035337A5BB91A
:10B3A000C4F81001D4F8103105F11503C4F8343590
:10B3B0000123C4F83835236073689A075CBF4FF4E3
:10B3C0008072C4F80423DB0644BF4FF48003C4F842
:10B3D000043314350023C4F84455C4F84835012318
:10B3E000A360E36002B0BDE8F08110B5002204461E
:10B3F00001212820FFF74DF92820F9F76DFA2046A2
:10B40000BDE81040FFF7A9BF10B500220446012196
:10B410000220FFF73EF90220F9F75EFA2046BDE868
:10B420001040FFF79ABF704708B5FAF71FFE08BD36
:10B4300030B543681360037A03F10053013BDB002E
:10B44000456814681D44AC4202D96FF0010030BD5C
:10B4500065798D4202D008341460F1E70020F6E7E8
:10B4600037B500F48053002B044600F03F0301A8D9
:10B470000EBF1546012500210193FAF7ABFFC4F377
:10B48000811304F4706444EA8304019B0C4303F5C4
:10B49000E07344EA450440F8234003B030BD73B57F
:10B4A0001546044600EB8106B44202D1002002B0EA
:10B4B00070BD23681A0C062A51D8DFE802F0041781
:10B4C0001D4B22394B0003F03F03C5F80C352368B0
:10B4D00001A803F03F030193FAF77CFF019B0122CF
:10B4E00002FA03F3C0F8083511461CE003F03F03ED
:10B4F000C5F814350022F7E703F03F03C5F8083517
:10B50000E5E703F03F03C5F80835236801A803F019
:10B510003F030193FAF75EFF019B012101FA03F358
:10B52000C0F80C3500222068FFF79AFF0434BBE70F
:10B5300003F03F03C5F80C35236801A803F03F036F
:10B540000193FAF747FF019B012202FA03F3C0F8C7
:10B550000C35C9E703F03F03C5F81035CAE76FF0B3
:10B560008500A4E708B50020F9F758FDFDF75ABBA0
:10B5700008B5F9F7ABF8F9F75DF9BDE80840FDF754
:10B5800051BB004700F06ABB08B50020F9F7C6F9C7
:10B5900008B9F9F7A1F94FF080430022C3F8182544
:10B5A00008BD08B510B101282CD008BD4FF080426D
:10B5B000D2F81834D2F81814C8030BD4D2F81434C3
:10B5C000D9070FD5D2F81C349B0708D40223C2F840
:10B5D0000433EAE703F00303012B04D013B1002086
:10B5E000FBF73EF800234FF08042C2F818350023E5
:10B5F000C2F80431D2F804310223C2F80433012323
:10B600009360D2E74FF080430022C3F80021D3F8C3
:10B610000021C3F804031860C7E7FBF721B8F7B5AA
:10B62000019001A8DDE9084716461D46FBF7C0F862
:10B63000019BB6F1000C18BF4FF0010C00EB83002A
:10B640000B1E18BF0123002D43EA4C0314BF4FF01B
:10B650000C0C4FF0000C002C43EA0C0314BF4FF409
:10B66000E06C4FF0000C002F43EA0C03D0F80027E9
:10B6700014BF4FF4403C4FF0000C43EA0C0322EAA5
:10B68000030301B109780EB13678760019430DB184
:10B690002D78AD0031430CB12478240229430FB139
:10B6A0003F783F040C433C43C0F8004703B0F0BD73
:10B6B0001FB50DF10F03019300238DF80F100093B8
:10B6C0001A461946FFF7ABFF05B05DF804FB07B556
:10B6D000019001A8FBF7D8FB019B03F5E073022260
:10B6E00040F8232003B05DF804FB07B5019001A8E2
:10B6F000FBF7CAFB019A01239340C0F8083503B059
:10B700005DF804FB07B5019001A8FBF7BDFB019AAA
:10B7100001239340C0F80C3503B05DF804FB37B546
:10B72000D0F818358A69DBB28DF807300B6A93427E
:10B730003EBF4A699DF80740D4540B6A91F82450E3
:10B740000C695A1C0A62023335B1A3428C6938BFB6
:10B750000B619C4288BF8B610D699D4205D9CA6807
:10B76000D35CC0F81C3501200AE08C699C4201D9E9
:10B77000CB7FF6E7AA42F6D3A2422CBF00200120DD
:10B7800003B030BD07B5019001A8FBF711FD019A88
:10B7900001239340C0F8083503B05DF804FB07B5FA
:10B7A000019001A8FBF704FD019A01239340C0F822
:10B7B0000C3503B05DF804FB431C07B509D00190BC
:10B7C00001A8FBF7F5FC019B03F5E073022240F8AA
:10B7D000232003B05DF804FB837F5A070BD4C07F9E
:10B7E000FF2808D09B0758BF81F0010109B9FFF776
:10B7F000D6BFFFF7C7BF70472DE9F04700240646C4
:10B800000F46904600F5A0754FF48039A2462B688C
:10B810007BB1D6F8043309FA04F21A4209D0A00029
:10B82000C5F800A02B6800F5A07398B2D7E90031E5
:10B8300098470134444505F10405E8D1BDE8F08797
:10B8400003680122DA60704730B54FF48034006835
:10B850008C4063B18B0003F5A0730025C550C3581D
:10B86000C0F8044301F5A87140F8212030BDC0F8AC
:10B870000843F7E770B4046840F20116D4F80052A8
:10B880008E4025EA0605C4F80052D4F800522B4336
:10B89000C4F800329DF80C3070BCFFF7D5BF70477C
:10B8A00038B1C3681888C0F30800A0F58073584207
:10B8B00058417047406970B413460D4660B901465F
:10B8C0002A4670BCFBF7EABE013130F8114034441F
:10B8D000A4B29442F8D9F3E7002147F6FF764FF679
:10B8E000FD72F2E7F8B505460E464FF02003EFF380
:10B8F000118783F31288BFF36F8FFCF7F9FD314690
:10B9000004462846FFF72EFE87F31188BFF36F8F9A
:10B910002046BDE8F840F9F775BAFFF793B8FFF78E
:10B9200086B830B50024846141EA020414F00304AF
:10B93000C0E9023201610CD12546A342456103D121
:10B94000C0E90000002030BD0D6001340D461144F7
:10B95000F3E76FF01500F6E7F8B504460D464FF033
:10B960002003EFF3118683F31288BFF36F8F4769CB
:10B970007FB900F0C1F860B12A684261C0F8B070C8
:10B9800000F0AAF8314604F10800BDE8F840FCF7E1
:10B9900075BC2B6862691A602B686361A369013BFF
:10B9A000A36186F31188BFF36F8FF8BDEFF30580B5
:10B9B000003818BF0120704778307047FCF770BC22
:10B9C00010B500238B4202D11360002010BDC45C6F
:10B9D000AA2CF9D10133F5E70A46D0E92701FFF790
:10B9E000EFBF08B5F8F762FDBDE80840FFF71BBDE3
:10B9F00090F90E308B4201D0FCF7FABB0020704763
:10BA000003460020C3E90200C3E900337047D0E9D0
:10BA1000003213605A600023C0E90033704708B554
:10BA2000FFF7F5FF437B23F002034373002383609A
:10BA300008BD90F90E3091F90E00834214BFC01A70
:10BA40000020704710B501464FF02003EFF311843A
:10BA500083F31288BFF36F8F10F80B3C13F0280F9D
:10BA60000DD151F8103C18380BB1FFF7D8FF11F881
:10BA70000B3C23F0140301F80B3CFCF7BFFA84F3F2
:10BA80001188BFF36F8F10BD38B504460D46FCF723
:10BA9000E9FA637B43F002036373E5B12B68A560A9
:10BAA0009D4209D16B68C4E900531C606C6012E0D0
:10BAB0006A689342F6D01B68002BF3D094F90E20ED
:10BAC00093F90E108A42F3D09142F1DD5A68C4E92D
:10BAD000003214605C6038BD10B54FF02003EFF306
:10BAE000118483F31288BFF36F8FFCF787FA84F316
:10BAF0001188BFF36F8F10BD38B54FF02003EFF3FF
:10BB0000118583F31288BFF36F8F0468A0420DD0B4
:10BB100034B12046FFF783FF04F1180000F056F817
:10BB200085F31188BFF36F8F204638BD0024F7E7F7
:10BB300010B54FF02003EFF3118483F31288BFF3A5
:10BB40006F8FFFF76CFF84F31188BFF36F8FBDE831
:10BB50001040183000F03AB8034620B9EFF30582E0
:10BB60000AB9F8F709BF83F31188BFF36F8F7047E5
:10BB70004FF02003EFF3118083F31288BFF36F8F30
:10BB8000FFF7EABF38B54FF02003EFF3118583F3D9
:10BB90001288BFF36F8F0468A04213D0A4B1C4F819
:10BBA000B01062612046FFF73AFF04F1180000F080
:10BBB0000DF82046FCF722FA012085F31188BFF327
:10BBC0006F8F38BD0020F8E72046F6E710B54FF03C
:10BBD0002002EFF3118482F31288BFF36F8F0368A2
:10BBE0003BB1FCF73FFD002084F31188BFF36F8F5A
:10BBF00010BD6FF01500F7E710B54FF02003EFF31D
:10BC0000118483F31288BFF36F8FFCF703FD84F375
:10BC10001188BFF36F8F10BD70B504460D464FF00D
:10BC20002003EFF3118683F31288BFF36F8FFCF7C5
:10BC3000F1FC012807DDA04205DBA0422946A8BF90
:10BC40002046FAF78BFB86F31188BFF36F8F70BD28
:10BC500008B5FCF7FBFD08BDFCF7F8BD08B1F9F726
:10BC6000F3B97047F8B50D46D0E900138842044691
:10BC700005D16368C5E900431D6065601DE0002BC8
:10BC8000F7D0986800B16038A2F160073946FFF735
:10BC9000D0FE0028EDDC2668B442EAD0002EE8D0C1
:10BCA000B16801B160393846FFF7C3FE002805DDF1
:10BCB0007368C5E900631D607560F8BD63689E42E6
:10BCC000D7D03668EAE72DE9F84F00258B461446B1
:10BCD0001F4682462E46A8465D4502DB3046BDE83B
:10BCE000F88F4FF02003EFF3118983F31288BFF32D
:10BCF0006F8F9AF80D3003F01F03013B072B0FD80D
:10BD0000DFE803F01E040E0A0E0E0E25DAF81030DE
:10BD10009B682BB1022320E0DAF810301B688BBB44
:10BD200047BB237833B39AF80D3003F01F03013B70
:10BD3000072B30D8DFE803F033282F282F2F2F3898
:10BD4000DAF810309B68002BEAD0012305E0DAF81E
:10BD500010301B6A002BE3D01023DAF80C20CAF84D
:10BD60000880C2F345310B4363F35232CAF80C200A
:10BD700084F8008089F31188BFF36F8F01350AF1D1
:10BD8000140AA9E70423E8E7DAF81000224651462E
:10BD90001030FFF767FFCAF808400136EAE7DAF823
:10BDA000100022465146F4E7DAF8100022465146C8
:10BDB0002430EEE72DE9F843846805460E4644B189
:10BDC0006378012B2ED114F8533C13F002030AD1EF
:10BDD0002370EB68C3F345321643002066F35233F9
:10BDE000A860EB603EE054E90E23B3F1FF3F08BFCB
:10BDF00012F1020F32D0A4F160084046FFF798FE1E
:10BE0000082E0CBF6FF003030023236514F8533C86
:10BE1000DB0609D154F8487C37B94046FFF75CFE91
:10BE20002770D6E7022B01D00023D1E72378002B1F
:10BE3000CFD054F8047C002FF2D04FF00008A4F1CA
:10BE4000140904F11400FFF7C1FEC4F82C80494620
:10BE5000384600F075F884F80080BAE700232370B4
:10BE60006FF00A00BDE8F8831423F0B503FB01006E
:10BE700000244FF48B7601B9F0BD10F8073C40F870
:10BE80000C4C03F01F03082BA0F114070CD826FA62
:10BE900003F3DB0708D550F8143C2BB150F8105CC5
:10BEA0002B605D6040E9054482F31188BFF36F8F1A
:10BEB0004FF02003EFF3118283F31288BFF36F8FEB
:10BEC00001393846D7E710B5D204090201F4F85118
:10BED00002F400220A43017B00240A43C0E9032341
:10BEE000846010BD03460068834208D0D0E9003268
:10BEF00013605A600023C0E90033FFF75BBF70474F
:10BF00000023C0E90000836070470023836070470E
:10BF100083680B60C3681360704770470268012331
:10BF20008B4022EA0303036022FA01F000F00100D3
:10BF3000704720B100221146C030FFF723BE704782
:10BF400037B5019008464FF02003EFF3118583F3D6
:10BF50001288BFF36F8F01A9FCF7D4FD044685F367
:10BF60001188BFF36F8F002809DD4FF02003EFF336
:10BF7000118083F31288BFF36F8FFFF7EDFD20462A
:08BF800003B030BDFAF74EBA20
:08BF8800AC41FF7F0100000045
:10BF9000F54F0000000000000151000010C000003B
:10BFA0004D790000000000007555000028C0000019
:10BFB0007555000040C000006DB500000000000095
:10BFC000EBB3000058C0000009B4000070C00000CE
:10BFD000F961000000000000252E000000000000B4
:10BFE00071B500000000000085890000000000001D
:10BFF0002BAD000088C0000037AF0000A0C00000DB
:10C00000BD0800000000000009130000000000004F
:10C0100016EC000030CB000040CB0000CC04002028
:10C0200054110020DCC100001CEC000058CB0000C3
:10C0300078CB0000D0040020A8110020D6C1000059
:10C0400023EC000068CB000078CB0000D404002073
:10C05000B4110020CEC1000030EC000048CC00003C
:10C06000A0CC0000E004002000020020C8C10000B5
:10C0700037EC000074CC0000A0CC0000E4040020E9
:10C080002C020020C2C100002AEC00009CCB000062
:10C09000E4CB0000D804002018010020BCC100003F
:10C0A0008CCD0000ECCB000040CC0000DC04002074
:08C0B00088010020B4C100006A
:10C0B80027E30000AC000020BC0800207C00002022
:10C0C8000200000054C80000B8080020000000006A
:0CC0D80030E3000038050020E0160020D6
:10C0E4000000000060C3000000000000C8C8000099
:10C0F400000000004CC300000000000088C70000DE
:10C1040000000000F4C700000000000088C3000025
:10C11400000000005CC200000000000078C80000BD
:10C1240000000000A0C80000000000009CC6000041
:10C1340000000000ECCA00000000000010C3000072
:10C1440000000000D4C200000000000084C200000F
:10C15400000000008CC8000000000000B4C800000B
:10C16400000000009CC3000000000000E8C20000C2
:10C174000000000098C2000000000000C0C20000DF
:10C184000000000038C300000000000024C30000C9
:10C1940000000000ACC200000000000074C30000F6
:10C1A4000000000070C2000000000000FCC200009B
:10C1B400030000800080FF7F00800080FF7F0080FC
:10C1C4000080FF7F00800080FF7F008000800700E8
:0EC1D400FF7F00800080FF7F00800080FF7FE3
:0EC1E200FFFFFFFFFFFFFFFFFFFFFFFFFFFF5D
:10C1F0001B5B4A00001B5B4800001B5B324A0000CF
:10C200001B5B4A00001B5B6D00001B3700001B38E6
:10C2100000001B5B3F336C00001B5B4800001B5B96
:10C22000324A00001B3700001B38000000000000ED
:10C230000338FDD87047000049060000A906000039
:10C2400035050000B9050000810700006108000005
:10C25000F1060000950500002508000023D5000028
:10C2600027D50000B0C3000071900000000000005E
:10C270005BD500006DD500000000000059120000E1
:10C2800000000000DBD50000E4D500000000000045
:10C290001512000000000000F5D50000FED50000DA
:10C2A00000000000FD1400000000000007D60000A0
:10C2B00016D6000000000000B111000000000000D0
:10C2C00025D6000034D600000000000059110000FF
:10C2D0000000000043D6000054D60000000000001B
:10C2E000A90E0000000000007BD6000099D60000D7
:10C2F000000000006514000000000000E4D600000B
:10C30000F5D600004CC40000050E0000000000003F
:10C3100012D700001FD70000A4C40000290C0000A1
:10C32000000000003AD7000055D7000000000000D0
:10C33000C11300000000000074D7000085D7000082
:10C340000000000061130000000000009AD7000008
:10C35000A4D70000ECC50000F50A000000000000B2
:10C36000BCD70000C3D70000000000007990000097
:10C3700000000000E3D70000F3D700000000000039
:10C38000F91000000000000028D8000034D8000098
:10C390000000000099100000000000007DD800009F
:10C3A0008BD80000000000003910000000000000E1
:10C3B00000000000B8C30000FED8000006D900004D
:10C3C0000000000055150000000000004AD90000E0
:10C3D00052D9000008C40000759000000000000061
:10C3E00086D9000093D9000000000000A1150000CC
:10C3F000000000000000000000000000000000003D
:10C4000000000000000000000000000010C4000058
:10C41000CDD90000D3D9000000000000F1120000C7
:10C4200000000000F0D90000F6D900000000000074
:10C43000D912000000000000000000000000000011
:10C4400000000000000000000000000000000000EC
:10C4500054C4000012DA000021DA000000000000DD
:10C46000850E00000000000049DA00005ADA0000E2
:10C4700000000000610E00000000000084DA0000EF
:10C4800095DA0000000000003D0E000000000000F2
:10C49000000000000000000000000000000000009C
:10C4A0000000000000000000ACC40000BFDA000083
:10C4B000C7DA000000000000E90D000000000000E5
:10C4C000D8DA0000E0DA000000000000CD0D000026
:10C4D00000000000F1DA0000F9DA000000000000BE
:10C4E000B10D0000000000000ADB000012DB0000BC
:10C4F00000000000950D00000000000023DB00009C
:10C500002BDB000000000000790D0000000000009F
:10C510003CDB000044DB0000000000005D0D00007B
:10C520000000000055DB00005DDB000000000000A3
:10C53000410D0000000000006EDB000076DB000013
:10C5400000000000250D00000000000086DB000058
:10C550008EDB000000000000090D0000000000005C
:10C560009FDB0000A7DB000000000000ED0C0000D6
:10C5700000000000B8DB0000C1DB0000000000008C
:10C58000D10C000000000000D3DB0000DCDB000069
:10C5900000000000B50C000000000000EEDB000011
:10C5A000F7DB000000000000990C00000000000014
:10C5B00009DC000012DC0000000000007D0C00001F
:10C5C0000000000024DC00002DDC00000000000062
:10C5D000610C0000000000000000000000000000EE
:10C5E000000000000000000000000000000000004B
:10C5F000F4C500003FDC000049DC00000000000042
:10C60000050C00000000000070DC00007ADC000077
:10C6100000000000E10B000000000000A1DC0000B1
:10C62000ABDC000000000000BD0B000000000000BB
:10C63000C9DC0000D3DC000000000000990B000002
:10C6400000000000F1DC0000FFDC00000000000042
:10C65000750B00000000000036DD000044DD000026
:10C6600000000000510B0000000000007BDD000016
:10C670008EDD0000000000002D0B00000000000017
:10C6800000000000000000000000000000000000AA
:10C6900000000000008000400004000011E00000E5
:10C6A00018E00000B0C6000000000000000000001C
:10C6B00000000000B8C6000028E000002FE00000E5
:10C6C00000000000D9280000000000003EE000004B
:10C6D00045E0000044C7000000000000000000002A
:10C6E0004DE0000054E00000000000007D28000044
:10C6F000000000006EE0000076E000000000000096
:10C7000081270000000000008BE0000092E00000A4
:10C71000000000005527000000000000A1E000001C
:10C72000A9E0000000000000292700000000000030
:10C7300000000000000000000000000000000000F9
:10C7400000000000000000004CC70000B9E000003D
:10C75000BEE0000000000000F796000000000000AE
:10C76000CBE00000D0E0000000000000EF960000E9
:10C7700000000000000000000000000000000000B9
:10C7800000000000000000005FE1000066E1000022
:10C790009CC7000000000000000000000000000036
:10C7A000A4C7000091E1000076E100000000000055
:10C7B000852A00000000000098E100009DE10000D3
:10C7C00000000000992900000000000000000000A7
:10C7D0000000000000000000000000000000000059
:10C7E00010C0000088C0000088C00000B8C0000071
:10C7F000B8C000009FE20000A6E2000008C80000E8
:10C80000192B0000000000000000000010C800000C
:10C81000F0D50000E0E20000000000004D2D000017
:10C820000201000000000000000000000000000005
:10C8300000000000000000003A000000592E000037
:10C8400009970000259700004B97000039970000DA
:10C8500000000000661600201E0000006DA1000010
:10C86000B8C0000074000020CC0B002000000000C5
:10C87000D4000020B400002057E6000015E60000B8
:10C8800000000000E13A000001000000EFE60000B7
:10C89000F6E60000DCC80000A54100000101000030
:10C8A0009BE70000A3E7000000000000D540000067
:10C8B00001000000B4E70000BAE700000CC9000066
:10C8C0000000000000000000E0E70000E6E70000D4
:10C8D00000000000714100000100000000000000A5
:10C8E000E4C80000F4E70000FCE7000000000000DE
:10C8F0009540000001000000000000000000000062
:10C900000000000000000000000000000000000027
:10C9100014C9000040E800004FE8000078C900009A
:10C920000000000000000000FFE8000006E9000031
:10C9300044CA000000000000000000001DE90000E3
:10C9400022E9000000CA00001941000001010000B6
:10C9500035E900003BE90000BCC900000000000010
:10C9600000000000000000000000000000000000C7
:10C9700000000000000000000000000080C900006E
:10C980004DE9000057E9000000000000B9A30000D5
:10C99000010000008FE9000096E90000000000009F
:10C9A000DBA3000001000000000000000000000008
:10C9B0000000000000000000000000000000000077
:10C9C000C4C90000CDE90000D3E900000000000068
:10C9D00097A300000100000001EA000006EA000041
:10C9E00000000000BD400000010000000000000049
:10C9F0000000000000000000000000000000000037
:10CA00000000000008CA00007DE6000032EA0000D5
:10CA100000000000FDA300000100000078D6000027
:10CA200071EA00000000000063A4000001000000A3
:10CA300000000000000000000000000000000000F6
:10CA400000000000000000004CCA00007DE600006D
:10CA500084EA0000000000001FA4000001000000A4
:10CA600078D600009CEA00000000000041A400000D
:10CA700001000000000000000000000000000000B5
:10CA80000000000000000000000000007FA6000081
:10CA9000100100200801002000010020000000001B
:10CAA000F8000020C5470000D946000021470000DB
:10CAB00079470000000000200000000000000B0685
:10CAC00002000000C8CA00000000000058EB00008F
:10CAD000260002070000002060EB000022000B117E
:10CAE0008D5000005D50000000000000DFEB0000F2
:10CAF000F1EB000000CB00004552000000000000F8
:10CB00000000000008CB000008EC00000FEC000063
:10CB1000000000004552000001000000000000007D
:10CB20000000000000000000000000000000000005
:10CB3000A95100006D530000A5AB0000ABAB000095
:10CB40000952000021AB000085AB0000000000008E
:10CB500095AA000000000000FFFF00000003005045
:10CB60000000000001000000FFFFFFFF0000005078
:10CB70000000000000000000F9550000B7AB000005
:10CB8000C5AB0000DBAB0000E7AB0000F3AB00007F
:10CB9000A154000005AC000000000000003000407F
:10CBA00000000000000000FF00FF00000000000087
:10CBB0000000000101000000BCCB0000003000407C
:10CBC000C8CB000001000000D0CB00000300000033
:10CBD0001B0004001A0005001D00060000000000F4
:10CBE00000000000C157000007AD000000F0024047
:10CBF00000000000FFFF00000048E801000000FF07
:10CC00000000FF0000000000000000FF0200000123
:10CC10000100000018CC000000F0024024CC00000D
:10CC2000010000002CCC0000030000000C000400F8
:10CC30000E0006000D00050040C000000F000100BE
:10CC4000C55A000013AF0000008002400000000041
:10CC50000000000058CC00000080024064CC0000BE
:10CC6000010000006CCC0000020000000400000085
:10CC7000C50001000020004000000000000000008E
:10CC800084CC00000020004090CC00000100000097
:10CC900098CC00000200000016000000D100010046
:10CCA0008FB00000B55E000081B00000515D000053
:10CCB00071B0000021B20000B5B00000E1B000008A
:10CCC0000FB1000019B1000053B100005FB10000C6
:10CCD00019B1000043B100006BB1000079B1000050
:10CCE00087B10000BDB10000C1B1000090BF0000DD
:10CCF000D0BF0000D8BF000000C0000010C000007E
:10CD0000F5FFFFFFFF8FFFFFFF8FFFFFFE8FFFFF8E
:10CD1000FE8FFFFFFD8FFFFFFC8FFFFFFC8FFFFFEC
:10CD20006D757465785F667265652063616C6C65AE
:10CD3000642077697468204E554C4C207061726194
:10CD40006D6574657200000043616E277420696E22
:10CD5000697469616C697A65206D757465782C20D9
:10CD6000776173204E554C4C0D0A0000436F756C73
:10CD700064206E6F74206C6F636B20706F776572C8
:10CD80002073617665206D75746578005350495F36
:10CD900033005374617274696E6720526164696F05
:10CDA0002054657374206578616D706C650A005558
:10CDB0006E61626C6520746F2067657420746865AD
:10CDC00020436C6F636B206D616E616765720A0052
:10CDD000436C6F636B207265717565737420666157
:10CDE000696C65643A2025640A00436C6F636B20AC
:10CDF000636F756C64206E6F74206265207374615C
:10CE0000727465643A2025640A00436C6F636B207A
:10CE100068617320737461727465640A0025733AE3
:10CE20002062616420706172616D65746572732047
:10CE3000636F756E740A00556B6E6F776E2061724A
:10CE400067756D656E743A2025730A004E52465F11
:10CE5000524144494F5F4D4F44455F494545453830
:10CE600030323135345F3235304B42495400446101
:10CE7000746120726174653A2025730A004E52462F
:10CE80005F524144494F5F4D4F44455F424C455FBF
:10CE90004C523530304B424954004E52465F52415D
:10CEA00044494F5F4D4F44455F424C455F4C5231C2
:10CEB00032354B424954004E52465F524144494F2D
:10CEC0005F4D4F44455F424C455F324D42495400EF
:10CED0004E52465F524144494F5F4D4F44455F4279
:10CEE0004C455F314D424954004E52465F524144D9
:10CEF000494F5F4D4F44455F4E52465F324D424968
:10CF000054004E52465F524144494F5F4D4F444595
:10CF10005F4E52465F314D4249540025733A2062BC
:10CF2000616420706172616D657465727320636FF6
:10CF3000756E742E0A00524144494F5F5458504F49
:10CF40005745525F5458504F5745525F4E656734AE
:10CF50003064426D00545820706F7765723A202516
:10CF6000730A00524144494F5F5458504F5745523D
:10CF70005F5458504F5745525F4E65673330644297
:10CF80006D00524144494F5F5458504F5745525FCE
:10CF90005458504F5745525F4E6567323064426D6A
:10CFA00000524144494F5F5458504F5745525F54C7
:10CFB00058504F5745525F4E6567313664426D0099
:10CFC000524144494F5F5458504F5745525F54584F
:10CFD000504F5745525F4E6567313264426D005283
:10CFE0004144494F5F5458504F5745525F54585031
:10CFF0004F5745525F4E65673864426D0052414459
:10D00000494F5F5458504F5745525F5458504F57EF
:10D0100045525F4E65673464426D00524144494F4A
:10D020005F5458504F5745525F5458504F574552D0
:10D030005F3064426D00524144494F5F5458504F35
:10D040005745525F5458504F5745525F506F733297
:10D0500064426D00524144494F5F5458504F574508
:10D06000525F5458504F5745525F506F733364426C
:10D070006D00524144494F5F5458504F5745525FDD
:10D080005458504F5745525F506F733464426D008F
:10D09000524144494F5F5458504F5745525F54587E
:10D0A000504F5745525F506F733564426D00524187
:10D0B00044494F5F5458504F5745525F5458504F52
:10D0C0005745525F506F733664426D005241444978
:10D0D0004F5F5458504F5745525F5458504F574523
:10D0E000525F506F733764426D00524144494F5F45
:10D0F0005458504F5745525F5458504F5745525F00
:10D10000506F733864426D00556B6E6F776E20619F
:10D110007267756D656E743A2025732E0A0054523D
:10D12000414E534D49545F5041545445524E5F3126
:10D1300031303031313030005472616E736D69734B
:10D1400073696F6E207061747465726E3A20257316
:10D150000A005452414E534D49545F504154544576
:10D16000524E5F3131313130303030005452414E07
:10D17000534D49545F5041545445524E5F52414EB5
:10D18000444F4D00506172616D65746572733A0A67
:10D190000044617461207261746520756E6B6E6FFE
:10D1A000776E206F72206465707265636174656468
:10D1B0003A2025640A0D0A00545820706F77657272
:10D1C00020756E6B6E6F776E3A2025640A0054727C
:10D1D000616E736D697373696F6E207061747465CD
:10D1E000726E20756E6B6E6F776E3A2025640A0042
:10D1F0005374617274204368616E6E656C3A2025C9
:10D200006868750A456E64204368616E6E656C3AA5
:10D2100020256868750A54696D65206F6E20656108
:10D220006368206368616E6E656C3A202575206DB9
:10D23000730A44757479206379636C653A202575A7
:10D240002070657263656E740A0A004368616E6ED1
:10D25000656C206D757374206265206265747765F6
:10D26000656E203020616E642038300A005374618E
:10D270007274206368616E6E656C207365742074CF
:10D280006F3A2025640A00456E64206368616E6E03
:10D29000656C2073657420746F3A2025640A00441D
:10D2A000656C61792074696D65206D757374206299
:10D2B00065206265747765656E203020616E64203C
:10D2C0003939206D730A0044656C61792074696D89
:10D2D000652073657420746F3A2025640A005258E3
:10D2E0002073776565700A00545820737765657000
:10D2F0000A00546865206D6F64756C617465642004
:10D300005458206861732066696E69736865640AA1
:10D31000005265636569766564207061796C6F6140
:10D32000643A0A004E756D626572206F6620706106
:10D33000636B6574733A2025640A00496E76616CEC
:10D34000696420444344432076616C7565207072A3
:10D350006F76696465640A0044434443205644443C
:10D36000482073746174652025640A577269746576
:10D370002027302720746F20746F67676C652073D7
:10D3800074617465206F66204443444320524547CE
:10D39000300A57726974652027312720746F207412
:10D3A0006F67676C65207374617465206F662044D5
:10D3B00043444320524547310A00444344432073C9
:10D3C000746174652025640A577269746520273179
:10D3D00027206F722027302720746F20746F6767B3
:10D3E0006C650A00414E54312064697361626C655A
:10D3F000642C20414E543220656E61626C65640A73
:10D4000000414E543120656E61626C65642C204190
:10D410004E54322064697361626C65640A00466F21
:10D420007220257320636F6E6669672E6D6F646569
:10D43000206368616E6E656C206D75737420626523
:10D44000206265747765656E20256420616E6420B6
:10D4500025640A004368616E6E656C2073657420F4
:10D46000746F2025640A00537461727420746865B7
:10D4700020545820636172726965720A00537461A6
:10D48000727420746865206D6F64756C6174656476
:10D4900020545820636172726965720A0044757481
:10D4A00079206379636C65206D75737420626520E3
:10D4B0006265747765656E203120616E6420393055
:10D4C0002E0A0046726F6E742D656E64206D6F6457
:10D4D000756C65202846454D292054782067616980
:10D4E0006E2073657420746F2025640A0046726F85
:10D4F0006E742D656E64206D6F64756C65202846B2
:10D50000454D292061637469766174696F6E20648A
:10D51000656C61792073657420746F2025642075B3
:10D52000730A0066656D0053657420746865206633
:10D53000726F6E742D656E64206D6F64756C6520FE
:10D540002846454D2920706172616D65746572735E
:10D55000203C7375625F636D643E00746F67676C37
:10D56000655F646364635F737461746500546F67BF
:10D57000676C652044434443207374617465203CA8
:10D5800073746174653E2C206966207374617465E0
:10D59000203D2031207468656E20746F67676C656C
:10D5A0002044432F44432073746174652C206F72B0
:10D5B000206966207374617465203D203020746892
:10D5C000656E20746F67676C652044432F44432069
:10D5D00056444448207374617465007072696E74B7
:10D5E0005F7278005072696E7420525820706179B1
:10D5F0006C6F61640073746172745F72780053744D
:10D600006172742052580073746172745F74785F31
:10D610007377656570005374617274205458207379
:10D62000776565700073746172745F72785F737789
:10D630006565700053746172742052582073776569
:10D64000657000706172616D65746572735F707290
:10D65000696E74005072696E742063757272656EC3
:10D66000742064656C61792C206368616E6E656CF2
:10D6700020616E6420736F206F6E0073746172742A
:10D680005F647574795F6379636C655F6D6F6475F2
:10D690006C617465645F7478004475747920637993
:10D6A000636C6520696E2070657263656E742028F6
:10D6B00074776F20646563696D616C206469676964
:10D6C00074732C206265747765656E20303120613B
:10D6D0006E6420393029203C647574795F63796306
:10D6E0006C653E007472616E736D69745F70617415
:10D6F0007465726E0053657420746865207472617D
:10D700006E736D697373696F6E2070617474657286
:10D710006E006F75747075745F706F776572004F0F
:10D72000757470757420706F7765722073657420DE
:10D730003C7375625F636D643E0073746172745F05
:10D7400074785F6D6F64756C617465645F6361723A
:10D750007269657200537461727420746865206D1B
:10D760006F64756C617465642054582063617272D3
:10D770006965720073746172745F74785F6361725B
:10D780007269657200537461727420746865205404
:10D7900058206361727269657200646174615F72BE
:10D7A00061746500536574206461746120726174F2
:10D7B00065203C7375625F636D643E0063616E63F8
:10D7C000656C0043616E63656C20746865207377D7
:10D7D000656570206F72207468652063617272697C
:10D7E00065720074696D655F6F6E5F6368616E6E10
:10D7F000656C0054696D65206F6E206561636820FB
:10D800006368616E6E656C20696E206D732028629E
:10D8100065747765656E203120616E642039392921
:10D82000203C74696D653E00656E645F6368616E7F
:10D830006E656C00456E64206368616E6E656C2079
:10D84000666F72207468652073776565702028693B
:10D850006E204D487A206173206469666665726542
:10D860006E63652066726F6D2032343030204D4813
:10D870007A29203C6368616E6E656C3E007374614A
:10D8800072745F6368616E6E656C0053746172746C
:10D89000206368616E6E656C20666F7220746865C7
:10D8A000207377656570206F7220746865206368E7
:10D8B000616E6E656C20666F722074686520636FA0
:10D8C0006E7374616E742063617272696572202870
:10D8D000696E204D487A20617320646966666572BE
:10D8E000656E63652066726F6D2032343030204D76
:10D8F000487A29203C6368616E6E656C3E007478DE
:10D900005F6761696E005365742074686520667294
:10D910006F6E742D656E64206D6F64756C65202864
:10D9200046454D29205478206761696E20696E2034
:10D93000616E2061726269747261727920756E69BC
:10D940007473203C6761696E3E00616E74656E6E33
:10D95000610053656C656374207468652066726F3E
:10D960006E742D656E64206D6F64756C652028463D
:10D97000454D2920616E74656E6E61203C73756241
:10D980005F636D643E006163746976655F64656CB6
:10D99000617900536574207468652066726F6E74D7
:10D9A0002D656E64206D6F64756C65202846454D4D
:10D9B000292061637469766174696F6E2064656C97
:10D9C0006179203C74696D652075733E00616E74E9
:10D9D0005F3100414E543120656E61626C65642C8C
:10D9E00020414E54322064697361626C65642E007C
:10D9F000616E745F3200414E54312064697361621C
:10DA00006C65642C20414E543220656E61626C65F9
:10DA100064007061747465726E5F72616E646F6DC4
:10DA20000053657420746865207472616E736D694B
:10DA30007373696F6E207061747465726E20746F99
:10DA40002072616E646F6D2E007061747465726E09
:10DA50005F313131313030303000536574207468BB
:10DA600065207472616E736D697373696F6E207077
:10DA700061747465726E20746F20313131313030D1
:10DA800030302E007061747465726E5F31313030E9
:10DA900031313030005365742074686520747261D0
:10DAA0006E736D697373696F6E20706174746572E3
:10DAB0006E20746F2031303130313031302E0070B3
:10DAC0006F733864426D00545820706F7765723AF6
:10DAD000202B382064426D00706F733764426D00F4
:10DAE000545820706F7765723A202B372064426D4E
:10DAF00000706F733664426D00545820706F776504
:10DB0000723A202B362064426D00706F7335644288
:10DB10006D00545820706F7765723A202B35206461
:10DB2000426D00706F733464426D00545820706F02
:10DB30007765723A202B342064426D00706F733326
:10DB400064426D00545820706F7765723A202B3311
:10DB50002064426D00706F733264426D005458202F
:10DB6000706F7765723A202B322064426D00706FBF
:10DB7000733064426D00545820706F7765723A209C
:10DB8000302064426D006E65673464426D00545805
:10DB900020706F7765723A202D342064426D006EDC
:10DBA00065673864426D00545820706F7765723A2B
:10DBB000202D382064426D006E6567313264426DFD
:10DBC00000545820706F7765723A202D31322064EE
:10DBD000426D006E6567313664426D0054582070A6
:10DBE0006F7765723A202D31362064426D006E6584
:10DBF00067323064426D00545820706F7765723A16
:10DC0000202D32302064426D006E656733306442EF
:10DC10006D00545820706F7765723A202D33302094
:10DC200064426D006E6567343064426D0054582064
:10DC3000706F7765723A202D34302064426D006E2B
:10DC400072665F314D6269740031204D6269742FD4
:10DC500073204E6F726469632070726F70726965B1
:10DC60007461727920726164696F206D6F64650000
:10DC70006E72665F324D6269740032204D62697463
:10DC80002F73204E6F726469632070726F707269B7
:10DC9000657461727920726164696F206D6F64656B
:10DCA00000626C655F314D6269740031204D6269BC
:10DCB000742F7320426C7565746F6F7468204C6F9D
:10DCC0007720456E6572677900626C655F324D62E0
:10DCD00069740032204D6269742F7320426C75653F
:10DCE000746F6F7468204C6F7720456E657267792A
:10DCF00000626C655F6C723132354B626974004C46
:10DD00006F6E672072616E676520313235206B62FD
:10DD100069742F732054582C20313235206B62697E
:10DD2000742F7320616E6420353030206B6269740B
:10DD30002F7320525800626C655F6C723530304B27
:10DD4000626974004C6F6E672072616E6765203582
:10DD50003030206B6269742F732054582C2031327C
:10DD600035206B6269742F7320616E64203530300A
:10DD7000206B6269742F732052580069656565389D
:10DD800030323135345F3235304B62697400494589
:10DD90004545203830322E31352E342D3230303654
:10DDA00020323530206B6269742F730025643A206D
:10DDB0006F7574206F662072616E67652046454DF1
:10DDC000206761696E2076616C7565206F722073C3
:10DDD000657474696E67206761696E206973206E6F
:10DDE0006F7420737570706F727465640A00556E7D
:10DDF00065787065637465642074657374207479E4
:10DE000070653A2025640A006E7266785F74696DE9
:10DE100065725F696E6974206661696C65642077FC
:10DE20006974683A2025640A0000000100000008B7
:10DE3000042008044010000000000000000020281A
:10DE40006E696C29004661696C656420746F20728C
:10DE500065626F6F743A207370696E6E696E6720C9
:10DE6000656E646C6573736C792E2E2E0A005A658C
:10DE7000706879722076657273696F6E2025642EE2
:10DE800025642E25640A00557074696D653A202555
:10DE900075206D730A005363686564756C65723A2A
:10DEA0002025752073696E6365206C61737420632F
:10DEB000616C6C0A00546872656164733A0A002AE6
:10DEC000004E41002573257020252D3130730A0046
:10DED000096F7074696F6E733A20307825782C2042
:10DEE0007072696F726974793A2025642074696D63
:10DEF000656F75743A20256C6C640A00097374614F
:10DF000074653A2025732C20656E7472793A202549
:10DF1000700A00556E61626C6520746F20646574D0
:10DF200065726D696E6520756E75736564207374B6
:10DF300061636B2073697A6520282564290A0A00C9
:10DF400009737461636B2073697A6520257A752C77
:10DF500020756E7573656420257A752C2075736144
:10DF6000676520257A75202F20257A75202825754C
:10DF7000202525290A0A00257020495251202530E4
:10DF800032642020202020287265616C2073697A19
:10DF90006520257A75293A09756E757365642025A3
:10DFA0007A7509757361676520257A75202F20259C
:10DFB0007A752028257A75202525290A006379633A
:10DFC0006C65733A202575206877206379636C65EA
:10DFD000730A00257020252D313073202872656169
:10DFE0006C2073697A6520257A75293A09756E75F2
:10DFF00073656420257A7509757361676520257AD4
:10E0000075202F20257A7520282575202525290A99
:10E01000006B65726E656C004B65726E656C20639B
:10E020006F6D6D616E6473006379636C6573004B33
:10E0300065726E656C206379636C65732E00726522
:10E04000626F6F74005265626F6F742E007374613B
:10E05000636B73004C6973742074687265616473D8
:10E0600020737461636B2075736167652E0074683B
:10E070007265616473004C697374206B65726E65C0
:10E080006C20746872656164732E00757074696DBC
:10E0900065004B65726E656C20757074696D652ED8
:10E0A0000076657273696F6E004B65726E656C20E9
:10E0B00076657273696F6E2E00636F6C6400436FD8
:10E0C0006C64207265626F6F742E007761726D00F0
:10E0D0005761726D207265626F6F742E005B2570E0
:10E0E0005D00202072657175697265733A20257331
:10E0F0000A0052454144590044495341424C454469
:10E1000000646576696365733A0A002D2025730003
:10E1100020282573290A002D2025730A0050524516
:10E12000204B45524E454C20313A0A002D204E6F6F
:10E130006E650A00505245204B45524E454C2032E8
:10E140003A0A00504F53545F4B45524E454C3A0AE1
:10E15000004150504C49434154494F4E3A0A0064E3
:10E1600065766963650044657669636520636F6DF4
:10E170006D616E6473004C69737420636F6E6669C1
:10E18000677572656420646576696365732062797A
:10E19000206C6576656C73006C697374004C6973F0
:10E1A0007420636F6E666967757265642064657656
:10E1B00069636573005573696E67206461746120DB
:10E1C00077696474682025640A00496E636F72720F
:10E1D00065637420646174612077696474680A00FF
:10E1E000526561642076616C756520307825780A07
:10E1F0000057726974696E672076616C75652030AE
:10E200007825780A006465766D656D206C6F6164B1
:10E2100020737570706F7274732073657474696E97
:10E220006720627970617373206F6E20612073695B
:10E230006E676C6520696E7374616E63652E0A008B
:10E240004C6F6164696E672E2E2E0A70726573734F
:10E25000206374726C2D78206374726C2D7120743D
:10E260006F206573636170650A004E756D6265723B
:10E27000206F6620627974657320726561643A204C
:10E2800025640A002D2D002D6500556E6B6E6F778D
:10E290006E206F7074696F6E20222573220A0064ED
:10E2A00065766D656D00526561642F77726974657E
:10E2B00020706879736963616C206D656D6F727928
:10E2C000226465766D656D20616464726573732088
:10E2D0005B7769647468205B76616C75655D5D0071
:10E2E00055736167653A0A6465766D656D206C6F7C
:10E2F0006164205B6F7074696F6E735D205B616435
:10E3000064726573735D0A4F7074696F6E733A0A55
:10E310002D65096C6974746C652D656E6469616E38
:10E3200020706172736500756172743A7E242000FA
:10E330007368656C6C5F7561727400537562636FAE
:10E340006D6D616E64733A0A005741524E494E47F3
:10E350003A2041207072696E742072657175657320
:10E360007420776173206465746563746564206FDD
:10E370006E206E6F742061637469766520736865C2
:10E380006C6C206261636B656E642E0A006E6F7444
:10E39000207465726D696E617465643A2025630A44
:10E3A00000506C65617365207370656369667920E0
:10E3B0006120737562636F6D6D616E642E0A004536
:10E3C00072726F723A20726571756573746564203C
:10E3D0006D756C7469706C652066756E6374696FB9
:10E3E0006E20657865637574696F6E730A003A20F4
:10E3F000636F6D6D616E64206E6F7420666F756EF5
:10E400006400546F6F206D616E7920617267756D65
:10E41000656E747320696E2074686520636F6D6D1E
:10E42000616E642E0A0025733A2077726F6E672042
:10E43000706172616D6574657220636F756E740AC8
:10E44000000A25732573005368656C6C207468722C
:10E45000656164206572726F723A20256400506CA9
:10E460006561736520707265737320746865203C04
:10E470005461623E20627574746F6E20746F2073F5
:10E48000656520616C6C20617661696C61626C65A8
:10E4900020636F6D6D616E64732E0A00596F752075
:10E4A00063616E20616C736F20757365207468659D
:10E4B000203C5461623E20627574746F6E20746FEC
:10E4C0002070726F6D7074206F72206175746F2D83
:10E4D000636F6D706C65746520616C6C20636F6D2B
:10E4E0006D616E6473206F7220697473207375623E
:10E4F000636F6D6D616E64732E0A00596F752063D2
:10E50000616E2074727920746F2063616C6C20637B
:10E510006F6D6D616E64732077697468203C2D683F
:10E520003E206F72203C2D2D68656C703E2070611E
:10E5300072616D6574657220666F72206D6F7265B1
:10E5400020696E666F726D6174696F6E2E0A000AC3
:10E550005368656C6C20737570706F72747320668D
:10E560006F6C6C6F77696E67206D6574612D6B657C
:10E5700079733A0A20204374726C202B2028612082
:10E580006B65792066726F6D3A20616263646566BF
:10E590006B6C6E707577290A2020416C7420202BDB
:10E5A000202861206B65792066726F6D3A20626663
:10E5B000290A506C65617365207265666572207406
:10E5C0006F207368656C6C20646F63756D656E7425
:10E5D0006174696F6E20666F72206D6F7265206462
:10E5E000657461696C732E0A000A417661696C6119
:10E5F000626C6520636F6D6D616E64733A0A00250D
:10E600003038583A20002530327820002020200071
:10E610007C007C0A005072696E74732074686520F7
:10E6200068656C70206D6573736167652E001B5B98
:10E6300025642563001B5B313B3325646D001B5B48
:10E6400034303325646D002573252D2A730025731E
:10E650003A002D68002D2D68656C7000202D20007B
:10E660002020004C6F7374206C6F67733A20256C08
:10E67000750A005B2533645D2025730A006F6666AA
:10E680000025733A257325730A0020756E6B6E6F33
:10E69000776E20706172616D657465723A20004515
:10E6A00063686F207374617475733A2025730A0070
:10E6B0004E6F20726573706F6E73652066726F6D3A
:10E6C00020746865207465726D696E616C2C2061C0
:10E6D0007373756D656420383078323420736372DB
:10E6E00065656E2073697A650A001B5B366E007281
:10E6F0006573697A6500436F6E736F6C652067653B
:10E700007473207465726D696E616C2073637265D9
:10E71000656E2073697A65206F7220617373756D01
:10E7200065732064656661756C7420696E20636131
:10E7300073652074686520726561646F7574206606
:10E7400061696C732E204974206D75737420626545
:10E7500020657865637574656420616674657220F0
:10E7600065616368207465726D696E616C2077699C
:10E77000647468206368616E676520746F20656EDD
:10E780007375726520636F72726563742074657847
:10E790007420646973706C61792E00686973746F9A
:10E7A000727900436F6D6D616E6420686973746F78
:10E7B00072792E007368656C6C0055736566756CB4
:10E7C0002C206E6F7420556E69782D6C696B6520F6
:10E7D0007368656C6C20636F6D6D616E64732E0081
:10E7E000636C65617200436C65617220736372656E
:10E7F000656E2E0064656661756C74004173737597
:10E800006D652038302063686172732073637265B0
:10E81000656E20776964746820616E642073656E2C
:10E820006420746869732073657474696E672074FA
:10E830006F20746865207465726D696E616C2E005E
:10E840006261636B73706163655F6D6F64650054D3
:10E850006F67676C65206261636B737061636520CD
:10E860006B6579206D6F64652E0A536F6D6520743A
:10E8700065726D696E616C7320617265206E6F7474
:10E880002073656E64696E67207365706172617470
:10E89000652065736361706520636F646520666FD2
:10E8A00072206261636B737061636520616E6420C6
:10E8B00064656C65746520627574746F6E2E205487
:10E8C00068697320636F6D6D616E6420666F72633B
:10E8D0006573207368656C6C20746F20696E746555
:10E8E00072707265742064656C657465206B6579FF
:10E8F000206173206261636B73706163652E0063D6
:10E900006F6C6F727300546F67676C6520636F6C18
:10E910006F7265642073796E7461782E0065636828
:10E920006F00546F67676C65207368656C6C206559
:10E9300063686F2E007374617473005368656C6C48
:10E9400020737461746973746963732E0062616308
:10E950006B737061636500536574206469666665F6
:10E9600072656E742065736361706520636F6465A2
:10E9700020666F72206261636B73706163652061F2
:10E980006E642064656C657465206B65792E006427
:10E99000656C6574650053657420746865207361E7
:10E9A0006D652065736361706520636F64652066C3
:10E9B0006F72206261636B737061636520616E6466
:10E9C0002064656C657465206B65792E00726573D3
:10E9D0006574005265736574207368656C6C207390
:10E9E00074617469737469637320666F72207468EC
:10E9F00065204C6F67676572206D6F64756C652E5E
:10EA00000073686F7700476574207368656C6C20CD
:10EA10007374617469737469637320666F722074B0
:10EA20006865204C6F67676572206D6F64756C65F3
:10EA30002E0044697361626C65207368656C6C209C
:10EA40006563686F2E2045646974696E67206B6525
:10EA5000797320616E64206D6574612D6B657973C7
:10EA600020617265206E6F742068616E646C6564ED
:10EA700000456E61626C65207368656C6C2065632F
:10EA8000686F2E0044697361626C6520636F6C6F00
:10EA90007265642073796E7461782E00456E6162D0
:10EAA0006C6520636F6C6F7265642073796E74613E
:10EAB000782E00436F6D6D616E64206275666665C9
:10EAC0007220697320746F6F2073686F7274207482
:10EAD0006F20657870616E6420616C6C20636F6D6F
:10EAE0006D616E6473206D61746368696E67207711
:10EAF000696C6463617264207061747465726E3AEB
:10EB00002025730A006D757465785F696E697420DD
:10EB100063616C6C65642077697468204E554C4C59
:10EB200020706172616D6574657200436F756C640D
:10EB3000206E6F7420616C6C6F63617465206D75FD
:10EB4000746578206265666F726520696E697469A4
:10EB5000616C697A696E6700464C4153485F3000CA
:10EB60005352414D5F30006E6F7420004846206361
:10EB70006C6F636B3A0A00092D20257372756E6EF7
:10EB8000696E67202875736572733A202575290AA6
:10EB900000092D206C6173742073746172743A20C3
:10EBA0002575206D7320282575206D732061676F92
:10EBB000290A00092D206C6173742073746F703AF8
:10EBC000202575206D7320282575206D73206167C1
:10EBD0006F290A004C4620636C6F636B3A0A006E23
:10EBE00072665F636C6F636B5F636F6E74726F6C82
:10EBF00000436C6F636B20636F6E74726F6C206385
:10EC00006F6D6D616E64730073746174757300531E
:10EC1000746174757300434C4F434B004750494F28
:10EC20005F31004750494F5F30005350495F30001B
:10EC3000554152545F3100554152545F300000003D
:10EC40000000000101000000000069646C65006DB7
:10EC500061696E00756E6B6E6F776E0070656E64C5
:10EC6000696E6700707265737461727400646561C7
:10EC7000640073757370656E6465640061626F72C1
:10EC800074696E67007175657565640064756D6D96
:0CEC90007900737973776F726B7100006C
:10EC9C000000000000127A000001000000000000DB
:10ECAC0040C000000F000100000000000000000048
:10ECBC0000000000000000000000000040C0000048
:10ECCC000800000040C000000700000028C0000041
:10ECDC000900000040C00000060000000000000019
:10ECEC0000A00040010400000003000050000000E0
:10ECFC000A0000003200000000000000FF000000CD
:10ED0C00DD90000000000000010000008C000020DD
:10ED1C00000000000000000000000000C0300020D7
:10ED2C0000000000000000000000000000000000D7
:10ED3C000000000000000000000200003CC80000C1
:10ED4C0068C80000C0320020000000000000000075
:10ED5C0000000000000000000000000000000000A7
:10ED6C004000000000330020000000000000000004
:10ED7C000000000000000000000000000000000087
:10ED8C0008000000FFFFFFFFFC0400200100000052
:10ED9C001005002001000000E80400200100000024
:10EDAC00240500200100000000000000000000000D
:10EDBC00DCCB00000000000028010020280100200E
:10EDCC000000000001000000380100203801002084
:10EDDC004001002040010020000000000100000064
:10EDEC005001002050010020000000000000000035
:10EDFC000000000000000000000000000000000007
:10EE0C0000000000000000000000000088C00000AE
:10EE1C0000000000000000000000000000000000E6
:10EE2C0038CC00000100000098010020980100205F
:10EE3C000000000001000000A8010020A801002033
:10EE4C00B0010020B0010020000000000100000013
:10EE5C00C0010020C00100200000000000000000E4
:10EE6C000000000000000000000000000000000096
:10EE7C00000000000000000000000000A0C0000026
:10EE8C000000000000000000000000000000000076
:10EE9C000000000000E10000000103001802002047
:10EEAC000000000000000000000000000000000056
:10EEBC00851600202000000000000000000000006B
:10EECC0000E10000000103004402002000000000EB
:10EEDC00000000000000000000000000A51600204B
:10EEEC0020000000000000000090D0030000000093
:10EEFC000000000000000000000000000000000006
:10EF0C0000000000000000000000000000000000F5
:10EF1C0000000000000000000000000000000000E5
:10EF2C0000000000000000000000000000000000D5
:10EF3C0000000000000000000000000000000000C5
:10EF4C0000000000000000000000000000000000B5
:10EF5C00000000000000000000000000FF000000A6
:10EF6C000000000000000000FFFF0F00DC0200208A
:10EF7C00DC020020E4020020E4020020000000007B
:10EF8C005D8C00008812002011000000598D0000DB
:10EF9C00C58C0000ED8C00002D8D0000300300208E
:10EFAC00F4020020280300200000000020030020B1
:10EFBC008C120020110000009012002011000000A3
:10EFCC009412002011000000100300201C030020EC
:0CEFDC00140300200C0300204003002060
:10EFE8004967000083B50000000000009BA60000F0
:10EFF80070C00000A1B200007171000083B500006C
:10F00800000000009BA60000000000009BA6000076
:10F01800C16C000083B50000000000009BA6000042
:10F028000000000089760000000000009BA6000098
:10F03800000000009BA60000000000009BA6000046
:10F04800000000009BA60000000000009BA6000036
:10F05800000000009BA60000000000009BA6000026
:10F06800000000009BA6000000000000796200007C
:10F07800000000009BA60000000000009BA6000006
:10F08800000000009BA60000000000009BA60000F6
:10F09800000000009BA60000000000009BA60000E6
:10F0A800000000009BA60000000000009BA60000D6
:10F0B800000000009BA60000000000009BA60000C6
:10F0C800000000009BA60000000000009BA60000B6
:10F0D800000000009BA60000000000009BA60000A6
:10F0E800000000009BA60000000000009BA6000096
:10F0F800000000009BA60000000000009BA6000086
:10F10800000000009BA60000000000009BA6000075
:10F11800000000009BA60000000000009BA6000065
:10F1280058C00000A1B20000000000009BA600002B
:10F13800000000009BA60000000000009BA6000045
:10F14800000000009BA60000000000009BA6000035
:10F15800000000009BA600007D75000083B500003C
:10F168000000000000000000000000000000000097
:0CF178000000000000000000000000008B
:10F18400E8040020E8040020000000000000000063
:10F194000E000000FC040020FC040020000000001D
:10F1A400000000000E0000001005002010050020E3
:10F1B40000000000000000000E00000024050020F4
:10F1C4002405002000000000000000000E000000E4
:0400000300004D1993
:00000001FF
